:020000040000fa
:080000000001040000000000f3
:020000040000fa
:10020000cf2322000e7f22000e0188000000000094
:100210000c000700a0a62500010020001100070027
:10022000000020000000e000020032000000020098
:1002300000000000ee430200000000000040da0071
:100240000000fe004440a90000bb20000000e000c8
:100250000300320000002000a00188004440a800f4
:100260000000060091018800800078000000eb008b
:1002700015003700e280400032a0b4009101ba00be
:10028000e280400032a0b4009102ba00e280400057
:1002900032a0b4000002eb00472bde00f507b200ed
:1002a000602ce10004003a000059eb008301e900f2
:1002b000fdff3e00040037006128e100010032002c
:1002c0000082eb00040007001101ba000200e00008
:1002d000e8ff3a00000006003159ba008301e90046
:1002e0000c0032002159ba008301e90008003200f5
:1002f0000400e00003003a00e280400032a0b400b5
:10030000f5ff370011d9ba008301e900faff3a007e
:100310008100e800e180400032a0b4000000060047
:1003200000000400000000000000040000000000c5
:1003300000000400000000000a4804000000000063
:10034000c872040000000000b07304000000000048
:100350006683040000000000901a04000000000002
:10036000fc1a040000000000421b04000000000012
:10037000a61b0400000000000c1c0400000000008c
:10038000721c040000000000d81c040000000000e3
:100390007a1d040000000000001e040000000000a0
:1003a000861e040000000000341f0400000000004e
:1003b000e01f040000000000d22004000000000044
:1003c0005621040000000000782104000000000015
:1003d0005022040000000000c622040000000000bb
:1003e00020230400000000007a2304000000000025
:1003f00074240400000000009426040000000000a3
:100400001e3d0400000000009e3d040000000000ae
:10041000d43d040000000000043e04000000000081
:100420000040da000000fe003200f8009101880070
:100430000008bb00410424006210e1000400320007
:10044000000220000010e1000a003a0051042400dc
:10045000013b88000500fc0051052000313b88006d
:10046000a10a2000313b880061e7a80000000000dd
:10047000000000003200f900000006003200f80021
:1004800060042400003b8800f2ff37003200f800cf
:100490009101880041002400013b88000208bb0054
:1004a000ecff37003200f800910188005100240071
:1004b000013b8800030120003218bb008301e900e2
:1004c000fdff3a00e3ff37003200f8009101880099
:1004d0008002780062004000e08048003549ba00a0
:1004e0003204e0000410a700100032008301e9008c
:1004f0000e0032002549ba003204e0000410a700c3
:100500000a0032008301e900080032000408a30059
:10051000eeff320015c9ba003204e0000410a70053
:10052000020032008301e900e8ff3a003200f900de
:100530000000060003f0a200889fbe008a9fbe0054
:100540008c1f7800d4010700db0133006450e10008
:100550004f0032006420e1005200320003826c0040
:1005600007003b000905d0000306d000820f5400ad
:100570000c065d000200390002003200890178009b
:10058000030678008582550004003d000003fd004d
:100590008103fd008502ea008b854200840f720012
:1005a00002003b0060001000e08018006011b800fd
:1005b0000005eb007a28e1000a0039000600780007
:1005c000c75ddd00f707b200878075002d0037009a
:1005d000828171000a017800610560008180d1008c
:1005e0000080d3008502e900f9ff3b0006044000cb
:1005f0008784480002003b0060041400e0841c0073
:100600000988a300070032008a817100828171008d
:10061000610164008904d1000884d3008b05e800df
:10062000170037000978a30013003a000b00e00020
:10063000130034008b05e9000804440089844c0051
:100640000a4474000978a3000d003a000b00e00092
:10065000070034008b05e9000804440089844c003d
:1006600001003a000b0020000978a300f7ff3200d8
:100670000001eb0002003700828171000a0178005e
:100680004a0107000cf0a70001f0a0009301370019
:100690006420e10002003a00838f6c009301330074
:1006a0000801be000200be008c013700889fbe001a
:1006b0008a9fbe008c1f780077010700100220007f
:1006c00002003b00706088007b0137008a006200f6
:1006d0006408e10002003a0070608800830137007e
:1006e0006108e100fcff32000800be00030478004e
:1006f0007000070001f0a1000900070008f0a60043
:10070000040037000001be0091042400b0fd200069
:1007100088ff070009f0a70001f0a2006f01370071
:10072000889fbe008a9fbe008c9fbe000004be0052
:10073000440107000800be00890678006420e1003b
:1007400008003900040032000160a00012022000fd
:10075000726088005300370091fc2300b0fd200038
:100760004e0037000006eb0009f0a10003f823005b
:10077000020020000800be009f00070006003400b1
:1007800001f82300000020000801be004900070016
:100790000004be002c0020000800be0093e82300e7
:1007a000320a230094000700120034000801be0042
:1007b000d1fd2300703d2b005fff07000005be0048
:1007c000b3f32300f27a26000800be004a010700b6
:1007d00003f823000200200056ff07000801be00b6
:1007e00055ff07000a01be00320007000004be00ea
:1007f0000c06e8000800be0001f0a1000200200085
:10080000039823007c0007000800be001600350096
:100810000801be00380107000005be0032cd2c00e3
:1008200043fb230044ff0700809fbe00126928009d
:1008300003d52b000a00be002f010700620f210024
:1008400013ef2b003cff07000a01be002a0107003e
:100850004f01be00170007000801be002601070077
:100860000801be0034ff07000c00e0000b0032005e
:100870000c10a70001f0a200b2fd200093fc2300a1
:100880006260e1000400320022a9200063f023002e
:100890000c10a70063f8230027ff07000df0a70046
:1008a00001f0a2004f06be004f05be004f04be007f
:1008b00000000600889fbe008a9fbe008c1f780043
:1008c000f5000700fc00330003866c006450e10073
:1008d0002e0032006420e100330032006150e1005c
:1008e0002f0032006120e100310032008585550083
:1008f000eb07b000090020000804200005003700c5
:100900000804440089844c000a00310006034300b7
:1009100087834b000001530081815b00f8ff3300a7
:100920000203be000800a0000804440089844c00b3
:10093000f6ff3900c639dd00830173000100320083
:10094000130020008904d1000884d3000998a30073
:10095000050032000800a7000300a0008904d100b0
:100960000884d3008b05e8008904d1000884d300f3
:100970000001eb000281d2008c00070001f0a10011
:100980000cf0a70001f0a000d40037006420e100c3
:10099000d60032000801be000200be00f7ff37009b
:1009a0006120e100d10032006000b800f3ff3700a1
:1009b0000000200001f82700f0ff3700839f680047
:1009c0000100e00002003d0060001000e08018001f
:1009d0000300e00002003d0060011100e081190009
:1009e0002e0107004f00e00002003b0060001000f5
:1009f000e0801800000006001400200037013700d6
:100a0000f4ff2f00350137000001be008d00070004
:100a10000470a70003f0a1006509b10016003200c0
:100a20000d0035006828e10006003500f0ff2f00ba
:100a3000f1ff27000300e00013003b000100280045
:100a40000000050000004000818048008502e900a8
:100a5000fcff3a0008003700f88f420002003c001b
:100a60008000eb00000005008100d1000080d30071
:100a70008502e800fcff3a000300e00002003b00b2
:100a800060001000e0801800000006000001be00b9
:100a90006c0007000470a70003f0a10003f8a30096
:100aa00013003a006509b10010003200090035005a
:100ab0006928e1000200350001002800000005005f
:100ac00000004000818048008502e900fcff3a00f8
:100ad00000000600f88f4200050035008100d100bb
:100ae0000080d3008502e800fcff3a000000060009
:100af0008000eb0000000500889fbe008a9fbe00ba
:100b0000010578000100e0000400350008003c0009
:100b10000000e000200032000500370060001000f7
:100b2000e080180002003b0001f02c001a003700a2
:100b30000004be006011b8006b0920000982cf00dc
:100b4000020039000882cf000441b000694252001f
:100b50000e00320008003b008281710061016400d8
:100b60008904d1000884d3008b05e8000442e80022
:100b7000f9ff3a00050037000804440089844c005e
:100b80008b05e9000442e900fbff3a00070007007b
:100b90000af0a70001f0a0004f05be004f04be0000
:100ba0000000060004002000cc0037008100200077
:100bb000618055000b003d000b00200061fe2f00fe
:100bc0000100e1001d0034008281710061016400b8
:100bd0008904d1000884d3000000e800faff3a003d
:100be00071002000610064000300700002006000da
:100bf0000900320061044400e0844c000988a5002b
:100c0000050032008b05e8006808e10002003a00a8
:100c10008904d1000884d300f20f20000258e100bb
:100c200005003d00c75ddd00f907b2008980750051
:100c300008007800000006000bf827008b00780001
:100c400000000500c70ade00f107b200f50fb20090
:100c500008003200e1cf4200020032000170a00023
:100c600024000500810f7000010032000408050017
:100c700044000500810f700002003a0014000500d6
:100c80008502e9000000400081c04800fcff3b00f5
:100c90000170a000240005000004be00e9ff070069
:100ca0000003be000405be000200be00e5ff070011
:100cb000844f7500000006000200be006450e10091
:100cc000050036006420e100020036000968a30038
:100cd00001003a000800be000160a0004f06780045
:100ce0004f05be004f04be0000000600f0ff2f00bd
:100cf000f1ff2700f9ff3700889fbe008a9fbe00e2
:100d00008c1f7800e4ff0700ebff330003866c00c4
:100d10006450e100240032006420e100270032002a
:100d20006150e100220032006120e1002100320028
:100d30008b854200eb07b1000134b800003ab800df
:100d40000804420089844a00013ab8000030b80023
:100d50008880400009014a00040033000000400080
:100d600081804800020149008b05e900c909dd00c6
:100d7000830170000100320013002000c814de005f
:100d80004814dd004709de001200b200c808de008a
:100d90000884700085ff070001f0a1000cf0a70097
:100da00001f0a000cdff37006120e100cfff32004d
:100db0000801be000200be00f7ff37006150e100ed
:100dc000fcff3a00c9ff3700889fbe008a9fbe0023
:100dd0008c1f78000004be009aff07000478a3006f
:100de00026003a006120e1002500320009f8a30046
:100df00025003a006420e10021003200f507b1002f
:100e00000508a30002003200000040008180480075
:100e10006044b800031020000200200000004000e1
:100e2000818048000805440089854c000a0541007e
:100e30008b8549000a0550008b855800030033005c
:100e40000a00be0002047400838474008301d10090
:100e50000281d300830f7100f0ff3a008904d100b2
:100e60000884d3006001490082017800c1adde0032
:100e7000fb07b0004dff070098ff37000960a00096
:100e80000800be0095ff3700120220007260880043
:100e9000f0ff2f00f1ff270090ff37006022b8001d
:100ea000060220000000d0008180d2000482d2001f
:100eb0008582d2000000a0000202520083825a0004
:100ec000030031000202420083824a000000a100b8
:100ed0000603e900f3ff3a0000000600889fbe0009
:100ee0008a9fbe00841f78006bff07004f007800c8
:100ef00011003300f0ff2f00838f6c0006003b00d1
:100f0000040565000a00a7000800370009f0a600e4
:100f10001000200008003700820f5400838f5c000f
:100f2000030039001000200001003e0000002000f6
:100f300009f0a7000000ea004f05be004f04be0004
:100f40000000e00000000600000478001000070028
:100f5000080078005c0107008001eb000200370008
:100f600061f079008301e800828f5100fcff3a00b4
:100f7000000006008001eb0002003700817178005c
:100f80008301e800828f5100fcff3a000000060058
:100f9000881f7800900d81000000e0000100320001
:100fa000000001002810220008007800d10007008e
:100fb0006c04440060122200800f5400faff3a00d3
:100fc0004f04780000000600800078003004e00044
:100fd000feff3a00010050000000e900000006009a
:100fe000889fbe008a9fbe008c9fbe0000017800d3
:100ff000011722001100e0000b003a004017220008
:10100000800b8900600b8900a10b8900710b89009e
:10101000214090000004a000a04098006140900092
:101020000004a000e0409800e7004100c208de0094
:10103000c20cdd00740b8100cd1b2200c0232200f6
:101040000d05500022002000811f780011000900ca
:101050000205d80000067800cf007800c308dd0044
:10106000e48540008001eb00c61b2200051722002a
:101070000100370001027800244090000008a3001e
:10108000020032000a003700110a7800940078004c
:10109000214090000008a300fbff3200090142003c
:1010a000828f500002003900840f51004600310049
:1010b00094007800848f5000eeff3e00868f500031
:1010c00002003900858f5000eaff3900600b810073
:1010d000800f52004f003a00858f50004d003a00bb
:1010e0008301e800e18f5100e2ff36008c8f54004d
:1010f000040036008a8f5400020031000b0478008f
:1011000012003700614ab8006151b900b0ff2f00ea
:10111000010020000200500083805800800f520020
:10112000818f5a000200350009047800070037005b
:101130000d805400f223220002004000110009003b
:101140000a80d8000a80b9000004780008007800fe
:101150002e01070080017800e10f40002d003200d1
:10116000600b810003087800620b8100640041007d
:10117000a2409000808f5100020032000104a000c4
:10118000010037000104a1002141980008804100be
:101190006400500080097800600b8900021722006b
:1011a00002087800610b8100214090000004a0003b
:1011b000a0409800234090000004a100a0419800a6
:1011c00002027800a7ff3700720b8900828f50005f
:1011d0000900360092007800a0162200a24190007b
:1011e00003487800410b8900140978008040eb0027
:1011f000700b810021409800700b8100000a78007c
:10120000244090000004a0002042980064004200a6
:10121000010037000000eb004f06be004f05be0086
:101220004f04be000000060064005000700b8900ef
:10123000a04090000104a100214098000000060099
:10124000889fbe008a9fbe0000057800e401500020
:1012500013001000c285de00234090000008a300a8
:1012600004003200730b8900234090000004a100a9
:10127000a04198000100780059ff070000047800a1
:101280000000e000170032008a0f50001500320005
:1012900060b8970008005000c284de00898f5500b6
:1012a00001003600890578004259dd008a00780087
:1012b0000800780028ff07008a0f54000900310059
:1012c0004248dd00000044008a0f5000050036004f
:1012d0000a00500000004400420b8100530b8100c3
:1012e0000288be00080078004f05be004f04be0013
:1012f00000000600889fbe008a1f78000004780066
:101300003000900063006000240032000800780084
:10131000430007003805900080ef2f0000006500b3
:1013200030049800280090000000e0000400320023
:10133000e804650002003a0035000700290498001f
:101340004800900068000700e10f400013003200e1
:10135000b80090000102b20010003a000ac8a300d1
:1013600018003200a00d81000000e00015003200de
:101370000001780081047800012a200012289000e2
:10138000880f5000070032004205b0004905b00048
:10139000818f54000b003200f8ff37000080eb0013
:1013a00009003700020078008f000700a00d8100bf
:1013b000090040008000eb0011289800010078002f
:1013c000010037000000eb004f0578004f04be001d
:1013d00000000600b10d81000100e00003003200b2
:1013e00011007800b00d89000300370020002000b4
:1013f0008600070080007800e18f400002003a007c
:10140000906e2600706088000100780000000600e1
:10141000b10d810001087800b00d890000000600c0
:10142000881f780000047800300090000008a300b6
:1014300007003200800078000120b20004003a006a
:1014400011049800a8009000010c780017003700e4
:101450000018a300190032000098a3001700320002
:10146000a80090000100e000140032001801900074
:101470000200e00011003200480090002300070045
:1014800098009000810f5000030032003800900057
:101490000003b300300498000000eb001004980033
:1014a00028009000000c7800380090000058a3003d
:1014b000020032000080eb00010037000000eb006a
:1014c0004f047800000006000c02e20004003d001a
:1014d0000f42ab00020032000f02ab00feff3200f1
:1014e0000040da00feff37000a00fa001100200079
:1014f000b1bf9f00c0bf9f006a80570000c0da00e4
:101500004fb897000080fa00000006000a00fa00b9
:1015100080017800e20f500028003e00c00d8100dd
:10152000e10f500008003200e02120000000e00040
:10153000050032006421200085212000a621200022
:101540008001780004003700c4202000e52020003e
:101550000621200043212000144090000004e000f8
:10156000040035008009eb00144090000074a000d6
:1015700010429800154090000028a30003003a0094
:10158000154090000024a000904298008001eb00dc
:1015900007003700154090000008a300fdff32004f
:1015a00063c078000000fb00000b78008301e800b6
:1015b000828f5100f7ff3a0008003700300020000a
:1015c000b0bf9f00c3bf9f00d1bf9f00e2bf9f007d
:1015d0006a80570000c0da006fb9970002007800f7
:1015e0000080fa00000006000a00fa005100200006
:1015f000b1bf9f00c0bf9f006a80570000c0da00e3
:101600005fb897000080fa0000000600889fbe00c7
:1016100080047800d00d81000000e00003003a0053
:10162000100007000000e0000a003500d00d810026
:101630000900e00002003a000004780006003700cc
:101640000004780009004000060007000000e000e8
:1016500001003d000084eb00080078004f04be004c
:1016600000000600800078000000e00004003a005e
:10167000c01b2200d00d8900010178000600370050
:101680000081eb00c0232200808f500002003e004a
:10169000d10d89000001eb00020078000000060077
:020000040000fa
:0200000401f009
:04000000e6bf000057
:020000040000fa
:0200000401f009
:04000400ff7f00007a
:020000040000fa
:0200000401f009
:040008007fff000076
:020000040000fa
:0200000401f009
:04001400ffff0000ea
:020000040000fa
:1000080010020000100200001002000010020000a0
:100018001002000010020000100200001002000090
:1000280024830000100200001002000010020000eb
:100038001002000010020000ac8200001002000054
:1000480010020000b28b0000528b00002055000007
:100058001002000010020000ae7200001002000042
:100068001002000010020000100200001002000040
:1000780010020000f48b0000ae880000100200009f
:100088001002000010020000100200001002000020
:100098001002000010020000100200001002000010
:1000a8001002000010020000100200001002000000
:1000b80010020000100200001002000010020000f0
:1000c80010020000100200001002000010020000e0
:1000d80010020000100200001002000010020000d0
:1000e80010020000100200001002000010020000c0
:0800f8001002000010020000dc
:020000040000fa
:10010800100200001002000010020000100200009f
:10011800100200001002000010020000100200008f
:1001280024830000100200001002000010020000ea
:100138001002000010020000ac8200001002000053
:1001480010020000b28b0000528b00002055000006
:100158001002000010020000ae7200001002000041
:10016800100200001002000010020000100200003f
:1001780010020000f48b0000ae880000100200009e
:10018800100200001002000010020000100200001f
:10019800100200001002000010020000100200000f
:1001a80010020000100200001002000010020000ff
:1001b80010020000100200001002000010020000ef
:1001c80010020000100200001002000010020000df
:1001d80010020000100200001002000010020000cf
:1001e80010020000100200001002000010020000bf
:0801f8001002000010020000db
:020000040000fa
:1016a0008c020000df020000300300008003000015
:1016b000d10300002204000073040000c2040000f3
:1016c00014050000b305000054060000f1060000f8
:1016d0008f0700002d080000ca0800006309000001
:1016e000fc090000340b00005c0c0000820d0000bf
:1016f000a40e0000bd0f0000d3100000e211000096
:10170000e7120000ef140000cc1600009218000051
:10171000401a0000d61b0000531d0000b51e00003b
:101720000b200000792200008d2400006f260000ad
:101730001428000090290000e02a0000112c00006d
:10174000252d0000052f000089300000d331000056
:10175000ec320000dd330000ae34000067350000dd
:101760000d36000020370000fb370000b2380000c3
:101770004a390000cc3900003b3a00009b3a000097
:10178000f33a0000833b0000f43b0000513c0000b2
:101790009f3c0000e13c00001a3d00004b3d000072
:1017a000783d0000c03d0000f93d0000283e0000eb
:1017b0004f3e0000703e00008d3e0000a53e000040
:1017c000bc3e0000e03e0000fd3e0000143f000073
:1017d000283f0000383f0000473f0000533f000013
:1017e0005e3f0000703f00007f3f00008a3f000026
:1017f000943f00009c3f0000a43f0000aa3f00006f
:10180000af3f0000b83f0000c03f0000c53f0000f0
:10181000cb3f0000ce3f0000d23f0000d53f00008c
:10182000d83f0000dc3f0000e03f0000e33f000045
:10183000e53f0000e83f0000e93f0000eb3f00000b
:10184000ec3f0000ee3f0000f13f0000f13f0000e0
:10185000f33f0000f43f0000f53f0000f53f0000bb
:10186000f73f0000f73f0000f93f0000f83f00009d
:10187000fa3f0000fa3f0000fa3f0000fb3f000083
:10188000fb3f0000fc3f0000fc3f0000fc3f00006d
:10189000fe3f0000fd3f0000fd3f0000fd3f000057
:1018a000fe3f0000fe3f0000fe3f0000fe3f000044
:1018b000fe3f0000fe3f000000400000ff3f000030
:1018c000ff3f0000ff3f0000ff3f0000ff3f000020
:1018d000ff3f0000ff3f0000ff3f0000ff3f000010
:1018e000ff3f0000ff3f00000040000000400000fc
:1018f00000400000004000000040000000400000e8
:1019000000400000004000000040000000400000d7
:1019100000400000004000000040000000400000c7
:1019200000400000000000009301000024030000bc
:10193000b704000048060000da0700006b09000049
:10194000fc0a00008c0c00001c0e0000ab0f000015
:101950003b110000c812000056140000e3150000ff
:101960006e170000f9180000831a00000c1c00001c
:10197000941d00001a1f0000a02000002422000077
:10198000a723000029250000a82600002728000022
:10199000a4290000202b0000992c0000122e00002a
:1019a000872f0000fc3000006f320000df330000a2
:1019b0004e350000ba360000253800008d39000091
:1019c000f33a0000573c0000b93d0000173f00000b
:1019d00074400000ce410000264300007b4400001c
:1019e000cd4500001d4700006a480000b4490000d2
:1019f000fc4a0000404c0000824d0000c04e000038
:101a0000fc4f000034510000695200009b5300005d
:101a1000ca540000f65500001e570000435800004d
:101a200064590000835a00009d5b0000b45c000014
:101a3000c85d0000d75e0000e45f0000ec600000bd
:101a4000f1610000f2620000ef630000e964000051
:101a5000de650000d0660000bd670000a7680000da
:101a60008c6900006e6a00004b6b0000246c000063
:101a7000f96c0000ca6d0000976e00005f6f0000f7
:101a800023700000e37000009e710000557200009a
:101a900008730000b6730000607400000575000054
:101aa000a575000042760000d97600006c77000032
:101ab000fb77000084780000097900008a79000033
:101ac000067a00007d7a0000ef7a00005d7b00005e
:101ad000c67b00002a7c0000897c0000e47c0000ba
:101ae000397d00008a7d0000d77d00001d7e00004a
:101af000607e00009d7e0000d67e0000097f000011
:101b0000397f0000627f0000877f0000a77f000010
:101b1000c27f0000d87f0000ea7f0000f67f00004f
:101b2000fe7f0000ff7f00006d6100007468000010
:101b30002e6300006f70000079000000636f0000ea
:101b4000706900006573000020730000726300007c
:101b5000207400006f2000006465000073740000b2
:101b6000206500006c6500006d6500006e7400006b
:101b70002062000079200000656c0000656d0000a7
:101b8000656e00007400000064650000737400005e
:101b9000007300007263000000000000948d0000dc
:101ba0009e8d0000ffff0000c48d0000ffff0000bd
:101bb000c98d000000000000000000006d61000001
:101bc000746800002e660000696c00006c00000064
:101bd000666900006c6c0000732000006465000002
:101be0007374000020770000697400006820000012
:101bf000636f00006e730000746100006e7400007b
:101c000020760000616c0000756500000076000021
:101c1000616c00007565000000000000de8d0000b2
:101c2000e88d0000ffff0000c48d000001000000ef
:101c3000078e000000000000000000006d61000041
:101c4000746800002e61000064640000736300008b
:101c5000616c0000617200000061000064640000bb
:101c600020730000636100006c61000072200000be
:101c7000746f0000206500006163000068200000b0
:101c8000656c0000656d0000656e0000742000004a
:101c90006f66000020730000726300002061000086
:101ca0006e64000020730000746f00007265000015
:101cb0002072000065730000756c00007420000045
:101cc000746f000020640000657300007400000061
:101cd00073630000616c000061720000000000008e
:101ce0001e8e00002d8e0000ffff0000c48d00003e
:101cf000ffff0000c98d000001000000688e000099
:101d000000000000000000006d6100007468000029
:101d10002e61000064640000006100006464000043
:101d20007320000073720000633100002061000026
:101d30006e64000020730000726300003220000017
:101d4000746f00002064000065730000742c0000b4
:101d5000206500006c6500006d6500006e74000079
:101d60002062000079200000656c0000656d0000b5
:101d7000656e0000740000007372000063310000a3
:101d8000007300007263000032000000848e0000c7
:101d90008d8e0000ffff0000c48d0000ffff0000db
:101da000bc8e0000ffff0000c18e0000000000009c
:101db000000000006d610000746800002e730000d8
:101dc000756200000073000075620000737400000b
:101dd00072610000637400007320000073720000e1
:101de0006332000020660000726f00006d2000006a
:101df0007372000063310000207400006f20000047
:101e000064650000737400002c200000656c000005
:101e1000656d0000656e00007420000062790000ae
:101e2000206500006c6500006d6500006e740000a8
:101e300000000000da8e0000e38e0000ffff0000cb
:101e4000c48d0000ffff0000bc8e0000ffff0000fb
:101e5000c18e000000000000000000006d61000065
:101e6000746800002e6d0000756c0000006d0000ad
:101e7000756c000074690000706c000069650000fa
:101e800073200000737200006331000020610000c5
:101e90006e640000207300007263000032200000b6
:101ea000746f00002064000065730000742c000053
:101eb000206500006c6500006d6500006e74000018
:101ec0002062000079200000656c0000656d000054
:101ed000656e0000740000002e8f0000378f000038
:101ee000ffff0000c48d0000ffff0000bc8e00005b
:101ef000ffff0000c18e0000000000000000000095
:101f00006d610000746800002e64000069760000b6
:101f100000640000697600006964000065730000d9
:101f2000207300007263000031200000627900001d
:101f3000207300007263000032200000746f000004
:101f40002064000065730000742c00002065000010
:101f50006c6500006d6500006e740000206200007a
:101f600079200000656c0000656d0000656e000062
:101f700074000000808f0000898f0000ffff0000c8
:101f8000c48d0000ffff0000bc8e0000ffff0000ba
:101f9000c18e000000000000000000006d61000024
:101fa000746800002e6d0000696e0000007700006c
:101fb00072690000746500007320000074680000fe
:101fc000652000006d6900006e6900006d750000fd
:101fd0006d2000006f660000207300007263000037
:101fe00031200000616e0000642000007372000068
:101ff00063320000207400006f2000006465000060
:10200000737400002c200000656c0000656d0000fa
:10201000656e0000742000006279000020650000f9
:102020006c6500006d6500006e740000000000002b
:10203000ce8f0000d78f0000ffff0000c48d00008e
:10204000ffff0000bc8e0000ffff0000c18e0000fb
:1020500000000000000000006d61000074680000d6
:102060002e6d0000617800000077000072690000aa
:102070007465000073200000746800006520000093
:102080006d610000786900006d7500006d20000032
:102090006f660000207300007263000031200000b2
:1020a000616e000064200000737200006332000063
:1020b000207400006f20000064650000737400004d
:1020c0002c200000656c0000656d0000656e00004e
:1020d0007420000062790000206500006c6500003b
:1020e0006d6500006e740000000000002c90000080
:1020f00035900000ffff0000c48d0000ffff0000ce
:10210000bc8e0000ffff0000c18e00000000000038
:10211000000000006d610000746800002e63000084
:102120006c6100006d700000006300006c610000d5
:102130006d700000207300007263000020740000c6
:102140006f2000006c6f0000772f000068690000ae
:1021500067680000206200006f7500006e64000078
:1021600073200000696e0000746f0000206400009e
:1021700065730000742c0000206500006c65000091
:102180006d6500006e740000206200007920000080
:10219000656c0000656d0000656e00007400000055
:1021a0006c6f00007700000068690000676800003d
:1021b000000000008a90000095900000ffff0000e2
:1021c000c48d0000ffff0000c98d0000ffff00006c
:1021d000d0900000ffff0000d4900000000000003d
:1021e000000000006d610000746800002e640000b3
:1021f0006f740000007700007269000074650000d1
:10220000732000007468000065200000646f000007
:1022100074200000707200006f640000756300009d
:10222000742000006f6600002073000072630000dd
:1022300031200000616e0000642000007372000015
:1022400063320000207400006f200000646500000d
:10225000737400002c2000006166000074650000ab
:1022600072200000612000007368000069660000b1
:1022700074000000736800006966000074000000cc
:10228000f2900000fb90000001000000c48d0000ef
:10229000ffff0000bc8e0000ffff0000c18e0000a9
:1022a000010000003a910000000000000000000062
:1022b0006d610000746800002e73000074610000fe
:1022c0007400000070650000726600006f7200000c
:1022d0006d730000207300007461000074690000d9
:1022e0007374000069630000732000006f6e0000cb
:1022f0002073000072630000006d0000696e000032
:10230000006d000061780000006d00006561000054
:102310006e0000005891000062910000ffff000075
:10232000c98d0000010000007d9100000100000047
:102330008191000001000000859100000000000074
:10234000000000006d610000746800002e61000054
:1023500072670000626f0000756e00006473000019
:1023600000670000657400002074000068650000cc
:10237000206900006e64000069630000657300005e
:102380002028000061720000676d0000696e000087
:102390002c20000061720000676d00006178000071
:1023a000292000006f6600002074000068650000ae
:1023b000206c0000696d0000697400002076000048
:1023c000616c000075650000732000006f660000fe
:1023d000207300007263000000610000726700005b
:1023e0006d6900006e00000061720000676d000002
:1023f0006178000000000000a2910000b19100008f
:10240000ffff0000c98d000001000000ed910000f9
:1024100001000000f4910000000000000000000036
:102420006d610000746800002e7300006f72000080
:1024300074000000736f00007274000020610000df
:102440007272000061790000206900006e200000b7
:10245000706c0000616300006500000061720000a4
:102460007261000079000000109200001a920000d2
:10247000ffff00002e92000000000000000000009e
:102480006d610000746800002e6d0000756c000026
:10249000646900007600000070650000726600004c
:1024a0006f7200006d73000020640000657300000f
:1024b000742000003d200000286100002a62000016
:1024c000292f000063200000696e00002033000007
:1024d0003220000062690000747300002065000073
:1024e0006c6500006d6500006e74000020620000e5
:1024f00079200000656c0000656d0000656e0000cd
:102500007400000061000000620000006300000031
:10251000409200004c920000ffff0000c48d0000bc
:10252000ffff000082920000ffff00008492000085
:10253000ffff000086920000000000000000000085
:102540006d610000746800002e610000746100007d
:102550006e3200000070000065720000666f0000bf
:10256000726d000073200000646500007374000049
:10257000203d000020610000746100006e32000008
:10258000287900002c78000029200000656c0000ec
:10259000656d0000656e0000742000006279000027
:1025a000206500006c6500006d6500006e74000021
:1025b000007900000078000000000000a0920000f8
:1025c000ab920000ffff0000c48d0000ffff000081
:1025d000d9920000ffff0000db9200000000000025
:1025e000000000006d610000746800002e730000a0
:1025f000696e00000070000065720000666f0000e8
:10260000726d0000732000006465000073740000a8
:10261000203d000020730000696e00002878000053
:1026200029200000656c0000656d0000656e0000eb
:102630007420000062790000206500006c650000d5
:102640006d6500006e74000000000000f292000052
:10265000fb920000ffff0000c48d0000ffff0000a0
:10266000db92000000000000000000006d6100002f
:10267000746800002e6300006f730000007000009b
:1026800065720000666f0000726d0000732000002c
:102690006465000073740000203d000020630000aa
:1026a0006f7300002878000029200000656c00008e
:1026b000656d0000656e0000742000006279000006
:1026c000206500006c6500006d6500006e74000000
:1026d00000000000369300003f930000ffff000061
:1026e000c48d0000ffff0000db920000000000002e
:1026f000000000006d610000746800002e72000090
:102700006f74000032000000726f000074610000fe
:102710007465000073200000762000006f660000e2
:10272000206100006e6700006c6500002061000001
:10273000207400006f2000006465000073740000c6
:1027400000760000000000007a93000084930000ef
:1027500002000000c48d000002000000a1930000f0
:102760000100000082920000000000000000000054
:102770006d610000746800002e730000717200002b
:102780007400000070650000726600006f72000047
:102790006d73000020640000657300007420000069
:1027a0003d20000073710000727400002878000062
:1027b00029200000656c0000656d0000656e00005a
:1027c0007420000062790000206500006c65000044
:1027d0006d6500006e74000000000000b8930000fa
:1027e000c2930000ffff0000c48d0000ffff000047
:1027f000db92000000000000000000006d6100009e
:10280000746800002e6e00007a730000657100008d
:1028100000770000726900007465000020740000f9
:102820006f200000646500007374000020740000d5
:1028300068650000206d000069640000646c0000a1
:1028400065200000696e00006465000078200000cb
:102850006f6600002074000068650000206c0000b6
:10286000617200006765000073740000207300004f
:1028700065710000756500006e6300006520000052
:102880006f660000206e00006f6e00002d7a000061
:10289000657200006f200000656c0000656d00002f
:1028a000656e00007473000020660000726f000007
:1028b0006d20000073720000632c0000202d0000ca
:1028c0003120000069660000206e00006f74000077
:1028d000206600006f7500006e640000206f00002d
:1028e0007220000069660000207300006d61000026
:1028f0006c6c0000657200002074000068610000cc
:102900006e2000006d6900006e4c0000656e0000d6
:1029100067740000680000006d6900006e4c0000e4
:10292000656e00006774000068000000fe93000000
:102930000994000001000000c48d0000ffff0000aa
:10294000c98d0000010000008c9400000000000010
:10295000000000006d610000746800002e7200002d
:10296000616e000064000000666900006c6c00008d
:102970002061000072720000617900002077000081
:102980006974000068200000726100006e6400003d
:102990006f6d000020760000616c0000756500001e
:1029a00073000000aa940000b4940000ffff000030
:1029b000c48d0000000000000000000069640000f9
:1029c000007300006f750000726300006500000076
:1029d0006172000067730000005f00007072000009
:1029e0006f6400007563000074490000640000001b
:1029f0007370000065650000642e00006c650000c7
:102a000066740000007300007065000065640000db
:102a10002e7200006967000068740000006c0000fe
:102a20006564000073000000707200006f780000a1
:102a3000006100006d620000696100006e740000ba
:102a4000006100006363000000630000616d00002e
:102a50002e6c0000696e00006500000063610000dc
:102a60006d2e0000726500006400000063610000cc
:102a70006d2e000067720000656500006e000000aa
:102a8000636100006d2e0000626c0000756500003f
:102a90000073000074650000707300002e6c00006d
:102aa000656600007400000073740000657000002b
:102ab000732e000072690000676800007400000057
:102ac0006d69000063000000736500006c00000089
:102ad0007263000035000000746900006d6500003d
:102ae000722e000070650000726900006f640000c3
:102af00000620000617400007465000072790000db
:102b000000670000797200006f0000006972000029
:102b10005f730000656e0000736f00007273000049
:102b20000049000052200000736500006e73000031
:102b30006f72000073200000757000006461000077
:102b40007465000064000000636100006d650000b2
:102b50007261000000630000616d0000657200009a
:102b60006120000075700000646100007465000061
:102b700064000000536500006c6500006374000091
:102b80006f72000020730000746100007475000013
:102b90007320000063680000616e0000676500003c
:102ba00064000000746900006d65000072000000a0
:102bb000546900006d6500007200000086950000f9
:102bc00091950000a4950000ab950000649500006d
:102bd000ba950000d2950000d895000000000000d2
:102be00000000000677200006f7500006e64000056
:102bf0002e670000657400005f760000616c0000c5
:102c000075650000730000007265000061640000db
:102c1000207400006865000020760000616c0000f0
:102c200075650000732000006f66000020740000ce
:102c30006865000020670000726f0000756e00007c
:102c400064200000736500006e7300006f72000066
:102c500073000000646500007374000000630000ee
:102c6000616d00002e730000657400005f6100005c
:102c7000776200005f61000065000000656e000083
:102c8000616200006c65000020280000312900000e
:102c90002f64000069730000616200006c65000031
:102ca0002028000030290000207400006865000022
:102cb00020610000757400006f6d000061740000f9
:102cc00069630000207700006869000074650000f7
:102cd00020620000616c0000616e0000636500000e
:102ce000206100006e640000206500007870000024
:102cf0006f730000757200006500000061770000ce
:102d0000620000006165000000630000616d00006a
:102d10002e730000657400005f650000787000008d
:102d20006f7300007572000065000000736500009d
:102d300074200000746800006520000063610000da
:102d40006d65000072610000206500007870000071
:102d50006f73000075720000650000006578000068
:102d6000706f000073750000726500000063000062
:102d7000616d00002e730000657400005f7200003a
:102d8000676200005f670000616900006e0000007c
:102d90007365000074200000746800006520000066
:102da000636100006d650000726100002072000028
:102db0002f6700002f62000020670000616900009b
:102dc0006e00000072650000645f00006761000033
:102dd000696e00000067000072650000656e00000b
:102de0005f670000616900006e000000626c000017
:102df000756500005f670000616900006e000000fb
:020000040000fa
:102e00002800fa0010179800211798001e10900053
:102e10000000e0000c003a002e1090000000e000de
:102e2000030035000000eb0030179800bd003700ac
:102e30002e1090000000e00003003d00020028007a
:102e400032179800b7003700ae119000630f98005a
:102e50006e0890000000e00003003d006e08900046
:102e60000000ea00600f98001e129000540f9800b6
:102e70005e0890000000e00003003d005e08900046
:102e80000000ea00500f98002e1090000000e000b3
:102e900003003a0000002400700f980098003700eb
:102ea000ee0990005e089000cf80de000202200054
:102eb0000e014100811f7800110009004388d800ed
:102ec00001097800cf00780001002000200f980051
:102ed000310f98006e0990000e1090000100200044
:102ee000c000dd0000002000811f780011000900f3
:102ef0004288d800cf007800400f98002e0890003c
:102f0000be089000c001dd00020020004e089000c5
:102f1000010020000000710081807100000f980006
:102f2000110f98000e0890009e0890004088de0067
:102f3000cf80de000080cf00700798007e009000f8
:102f40000000e0000500320000022000fe009000ba
:102f50000100500070079800090037000e0890002b
:102f60000080cf00700798007e0090000000e00015
:102f7000030032007e00900070001000700798007f
:102f80007e0090006c005000600798006e0090007a
:102f90000000e00013003d00805a84006103b90086
:102fa000860078000e089000000ab8001e08900005
:102fb00000b0b90005017800000141000e08900042
:102fc0000780b9000001410082027800442bdd0037
:102fd0004c20de0000007300cca8de00700f9800cb
:102fe0004000370010002000010020007e0190000a
:102ff0000002be00020378000603e900030033006c
:103000000402420085824a00fbff37000401be0033
:103010000e0890009e089000020050008380580027
:1030200040079800510798007e009000680050000b
:10303000300798004e009000de0090003e019000a6
:10304000820178008301e900030033008180d10010
:103050000080d300fbff3700200798002e0090006f
:103060004580de00100798002e0090007f0f600062
:10307000000220001e0150006e009000c300dd0021
:103080001e009000008040008000400000b5280035
:1030900000804000100078000281b9006e009000ae
:1030a000c300dd001e009000008040000000e8002a
:1030b0008000400000b5280000804000100078002b
:1030c0001e80b900020040008380480002022000f8
:1030d000811f7800110009004208d800cf00780055
:1030e000700f98002e1090000000e00004003d00da
:1030f00000002800fe08900001005000700f9800aa
:103100001e1090000000e000030034007e0a9000d2
:1031100034179800030037007e0890000000ea0092
:10312000301798003e1090000080fa000000060062
:103130000e00fa00889fbe008a9fbe0050079800cc
:103140005e0090000000e00017003d00de009000ef
:1031500000002c00808f500005003d00000028007a
:10316000de00900000804000100798000b00370040
:10317000de00900000002c00808f5000040034001e
:103180005e0090000000ea0010079800030037007e
:10319000100028006007980053003700100020003e
:1031a0002007980015003700de0090000000240082
:1031b000808f50000500340000002800de009000e1
:1031c00001005000100798000a003700de00900050
:1031d000f0ff2300808f500003003c005e01900050
:1031e0001207980003003700f0ff270060079800df
:1031f0003d0037000000eb00200798001e00900003
:103200004780de00400798009e009000f0072000f5
:1032100000806000300798004e0090008000400061
:1032200020c9280000804000100078006103b90028
:10323000010820003e009000008050006102b900ab
:103240008600780004007800000db80005b0b900d1
:103250000b0178000001410007a0b9000001410006
:10326000820578004e0090000000e80080004000d9
:1032700020c9280000804000100078006104b900d7
:103280003e0090006103b9008800780006007800d5
:10329000000ab80007c0b90005017800000141002c
:1032a00009b0b90000014100820278000a00420022
:1032b0008b804a004909dd004700de0000007100f4
:1032c000c788de00000f78002e0090000000e000ac
:1032d000030032001e00ea00600798000200370079
:1032e0001e017800620798006e0090004f05be0036
:1032f0004f04be000080fa00000006000200fa0041
:10330000000f7800000024001e00400088ff070026
:103310000080fa00000006000800fa00300798005c
:103320003e009000200798000000eb001007980076
:1033300000002400000f7800030037001e00780012
:103340004280de00000f78002e0090009e0f1000db
:10335000faff3c00150037001e0090009e00400060
:103360002e009000808f50000a003c001e0090004c
:103370009e0040002e0090000100500020079800a1
:103380001e0090000080d1001e0040001007980031
:10339000030037001e0090000080d1001007980045
:1033a0001e0078004280de00000f78001e00e00062
:1033b000e9ff3a001e0090000080fa0000000600bd
:1033c0000c00fa0040079800510798005e0090003a
:1033d000300798000000eb002007980048003700f5
:1033e0003e009000e10f5000080036003e009000c3
:1033f0006400b80052002000811f7800110009000d
:103400004288d800cf007800300798000000eb0019
:10341000200798000000eb001007980032003700ea
:103420001e00900000004000800078004e009000d8
:1034300000804000100178009e0090003e00900047
:103440000080400000004000800078004e009000a6
:103450000080400010007800000051000000e000f3
:103460001e0034001e009000000040008000780024
:103470004e00900000804000100f78001e00900069
:1034800000004000800078004e0090000081400065
:103490009e0090003e009000008040000000400030
:1034a000800078004e0090000080400010007800fe
:1034b000000978009e0090003e00900000804000cf
:1034c00000004000800078004e0090000080400026
:1034d0001e08780010002000200798001e009000b1
:1034e0000000e80010079800be0090001e00900049
:1034f000808040005e009000808f5000c8ff39003f
:103500003e009000e10f5000b5ff3e002e009000fd
:103510000000e000b2ff3a000080fa000000060060
:103520000a00fa00400798004e00900022000700b1
:10353000300798004e0090001f00070020079800f9
:103540004e0090001c000700100798000000eb00e0
:10355000000f7800130037004e009000c00090006c
:103560003e00900000004000008140004e009000ae
:10357000c00090002e00900000004000008040003d
:1035800010007800000978003e0090000000e8007c
:10359000300798002e0090000000e80020079800f7
:1035a0001e0fe8001e0090009e0f1000eaff390079
:1035b0000080fa00000006000200fa00000f780008
:1035c0001e007800600190001e00780090089000b6
:1035d0000100780000004000000041001001780068
:1035e0008100e9001e0078001108980002007800b0
:1035f0000080fa00000006000a00fa004007980068
:103600004e009000ecff0700300798004e0090003d
:10361000e9ff0700200798004e009000e6ff070032
:10362000100798000000eb00000f78001000370032
:103630004e009000c00090003e009000000040004e
:10364000008140004e009000c00090002e009000cd
:103650000000400000804000100078000009780061
:103660003e0090000000e800300798001e0fe800c0
:103670001e0090009e0f1000edff39000080fa0040
:10368000000006000e00fa00600798006e0090002f
:10369000c9ff0700500798006e009000c6ff0700a2
:1036a000400798006e009000c3ff070030079800a5
:1036b0006e009000c0ff0700200798006e00900089
:1036c000c00090003e0090000000400000804000dc
:1036d00090007800110798000000eb00000f7800c0
:1036e000150037006e009000c00090005e00900052
:1036f00000004000008140006e009000c00090007b
:103700004e009000000040000080400090007800d3
:103710001e00900000804000000978005e009000cc
:103720000000e800500798004e0090000000e800fc
:10373000400798001e0fe8002e0090009e0f10001a
:10374000e8ff39000080fa00000006000c00fa00d3
:10375000500798005e00900097ff07004007980010
:103760005e00900094ff0700300798005e00900014
:1037700091ff0700200798005e0090008eff070071
:10378000100798000000eb00000f78001d003700c4
:103790005e009000c00090004e00900000004000cd
:1037a000808140005e009000c00090003e009000cc
:1037b0000000400000804000100178005e00900092
:1037c000c00090002e0090000000400000804000eb
:1037d0001000780000004100800978004e00900041
:1037e0000000e800400798003e0090000000e8005c
:1037f000300798002e0090000000e8002007980095
:103800001e0fe8001e0090009e0f1000e0ff390020
:103810000080fa00000006000c00fa005007980033
:103820005e00900064ff0700400798005e00900073
:1038300061ff0700300798005e0090005eff070000
:10384000200798005e0090005bff070010079800bb
:103850000000eb00000f78001d0037005e009000b4
:10386000c00090004e0090000000400080814000a9
:103870005e009000c00090003e00900000004000fc
:1038800000804000100178005e009000c0009000b1
:103890002e009000000040000080400010007800e2
:1038a00000005100800978004e0090000000e80000
:1038b000400798003e0090000000e80030079800a4
:1038c0002e0090000000e800200798001e0fe8007e
:1038d0001e0090009e0f1000e0ff39000080fa00eb
:1038e000000006000c00fa00500798005e009000ef
:1038f00031ff0700400798005e0090002eff070090
:10390000300798005e0090002bff0700200798000a
:103910005e00900028ff0700100798000000eb00f1
:10392000000f78001d0037005e009000c00090007e
:103930004e00900000004000808140005e0090003a
:10394000c00090003e009000000040000080400059
:10395000100178005e009000c00090002e009000e2
:103960000000400000804000100078000090b90086
:10397000800978004e0090000000e80040079800a1
:103980003e0090000000e800300798002e009000f4
:103990000000e800200798001e0fe8001e009000bd
:1039a0009e0f1000e0ff39000080fa0000000600c2
:1039b0001400fa00881f7800100f98001e0890006d
:1039c000fdfe0700000f98001e089000fafe070099
:1039d000700798001e089000f7fe07006007980027
:1039e0001e089000f4fe0700500798000000eb004e
:1039f00040079800380037001e089000c000900073
:103a00007e00900000004000008040001000780020
:103a1000cf80de0020079800310798007e009000dc
:103a20000000e800700798001e089000c000900099
:103a30006e00900000004000008040001000780000
:103a4000cf80de00008fbe006e0090000000e80016
:103a5000600798001e00be00e00f5000e08f580085
:103a6000120032001e089000c00090000e08900066
:103a700000004000008440001e01be002e009000a7
:103a8000be009000de04020000000000000c780080
:103a90000e0890000000e800000f98004e00900013
:103aa0000000e800400798000b0037009e089000d7
:103ab00020002000f00098001e08900070014000d7
:103ac00023002000710029001e089000006c0200f5
:103ad0000000000004003700ce0090005e0090005f
:103ae000808f5000c4ff39004f0478000080fa0036
:103af000000006001600fa00000f98000e08900063
:103b0000adfe0700700798000e089000aafe07009f
:103b1000600798000e089000a7fe07005007980065
:103b20000e089000a4fe0700400798000000eb007c
:103b3000300798002c0037000e089000c00090005d
:103b40006e0090000000400000804000900078006f
:103b5000210798006e0090000000e80060079800c0
:103b60000e089000c00090005e0090000000400031
:103b70000080400090007800110798005e009000df
:103b80000000e800500798002e009000200f9800d9
:103b90009e009000110f98001e089000ae08900043
:103ba000810f5000020034002e089000100f980082
:103bb0009e089000010f78000e089000c000900051
:103bc0007e00900000004000008040001e08780049
:103bd0007e0090000000e800700798003e00900012
:103be0000000e80030079800be0090004e009000f2
:103bf000808f5000d0ff39000080fa0000000600de
:103c00001600fa00000f98000e0890006afe0700e8
:103c1000700798000e08900067fe07006007980084
:103c20000e08900064fe0700500798000e089000f0
:103c300061fe0700400798000000eb003007980085
:103c40002c0037000e089000c00090006e0090001d
:103c5000000040000080400090007800210798009c
:103c60006e0090000000e800600798000e089000c9
:103c7000c00090005e009000000040000080400006
:103c800090007800110798005e0090000000e800a6
:103c9000500798002e009000200f98009e00900082
:103ca000110f98001e089000ae089000810f500080
:103cb00002003d002e089000100f98009e08900012
:103cc000010f78000e089000c00090007e00900068
:103cd00000004000008040001e0878007e00900038
:103ce0000000e800700798003e0090000000e80027
:103cf00030079800be0090004e009000808f50006a
:103d0000d0ff39000080fa00000006001a00fa0017
:103d1000200f98002e08900027fe0700100f980033
:103d20002e08900024fe0700000f98002e08900037
:103d300021fe0700700798002e0890001efe070065
:103d4000600798002e0890001bfe0700500798009f
:103d50000000eb00400798003d0037002e0890005f
:103d6000c00090000e08900000004000008040005d
:103d700090007800310798000e0890000000e800dd
:103d8000000f98002e089000c00090007e00900068
:103d9000000040000080400090007800210798005b
:103da0007e0090000000e800700798002e08900048
:103db000c00090006e0090000000400000804000b5
:103dc00090007800110798006e0090000000e80055
:103dd00060079800be0090001e009000808f500089
:103de0000b003c002e009000400f9800be00900099
:103df000310f98003e089000ce089000810f5000cf
:103e000005003d004e089000300f9800020037007a
:103e10009e009000310f98003e089000000f78003f
:103e20002e089000c00090001e0890000000400086
:103e3000008040001e0878001e0890000000e80086
:103e4000100f98004e0090000000e8004007980016
:103e5000ce0090005e009000808f5000bfff3900c0
:103e60000080fa00000006001200fa00881f7800a7
:103e7000000f98000e089000cffd07007007980013
:103e80000e089000ccfd0700600798000e08900017
:103e9000c9fd0700500798000e08900040049000ec
:103ea0000e089000c4fd0700000040000000440020
:103eb00090007800410798000e089000befd0700b2
:103ec000300798006000b80010079800210798009c
:103ed000ce00900000022000808f500008003400c7
:103ee0000e089000c00090007e009000000040008e
:103ef000808040000000eb00800878002d00370033
:103f00003e0090000000e900300798004580a900bd
:103f100021028000100f2000008070002002880025
:103f20000e089000c00090006e009000000040005d
:103f3000008440000e089000c00090005e009000d9
:103f400000004000808040003e009000881f780004
:103f5000811f78001201c300380278000080080039
:103f600001000000b10278005200c000cf007800cc
:103f70004f0478004e009000f00f50000400340011
:103f80004e00900070005000400798005000c8009c
:103f90004e0090000000c8000e089000c000900085
:103fa0007e009000000040008080400010018000f2
:103fb000800878004f0478000080fa0000000600b6
:103fc0001400fa00881f7800100f98001e08900057
:103fd00079fd0700000f98001e08900076fd07008d
:103fe000700798001e08900073fd07006007980096
:103ff0001e08900070fd0700500798001e089000f2
:104000006dfd0700400798004e0090000000e000a2
:10401000610032001e089000c00090000e08900061
:1040200000004000008040009000780031079800b8
:104030000e0890000000e800000f98003e0090007d
:10404000cf80de0010079800210798001e0890001e
:10405000c00090007e009000000040000080400002
:10406000be009000010878001e089000c00090007b
:104070006e0090000000400000804000be009000f4
:104080000108780010002000000f7800330037008e
:104090001e089000c00090000e0890000000400034
:1040a0000080400090007800310798000e089000d2
:1040b0000000e800000f98001e089000c00090006b
:1040c0007e009000000040000080400090007800da
:1040d0003e009000808f5000070034001e089000c2
:1040e000c00090007e009000000040000080400072
:1040f000be009000010878001e089000c0009000eb
:104100006e009000000040000080400090007800a9
:104110003e009000808f500007003d001e08900078
:10412000c00090006e009000000040000080400041
:10413000be009000010878003e0090006101b900c7
:104140001e009000ae0090000000410081804900f8
:1041500010079800210798001e0fe8004e009000fd
:104160009e0f1000caff39001e089000c00090008a
:104170005e00900000004000008440004e0090006f
:104180006101b8001e009000ae009000de04020045
:1041900000000000000c78004f0478000080fa0056
:1041a000000006001200fa00000f98000e089000b0
:1041b00001fd0700700798000e089000fefc070044
:1041c000600798000e089000fbfc0700500798005d
:1041d0000e089000f8fc070040079800f0ff270049
:1041e0003007980000002800200798004e0090003b
:1041f0000000e0002b0032000000eb00000f780010
:10420000250037000e089000c00090007e0090004e
:1042100000004000008040009000780011079800e6
:104220007e0090000000e800700798009e0090005b
:104230003e009000808f500009003d001e0090005d
:10424000300798000e089000c00090006e009000ab
:1042500000004000808040001e0078008008780048
:104260009e0090002e009000808f500009003400c6
:104270009e009000210798000e089000c00090005a
:104280005e00900000004000808040001e0078002a
:10429000800878001e0fe8004e0090009e0f10006e
:1042a000d8ff39000080fa00000006000600fa007e
:1042b000200798002e009000bffc07001007980010
:1042c0002e009000bcfc0700000f78002e0090002c
:1042d000c00090001e0090000000400000804000e0
:1042e0009e00780036fc07000080fa0000000600ff
:1042f0001a00fa00881f7800400f98004e089000be
:10430000adfc0700300f98004e089000aafc070093
:10431000200f98004e089000a7fc0700100f98008f
:104320004e089000a4fc0700000f98004e08900073
:10433000a1fc0700700798000000eb0060079800e0
:10434000500037004e089000c00090002e089000ea
:10435000000040000080400010007800cf80de00a8
:1043600040079800510798002e0890000000e800d0
:10437000200f98004e089000c00090001e0890008a
:10438000000040000080400010007800cf80de0078
:1043900020079800310798001e0890000000e800f0
:1043a000100f98004e089000c00090000e0890007a
:1043b000000040000080400010007800cf80de0048
:1043c000008fbe000e0890000000e800000f98006b
:1043d0001e00be00e00f5000e08f58001e003200ab
:1043e0004e089000c00090003e0890000000400081
:1043f00000844000ce0090002e009000000ab8001b
:10440000ce0090003e0090000088b90005017800c1
:1044100000014100ae0090005e0090000088b900ed
:1044200000014100820278001e01be000400be00af
:10443000de04020000000000000c78003e0890003e
:104440000000e800300f98006e0090000000e800c7
:10445000600798000b003700ce0890002000200075
:10446000f00098004e0890007001400023002000ea
:10447000710029004e089000006c0200000000004e
:1044800004003700ee0090007e009000808f500006
:10449000acff39004f0478000080fa0000000600ed
:1044a0001000fa00881f7800700798007e009000c6
:1044b00041fc0700600798007e0090003efc07006a
:1044c000500798007e0090003bfc070040079800d2
:1044d0007e00900038fc0700300798000000eb00d9
:1044e00020079800220037007e009000c000900056
:1044f0005e009000000040000080400090007800c6
:10450000110798005e0090000000e8005007980036
:104510007e009000c00090004e009000000040001f
:1045200000804000100f78004e0090000000e8006e
:10453000400798007e009000c00090006e00900040
:1045400000004000008440009e0078001e009000a3
:104550002bfa0700000c78006e0090000000e800c5
:10456000600798002e0090000000e80020079800e7
:10457000ae0090003e009000808f5000daff3900be
:104580004f0478000080fa00000006000c00fa00da
:10459000881f7800500798005e00900006fc070016
:1045a000400798005e00900003fc07003007980069
:1045b0005e00900000fc0700200798000000eb0060
:1045c00010079800170037005e009000c0009000b0
:1045d0003e0090000000400000804000100f780076
:1045e0003e0090000000e800300798005e00900058
:1045f000c00090004e009000000040000084400089
:104600001e007800cafa0700000c78004e009000e7
:104610000000e800400798001e0090000000e8003d
:10462000100798009e0090002e009000808f500090
:10463000e5ff39004f0478000080fa000000060012
:104640000c00fa00881f7800500798005e00900068
:10465000d9fb0700400798005e009000d6fb0700da
:10466000300798005e009000d3fb070020079800f9
:104670000000eb0010079800170037005e00900064
:10468000c00090003e00900000004000008040000c
:10469000100f78003e0090000000e80030079800fe
:1046a0005e009000c00090004e00900000004000ae
:1046b000008440001e00780010fb0700000c78000a
:1046c0004e0090000000e800400798001e00900097
:1046d0000000e800100798009e0090002e00900057
:1046e000808f5000e5ff39004f0478000080fa0009
:1046f000000006001600fa00889fbe008a9fbe00d8
:10470000200f98002e089000abfb0700100f9800b8
:104710002e089000a8fb0700000f98002e089000bc
:10472000a5fb0700700798002e089000c0009000bd
:104730000e089000000040000080400090007800cb
:10474000610798002e089000c00090000e089000ad
:1047500000004000008040000080e8001001780068
:10476000520798002e089000c00090007e00900034
:104770000000400000804000900078004107980051
:104780004e009000ddfa0700300798004e009000c0
:1047900067fa0700200798003e0090006103b90007
:1047a0006e0090006102b900860078000400780075
:1047b000000db80005b0b9000b0178000001410000
:1047c00007a0b90000014100820578002e0090008a
:1047d0006104b9005e0090006103b90088007800b0
:1047e00006007800000ab80007c0b900050178008b
:1047f0000001410009b0b9000001410082027800c7
:104800000400550085805d004109dd004f00de0099
:1048100000007100cf88de00100798003e00900075
:104820006103b9005e0090006102b9008600780063
:1048300004007800000db80005b0b9000b01780045
:104840000001410007a0b900000141008205780085
:104850002e0090006104b9006e0090006103b90061
:104860008800780006007800000ab80007c0b90088
:10487000050178000001410009b0b90000014100c4
:10488000820278000a0042008b804a004109dd0064
:104890004f00de0000007100cf88de00000f7800be
:1048a0002e089000c00090001e08900000004000fc
:1048b000008040009e009000010878002e089000c3
:1048c000c00090001e0890000000400000804000e2
:1048d0000080e8001e0878004f05be004f04be00af
:1048e0000080fa00000006000c00fa00881f780023
:1048f000500798005e0090002ffb070040079800cb
:104900005e0090002cfb0700300798005e009000ce
:1049100029fb0700200798000000eb001007980013
:10492000170037005e009000c00090003e0090002d
:104930000000400000804000100f78003e00900012
:104940000000e800300798005e009000c000900072
:104950004e00900000004000008440001e007800df
:104960006dfa0700000c78004e0090000000e8008f
:10497000400798001e0090000000e8001007980013
:104980009e0090002e009000808f5000e5ff3900bf
:104990004f0478000080fa00000006001c00fa00b6
:1049a000500f98005e08900003fb0700400f98002e
:1049b0005e08900000fb0700300f98005e08900032
:1049c000fdfa0700200f98005e089000fafa070031
:1049d000100f98005e089000c00090002e08900014
:1049e000000040000080400090007800010f980017
:1049f0000000eb00100798000f0037001e00900029
:104a00000000e800100798009e0090001e0890002b
:104a1000808f5000080036005e089000c0009000b3
:104a20004e08900000004000808040000000eb0035
:104a300080087800a90037005e08900040019000cf
:104a4000be0890001e009000008040000000400062
:104a500000004100100078000000e000e7ff3a008d
:104a60001e00900070079800290037001e0090007b
:104a70000000e800100798009e0090001e089000bb
:104a8000808f5000220036007e0090000000e00081
:104a900008003a005e089000c00090004e089000a8
:104aa00000004000808040000080eb00800878001b
:104ab0008a0037007e009000000fe9000e08900089
:104ac0009e0f5000080036005e089000c000900065
:104ad0004e08900000004000808040000080eb0005
:104ae000800878007d0037005e089000c0009000cc
:104af0004e08900000004000808040007e00900042
:104b00000000e9000000d100800878007300370041
:104b10005e08900040019000be0890001e009000ca
:104b200000804000000040000000410010007800bc
:104b30000000e000cdff32000000eb0060079800ad
:104b40000000eb00400798000000eb0030079800e1
:104b5000ee00900051079800070037006e009000ab
:104b60000000e80060079800ee0090001e0890002a
:104b7000808f5000110031005e089000c00190004d
:104b8000ee0090001e009000008040001e09900082
:104b9000110009000280d8008000fd00800078002c
:104ba0003e0890000080400000004000008041006e
:104bb000100078000000e000e8ff3a00ee009000ee
:104bc0005e0090000080500020079800ae0090002a
:104bd0004e009000808f5000090034002e0090009d
:104be00040079800ee0090005e00900000804000ba
:104bf00022002000110009000200d80030079800b0
:104c0000ee0090001e089000808f50001a003100c6
:104c1000070037006e0090000000e8006007980071
:104c2000ee0090001e089000808f500012003100ae
:104c30005e089000c0019000ee0090001e00900001
:104c4000008040001e099000110009000280d80079
:104c50008000fd00800078003e0890000080400049
:104c60000000400000804100100078000000e000db
:104c7000e8ff3200b6ff3700ce0090000e0890002b
:104c8000808f500008003d005e089000c00090003a
:104c90004e08900000004000808040000080eb0043
:104ca000800878000d0037005e089000c00090007a
:104cb0004e0890000000400080814000be0090003f
:104cc0001e009000008040001e09900011000900a5
:104cd0000280d8008000fd00800978000080fa0082
:104ce000000006000200fa00000f78001e007800a5
:104cf000400d89000080fa00000006000000fa0064
:104d0000410d8100502526000088b9008000780000
:104d10009061230000804000400d8900400d81001b
:104d20000080fa00000006000800fa00881f7800e2
:104d3000300798003e0090001ffa070020079800f7
:104d40003e0090001cfa0700100798000000eb00de
:104d5000000f78000b0037003e009000c00090006c
:104d60002e0090000000400000844000e3ff070098
:104d7000000c78002e0090000000e800200798004a
:104d80001e0fe8001e0090009e0f1000f2ff390079
:104d90004f0478000080fa00000006000200fa00cc
:104da000000f78009e0078000000eb00800898005b
:104db0009e0078000000eb00f00098009e00780054
:104dc0000000eb00a01898001e007800a0009000e2
:104dd0000000eb00800878001e0078003000900092
:104de00000004000800078001e0078004000900025
:104df000010178008000eb00ba070200000000000b
:104e00000080fa00000006000a00fa00200798005f
:104e1000310798002e00900020009000900078004c
:104e20001107980010002000000f780013003700d1
:104e30002e009000a00090001e00780000004000ae
:104e400000804000900078003e009000808f50006d
:104e500009003a002e009000a00090001e0078008b
:104e600000004000008040000080e8001000780052
:104e700040079800060037001e8fe8001e009000d3
:104e80009e0f1000eaff39000000eb004007980079
:104e90004e0090000080fa00000006000600fa00b4
:104ea0001007980021079800ae0090001e009000a7
:104eb000d5ff0700000f78001e00e0002000320040
:104ec0001e00900070009000610060000004e0008f
:104ed000070032001e0090007001400023002000f7
:104ee000810029001e009000006c020000000000fc
:104ef0001e0090009e007800010898009e0090001f
:104f00000080eb00900898001e0090007000900058
:104f1000800078000100a0001e0090007100980041
:104f20001e009000700090000000d1006100600041
:104f30000004e000020032001e009000b8040700e8
:104f40001e0078000080fa00000006001200fa003f
:104f5000000f780011079800220798003307980087
:104f60003e0090006101b80072079800030f98009e
:104f700010012000010020007e0190008e099000a9
:104f8000800f5100818f5900ca003e007e009000c2
:104f90008e089000006001001100370015003700f6
:104fa000190037001d0037002100370025003700a9
:104fb000410037005e0037006200370066003700ae
:104fc0006a003700720037007a003700820037002d
:104fd0008a003700920037009a003700a700370098
:104fe0009e0090002e0090008008dd006107980070
:104ff000b20037009e0090002e0090008088de00f6
:1050000061079800ad0037009e0090002e009000d0
:105010008080400061079800a80037009e00900043
:105020002e0090008080500061079800a300370098
:105030009e0090002e0090000088b9006007980044
:105040009e0037002e0090000000e00014003a009f
:10505000000020000000e000040032008000eb00af
:105060001e00780000000200000000001e00780012
:1050700021002000710098009e007800708140009f
:1050800023002000710029001e007800006c02003f
:10509000000000000001eb00620798008700370065
:1050a0001e0090002e019000110009000200d8009f
:1050b00060079800810037002e0090000000e0009b
:1050c00014003a00000020000000e000040032005c
:1050d0008000eb001e0078000000020000000000cd
:1050e0001e00780021002000710098009e017800c9
:1050f0007081410023002000710029001e0078000b
:10510000006c0200000000000000eb006007980047
:105110006a0037001e0090002e0190001100090067
:105120000200d8008000fd0060079800630037008f
:105130009e0090002e009000808070006107980013
:105140005e0037009e0090002e0090008080680076
:1051500061079800590037009e0090002e009000d3
:105160008080600061079800540037008000eb00e9
:10517000610798009e0090002e009000808f5000e4
:105180004e003a0012002000620798004b003700e2
:105190008001eb00630798009e0090002e009000b5
:1051a000808f5000450032001000200060079800fa
:1051b000420037008000eb00610798009e009000dd
:1051c0002e009000808f50003c0034001200200020
:1051d00062079800390037008001eb0063079800f0
:1051e0009e0090002e009000808f5000330035000c
:1051f0001000200060079800300037008000eb00ae
:10520000610798009e0090002e009000808f500053
:105210002a003d0012002000620798002700370096
:105220008001eb00630798009e0090002e00900024
:10523000808f500021003c00100020006007980083
:105240001e0037001e0090000000e00003003a003e
:105250002e0090000000e00003003200110020004a
:1052600051079800020037000001eb005207980038
:10527000de01900063079800100037001e009000c8
:105280000000e000060032002e0090000000e00068
:105290000300320010002000400798000200370091
:1052a0008000eb00410798004e01900062079800d3
:1052b000020037008001eb00630798006e00900049
:1052c0000080fa00000006000a00fa00000f7800d3
:1052d00011079800220798002e00900040079800c0
:1052e0004e009000e10f50000b0032004e00900085
:1052f000e10f5000040039004e009000e20f500012
:105300000e003200110037001e0090000000ea007d
:10531000300798000f0037001e00900030079800fb
:105320003e0090000000e0000a003d003e009000ba
:105330000000ea0030079800060037001e009000c9
:105340000080ea0030079800020037000000eb0000
:10535000300798003e0090000080fa000000060030
:105360004200fa00601f98006e189000a0009000a4
:105370006e1890000008900000004000008040007f
:1053800090007800711798007e1090004c00de00ad
:105390006101b800721f980003279800e000200008
:1053a000010020007e1990008e219000800f510096
:1053b000818f590031023e007e1890008e209000af
:1053c000006001000e003700140037002a0037008b
:1053d000430037005e00370078003700c400370014
:1053e0001801370034013700600137006a013700c7
:1053f000cc013700f1013700fc0137001102370002
:105400006e189000f0009000e0ff2f008080600098
:105410006e18900071009800180237007e109000fe
:105420004400dd004480de00601798006e18900094
:10543000600190006e189000100890008000e80055
:105440006e189000110898006e18900010089000d7
:105450000000400000004100ee10900001087800bc
:105460006e189000000890008000e8006e18900010
:1054700001089800010237006e189000600190004a
:105480006e189000100890008000e8006e189000e0
:10549000110898006e18900010089000000040005d
:1054a000000141006e189000a00090006e1890005e
:1054b0000008900000004000008040000080e800ec
:1054c00010007800000978006e1890000008900025
:1054d0008080e8006e18900001089800e70137000e
:1054e000fe109000f0ff2000008060005017980030
:1054f0006e189000600190006e18900010089000e7
:105500008000e8006e189000110898006e18900056
:105510001008900000004000000141006e1890004b
:10552000c00090005e10900000004000008040002d
:1055300010007800000978006e18900000089000b4
:105540008000e8006e18900001089800cb01370039
:10555000fe109000f0ff20000080600040179800cf
:105560006e189000c00090004e10900000004000a7
:10557000808140006e189000e00090006e1890004e
:1055800010099000020078000000400000804000f8
:1055900010007800800978008200e9006e18900001
:1055a000110898006e189000000890008000e80034
:1055b0006e18900001089800b0013700fe109000ae
:1055c000f0ff200000806000301798006e189000f7
:1055d000a00090006e1890000008900000004000ad
:1055e000008040000080e800100178002217980039
:1055f0006e189000e00090006e1890001008900067
:105600000000400000804000100078001017980053
:105610009e1090002e109000808f50001f003900c7
:105620006e18900080089000000320000e004000db
:1056300001087800000320000e004000ae11900029
:1056400013009800000320000e0040009e10900000
:1056500021009800ee18900020002000f000980033
:10566000020320000e0141006300200061002900b8
:105670006e189000006c0200000000000000200086
:105680000000e0007d0132008000eb006e18900009
:105690000000020000000000780137006e18900042
:1056a000e00090006e18900010089000000040008c
:1056b000808140006e18900040019000be10900064
:1056c0001e109000008040000000400000004100db
:1056d00010007800800978006e1890000008900093
:1056e0008080e8006e189000010898006301370080
:1056f000fe109000f0ff200000806000001798006e
:105700006e189000a00090006e18900000089000a5
:1057100000004000008040000080e8001001780098
:10572000720f98006e189000e00090006e189000c4
:105730001008900000004000008040000080e90058
:1057400090017800530f98006e189000e0009000d0
:105750006e1890001008900000004000008040008b
:1057600010007800600f9800ee0890007e0890000e
:10577000808f50001f0039006e1890008008900044
:10578000600320000e004000010878006003200044
:105790000e004000fe0890001100980060032000f9
:1057a0000e0040006e09900022009800ee18900054
:1057b00020002000f0009800620320000e0141004c
:1057c00063002000610029006e189000006c020048
:1057d00000000000000020000000e000270132006f
:1057e0008000eb006e189000000002000000000036
:1057f000220137006e189000400190008e1090003a
:105800006e08900000804000000040000000410051
:10581000de099000030878006e18900010089000d0
:105820008080e9006e189000110898006e189000b2
:10583000000890008080e8006e1890000108980031
:105840000e0137006e189000e00090006e18900076
:105850001008900000004000008040009000780098
:10586000410f9800fe109000f00f200000816000b2
:10587000ce0890006e18900093fe0700300f98003d
:105880006e189000e00090006e18900010089000d4
:1058900000004000008040003e09900002087800af
:1058a0006e189000000890008000e8006e189000cc
:1058b00001089800f10037006e189000e000900099
:1058c0006e1890001008900000004000008040001a
:1058d0000080e90090017800230f98006e18900076
:1058e000e00090006e18900010089000000040004a
:1058f0000080400090007800110f9800fe1090008a
:10590000f00f200000806000800178001e099000e8
:10591000ae0890006e1890008cfd0700000f9800f4
:105920006e189000100890008000e9006e1890003a
:10593000110898006e189000e00090006e1890001a
:105940001008900000004000008040000e09900008
:10595000020878006e189000000890008000e800af
:105960006e18900001089800c40037007e10900067
:105970004400dd004480de00700798006e1890003f
:10598000800890007e009000808040006e1890009b
:1059900001089800b90037006e189000e0009000f0
:1059a0006e18900010089000000040000080400039
:1059b0000080e90090017800530798006e1890006d
:1059c000e00090006e189000100890000000400069
:1059d000008040009000780041079800fe10900081
:1059e000f00f200000806000800178004e019000e0
:1059f000de0090006e18900054fd070060079800cc
:105a00006e189000100890008080e9006e189000d9
:105a1000110898006e0090000000e0000d003200b8
:105a20007e1090004800de00610060000000e00091
:105a3000050032007e1090004900de006100600029
:105a40000000e00003003a0020002000300798002a
:105a5000090037006e189000a00090006e189000aa
:105a60000008900000004000008040000080e80036
:105a700010007800300798006e0090000000e000f1
:105a8000110032006e189000a00090006e18900077
:105a90000008900000004000008140006e18900057
:105aa000a00090006e1890000008900000004000d8
:105ab00000804000900078000020200000807000ee
:105ac00000097800100037006e189000a0009000c8
:105ad0006e18900000089000000040000081400017
:105ae0006e189000a00090006e18900000089000c2
:105af000000040000080400090007800f0df2f00a0
:105b000000806000000978006e1890008008900006
:105b10003e009000808040006e18900001089800c0
:105b2000560037006e189000a00090006e1890008c
:105b30000008900000004000008040000080e80065
:105b400010017800220798006e189000a0009000c5
:105b50006e18900000089000000040000080400097
:105b60006400400090017800130798001e00900028
:105b700000004000800178006e189000c000900086
:105b80002e0090000000400000814000fe109000b8
:105b9000f0ff2000808060006e189000006c020012
:105ba000000000006e18900000089000e300400024
:105bb0006e1890000108980030003700fe10900029
:105bc000f0ff2000808060006e189000583e0200b8
:105bd000000000006e189000000890008000e800af
:105be0006e1890000108980024003700fe10900005
:105bf000f0ff2000008f60006e18900060019000a0
:105c00006e189000100890008000e8006e18900058
:105c1000110898006e1890001008900000004000d5
:105c2000800041006e189000000890000000e8001d
:105c3000800878006e1890009e0078000108980097
:105c40000e0037006e189000e00090006e18900073
:105c50001009900002007800000040000080400021
:105c600010007800800078006e18900001089800fd
:105c70008200e9006e189000110898000080fa0078
:105c8000000006000e00fa00200798003107980077
:105c90000f007800600798000f0078004007980018
:105ca0003e009000e407020000000000000f7800b2
:105cb0009e007800638040000000e8000000e800db
:105cc0000000d100000040008f00780051079800cc
:105cd00080874700de0090000100e8000000d1004e
:105ce00000004000500798005e00900010079800e8
:105cf000000020000000e00004003200be00900020
:105d00002e0090000000020000000000ae00900095
:105d100020002000f00098001e0090008000780015
:105d20002e00900000089000800878001e00780087
:105d3000804078001e009000214098001e009000d6
:105d400063004000be0090001e017800ac07020016
:105d5000000000009e007800638040001e0190005b
:105d600080017800910029002e009000006c020054
:105d700000000000ce079000ee0790000080fa00bf
:105d8000000006000600fa00100798000000eb0073
:105d9000000f7800130037001e0078009e0090006e
:105da0000000400074004000e08078001e00900079
:105db00000089000808f500009003a001e009000fb
:105dc00070009000800078000110a0001e0090007c
:105dd000710098001000200020079800070037008d
:105de0001e0fe8001e009000201890009e0f50002b
:105df000e9ff3e000000eb00200798002e00900015
:105e00000080fa00000006000400fa00000f78008d
:105e1000110798001e007800700090008000780044
:105e20000120a0001e007800710098001e00900064
:105e30000000e00019003200050037001e00780065
:105e400047fd07001e0090000000e90010079800c1
:105e50001e00780070009000610060000004a20045
:105e60000004e00019003a001e0078007000900065
:105e70004200de00610060000004a2000004e000b7
:105e800012003a001e0090000000e000ebff3a0014
:105e90000e0037001e00780031fd07001e0078005c
:105ea00070009000610060000004a2000004e000a7
:105eb00006003a001e007800700090004200de00ec
:105ec000610060000004e000f2ff3a001e0078006c
:105ed000f0009000b0ff2f00808060001e0078006e
:105ee000710098000080fa00000006000400fa002b
:105ef000000f7800110798001e00780070009000d5
:105f0000800078000120a0001e0078007100980039
:105f10001e0090000000e000330032001200370045
:105f20001e00780097ff07000000e0000900320023
:105f30001e00780070009000800078000110a00022
:105f40001e007800710098001e007800b400070061
:105f5000370037001e00780001fd07001e0090008a
:105f60000000e900100798001e0078007000900003
:105f7000610060000004a2000004e00026003a0076
:105f80001e007800700090004200de00610060009a
:105f90000004a2000004e0001f003a001e00900070
:105fa0000000e000deff3a001b0037001e00780012
:105fb00074ff07000000e000090032001e007800b6
:105fc00070009000800078000110a0001e00780092
:105fd000710098001e00780091000700140037003f
:105fe0001e007800defc07001e00780070009000a4
:105ff000610060000004a2000004e00006003a0016
:106000001e007800700090004200de006100600019
:106010000004e000e5ff3a001e007800f000900068
:10602000b0ff2f00808060001e0078007100980093
:106030000080fa00000006000600fa00000f780059
:10604000110798001e007800700090000000a20068
:10605000610060000004e000030032000000eb007b
:1060600020079800160037001e007800700090008e
:106070000000d100610060000004e0000300320075
:106080000000eb00200798000d0037001e0078008c
:10609000201890000000e000040032009e009000f4
:1060a0001e00780091ff0700030037009e0090005b
:1060b0001e00780054ff0700100020002007980001
:1060c0002e0090000080fa00000006000600fa0092
:1060d000000f7800110798001e007800201890002b
:1060e000ef0f50000d003e001e007800a018900039
:1060f0001e01780001804000740040009e01900065
:10610000033079008100e8001e0078002118980013
:106110001000200020079800020037008001eb00eb
:10612000230798002e0090000080fa00000006006f
:106130000a00fa0020079800310798000000eb00e1
:1061400010079800250037001e009000ae00900058
:106150000000400074004000e08078003e009000a5
:10616000808f50001a003a002e00900020189000f6
:106170008000e9002e009000211898001e00900079
:10618000000f78000b0037001e0178001e00e800a9
:10619000ae0090000000400074004000e0817800f4
:1061a000ae009000020041007400400003b078008f
:1061b0001e0fe8002e009000201890009e0f500047
:1061c000f1ff3e0010002000400798000a00370051
:1061d0001e0090000000e800100798002e009000bc
:1061e000a01890001e009000808f5000d6ff3e0047
:1061f0000000eb00400798004e0090000080fa007d
:10620000000006000200fa00000f78009e007800ef
:106210000000eb00a01898000080fa0000000600c3
:106220000600fa00200798002e0090000008900059
:10623000000f78002e00900070009000100798006a
:10624000430020000e017800a10029002e009000dc
:10625000006c0200000000000080fa000000060050
:106260000600fa00200798000000eb0010079800d5
:106270001b0037002e009000a00090001e00900030
:106280000000400000804000100f78001e007800e1
:106290004c00de00ea0f50000e003a002e00900085
:1062a000a00090001e00900000004000008140000f
:1062b0002e009000a00090001e0090000000400002
:1062c0000080400090007800f0df2f000080600028
:1062d000000978001e0090000000e80010079800f8
:1062e0002e009000900090001e009000808f5000c3
:1062f000e0ff3e000080fa00000006002400fa00e3
:10630000400f9800510f9800620f9800730f98008b
:10631000de08900000002a00808f50000a003a003a
:106320006e08900090007800010f98000e08900011
:10633000e40f5000ee003e004e0890007a6c020020
:1063400000000000ea003700de08900010012a007b
:10635000808f500009003a0050002000100f980074
:106360007201470023002000c10029004e08900060
:10637000006c020000000000dd0037007e08900085
:106380000000e000da0032006e0890009000780013
:106390004e08900010007800808f5000d4003a0022
:1063a0006e0890000080e800600f98007e08900062
:1063b0000000e900700f98005e0890006101b800cd
:1063c000f0ff2500f1ff2f0002014000838148000b
:1063d0000217980013179800f00020000100200019
:1063e0000e1190009e119000800f5100818f590076
:1063f000bf003e000e1090009e1090000060010053
:106400000f0037002d0037003f0037004d003700e8
:10641000550037005e003700630037006500370025
:1064200073003700770037007900370085003700a8
:10643000a0003700a3003700a6003700a9003700ee
:106440006e08900090007800710798007e08900018
:106450000000e900600798000000eb00500798007a
:10646000120037004e08900020019000fe009000be
:106470005e009000008040000000400000014100ec
:106480005e00900000004000800078006e089000e0
:10649000008040000080e8001000780000097800cb
:1064a0005e0090000000e80050079800de009000b9
:1064b0006e009000808f5000eaff39004e08900077
:1064c00021002000710098004e08900064ff070032
:1064d000000020000000e000030032004e089000a1
:1064e00000000200000000008080eb004e089000d9
:1064f0006afa07000000e0007d003a004e089000b4
:1065000047ff07007a0037004e089000f000900027
:10651000d0ff2f00808060004e089000710098002e
:106520004e0890003eff0700000020000000e00041
:106530006f0032004e0890000000020000000000d2
:106540006b0037004e0890007000900080007800cb
:106550000110a0004e089000710098004e089000b5
:106560002fff0700620037004e0890007000900077
:10657000610060000004e0005d0032004e08900001
:1065800077fb07004e08900025ff070058003700f2
:10659000ce08900020002000f00098004e089000e7
:1065a0001fff0700520037004e0890001cff070035
:1065b0004f0037006e08900010007800200f980000
:1065c000ae0890004e089000c0fe07000080fb005f
:1065d000300f98007401470043002000b1002900eb
:1065e0004e089000006c02000000000040003700e0
:1065f0006e089000900078004e089000ccfe0700d6
:106600003b0037004e089000fefe070038003700c0
:106610006e08900010017800420798006e08900004
:106620000080e80090017800330798003e01900058
:10663000ce0090004e089000386c02000000000070
:106640002b0037006e08900090007800210798001a
:106650007e0890000000e900100798000000eb00a1
:10666000000f78000f0037004e089000c000900027
:106670002e0090001e0040000000400000814000fd
:106680001e00780000004000800078006e08900036
:10669000008040000080e8001000780000097800c9
:1066a0001e0fe8001e0090009e0f1000eeff390044
:1066b0000f0037004e089000024302000000000067
:1066c0000b0037004e0890009a43020000000000c3
:1066d000070037004e089000503e02000000000006
:1066e000030037004e0890007a6c020000000000a2
:1066f0000080fa00000006000c00fa002007980055
:1067000031079800420798004e00900090007800f2
:10671000110798001e0090000000e0000a003500fc
:106720009e0090002e009000b7f907008000eb005b
:10673000510798000000e00020003a0010002000ff
:10674000500798001d0037009e009000f0ff2900c0
:10675000808f5000170036004e0090000080e80047
:10676000100f78009e00900000002a00808f5000db
:10677000040032009e00900010012a00808f50001b
:1067800003003a008000eb00510798000b0037002f
:106790002e009000100078008000eb005107980058
:1067a0009e0f500005003200100020005007980096
:1067b0000200370011002000510798005e00900091
:1067c0000080fa00000006000200fa009c8a020025
:1067d000000000000000eb00000f78000c00370004
:1067e0009e00e800800222006140780000417800ad
:1067f0009e0078008002220061407800804078008e
:10680000c0cdb3000a8b0200000000001e8fe8001c
:106810009e007800700d2000808f5000f0ff360041
:10682000a68a0200000000000080fa0000000600b6
:106830000200fa00881f78009c8a02000000000015
:106840000000eb00000f78000c0037001e04e80089
:106850009e0078008002220061407800804078002d
:10686000c0cdb300b08a0200000000008040780074
:1068700080022200017478001e8fe8009e007800dc
:10688000700d2000808f5000f0ff3600a68a0200b5
:10689000000000004f0478000080fa0000000600ad
:1068a0000600fa00000f78001e007800200798000c
:1068b0002e009000e10f50000b0032002e009000df
:1068c000e20f50000c0032002e0090000000e000ab
:1068d000010032000c003700b1062200c0c0b30036
:1068e000804878000b003700b106220080c0b3005a
:1068f0008048780007003700b106220020c0b300ae
:1069000080487800030037000080eb0010079800f3
:10691000020037000000eb00100798001e009000f6
:106920000080fa00000006000400fa00000f780062
:10693000400420009e0f10000600320010012000cd
:106940009e0f100003003200300320009e0f100045
:1069500007003a001e00780080407800b005220051
:10696000014878000000eb00100798000200370093
:106970000080eb00100798001e0090000080fa00d5
:10698000000006000400fa00000f78001e00e0007e
:1069900015003200000220009e0f1000120032008d
:1069a000000320009e0f10000f00320000042000a2
:1069b0009e0f10000c003200000520009e0f1000fa
:1069c00009003200000620009e0f10000600320071
:1069d000000620009e0f100003003200000120007e
:1069e0009e0f100007003a001e00780080407800db
:1069f00050052200014878000000eb0010079800c5
:106a0000020037000080eb00100798001e00900085
:106a10000080fa00000006000a00fa002007980033
:106a200031079800ae0090003e009000808f50002b
:106a3000030039000080eb00400798002100370078
:106a4000be00900030382000808f500003003600d8
:106a50008080eb00410798001a0037002e0090005c
:106a60000000e900200798002e00900020479800c1
:106a70002e0090004800de00304798003e00900055
:106a8000004f78003e0090004800de00104798005c
:106a900010032200be40900001487800300322001d
:106aa000ae40900001487800900322009e40900084
:106ab00001487800b00322001e4878000000eb0077
:106ac000400798004e0090000080fa000000060089
:106ad0000a00fa002007980031079800ae009000e5
:106ae0003e009000808f5000030039000080eb00d2
:106af000400798001e003700be009000301f2000a5
:106b0000808f5000030036008080eb004107980022
:106b1000170037002e009000204798002e009000ac
:106b20004800de00304798003e009000004f78009b
:106b30003e0090004800de001047980050032200fd
:106b4000be4090000148780070032200ae409000e3
:106b500001487800d00322009e4090000148780050
:106b6000f00322001e4878000000eb004007980068
:106b70004e0090000080fa00000006000e00fa00af
:106b8000300798004107980052079800be00900017
:106b90004e009000808f5000030039000080eb0011
:106ba0006007980030003700ce009000301f2000b2
:106bb000808f5000030036008080eb006107980052
:106bc00029003700de00900030382000808f500010
:106bd000030036000080eb006007980022003700b9
:106be0003e009000404798003e0090004800de00c4
:106bf000504798004e009000204798004e009000ab
:106c00004800de00304798005e0090001047980072
:106c10005e0090004800de00004f7800900b2200dc
:106c2000de40900001487800b00b2200ce4090007a
:106c300001487800d00b2200be4090000148780047
:106c4000f00b2200ae40900001487800100c2200aa
:106c50001e487800300c22009e40900001487800c9
:106c60000000eb00600798006e0090000080fa00c2
:106c7000000006000600fa0010079800210798009f
:106c80001e0090000000e000060032002e00900080
:106c90000000e00003003200a0ccb300004f7800f9
:106ca0000e0037001e0090000000e00003003200dc
:106cb000a0c4b300004f7800080037002e009000f9
:106cc0000000e00003003200a0c8b300004f7800cd
:106cd00002003700a0c0b300004f78009e4078004b
:106ce00070052200014878000080fa0000000600cc
:106cf0000600fa0020479800314798000000eb009a
:106d0000000f78000e0037009e00780080022200fd
:106d1000e14078002e40900080cf500007003a00fc
:106d20009e00e800800222003e41900082707800c0
:106d30000000eb0020079800070037001e8fe800d6
:106d40009e007800700d2000808f5000eeff36000e
:106d50000081eb00220798002e0090000080fa00ce
:106d6000000006000800fa0020479800210798005c
:106d70000000eb00000f78000f0037009e00780045
:106d800080022200e14078002e40900080cf500029
:106d900008003a009e00e80080022200e1407800ee
:106da0002e009000014878000000eb0030079800aa
:106db000070037001e8fe8009e007800700d20004d
:106dc000808f5000edff36000080eb003007980008
:106dd0003e0090000080fa00000006000200fa0069
:106de000004f780011479800100422009e40900048
:106df00001487800300422001e4878000080fa0024
:106e0000000006000800fa00004f780011479800c3
:106e1000224798003347980044479800f0c4b300d5
:106e20009e4f1000030036000080eb0030079800f2
:106e300010003700500422001e4878007004220021
:106e40009e4090000148780090042200ae409000df
:106e500001487800b0042200ce409000014878003c
:106e6000d0042200be409000014878000000eb00f2
:106e7000300798003e0090000080fa0000000600f5
:106e80000400fa00008fbe001e00be004a09dd00ab
:106e90004600de0000007100c608de008040780079
:106ea00010052200014878001e00be004209dd00e6
:106eb0004e00de0000007100ce08de008040780049
:106ec000f004220001487800310522000040eb0068
:106ed000804878000080fa00000006000200fa00f6
:106ee000004f7800d00522001e4878000080fa008c
:106ef000000006000200fa00000f78001e00e0000b
:106f000007003200d00622009040780000c8b3008d
:106f100080c07000d00622000148780006003700cb
:106f2000d006220010407800804078000174a10053
:106f3000d0062200014878000080fa000000060018
:106f40000400fa00004f780011479800224798008b
:106f5000100722001e487800300722009e40900053
:106f60000148780050072200ae40900001487800a8
:106f70000080fa00000006000200fa00004f7800ce
:106f8000114798001e4078007f4060000045b00027
:106f900080407800700722000148780090072200a6
:106fa0009e409000014878000080fa000000060032
:106fb0000600fa0010079800414798004e409000e4
:106fc0000000fb00630060004500dd0080407800a9
:106fd00000c8b30000c0400080407800f00f2200dd
:106fe000014878000000eb00000f78000c0037002b
:106ff0001e00780000004000320520000001410022
:107000001e007800800078001e0090000080400084
:107010009040780080022200017178001e0fe80085
:107020001e007800e10f5000f1ff36000080fa00ea
:10703000000006000000fa009c8a02000000000028
:10704000f00f22001040780000417800e00f22008d
:107050001040780080407800c0cdb3000a8b020059
:1070600000000000a68a02000000000000092200c3
:1070700090407800a007220010407800020007002e
:107080000080fa00000006000600fa004047980061
:10709000514798000000eb00000f78009c8a020026
:1070a000000000000000eb00100798001c003700f3
:1070b0009e00900080022200e14078004e40900047
:1070c00080cf5000130039009e0090008002220003
:1070d000e14078005e40900080cf50000d003e00ff
:1070e0001e0090008000e8008002220061407800cd
:1070f000004178009e0090008002220061407800ec
:1071000080407800c0cdb3000a8b02000000000070
:107110001e0fe8001e0090000080e8001007980095
:107120009e009000700d2000808f5000e0ff360020
:10713000a68a0200000000001e0078000080fa000d
:10714000000006000400fa00100798000000eb00a1
:10715000000f78000c0037001e007800000040008f
:10716000b2062000000141001e0078008000780077
:107170001e009000008040009040780080022200b5
:10718000017178001e0fe8001e007800e10f50002a
:10719000f1ff36000080fa00000006000200fa004d
:1071a000004f780011479800500a22001e487800ce
:1071b000700a22009e409000014878000080fa008a
:1071c000000006000200fa00004f78001147980006
:1071d000900a22001e487800b00a22009e409000cb
:1071e000014878000080fa00000006000200fa0062
:1071f000004f780011479800d00a22001e487800fe
:10720000f00a22009e409000014878000080fa00b9
:10721000000006000200fa00004f78001e80fb000c
:107220004400dd006f40400080407800500c220098
:10723000014878000080fa00000006000200fa0011
:10724000004f7800114798001e80fb004400dd00cd
:10725000804078001e4090006f40600000c04000f9
:1072600080407800700c2200014878000080fa000d
:10727000000006000200fa00004f78001147980055
:107280001e4090000080fb004400dd00804078003c
:107290001e4078006f40600000c0400080407800d1
:1072a000900c2200014878000080fa0000000600df
:1072b0000400fa00008fbe001e00be004088de0001
:1072c000cf80de0080407800b00c220001487800ba
:1072d0001e00be004809dd004800de00000071000d
:1072e000c888de0080407800d00c22000148780079
:1072f0001e00780080407800f00c220001487800e1
:107300000080fa00000006000200fa00004f78003a
:10731000100d22001e4878000080fa0000000600d0
:107320000400fa00000f7800110798001e00780092
:107330004800de0080407800700d2200014878008f
:107340001e00780080407800900d220001487800ef
:107350001e0090004800de0080407800b00d220042
:10736000014878001e00900080407800d00d220077
:10737000014878000080fa00000006000600fa00cc
:10738000004f780011479800224798003347980033
:107390004447980055479800f00d2200ae409000f9
:1073a00001487800100e2200be409000014878008d
:1073b000300e22001e487800500e22009e409000a1
:1073c00001487800700e2200ce40900001487800fd
:1073d000900e2200de409000014878000080fa0004
:1073e000000006000a00fa00000f7800110798005c
:1073f0002207980033079800200d20001e0f400040
:107400001e009000200db000100798002e00900084
:1074100067004000200798003e0090006700400091
:10742000300798009e00900020352000808f50008b
:10743000030036000080eb00400798004900370049
:10744000be009000701e2000808f500003003600a8
:107450000080eb0040079800420037001e009000bb
:107460009e0f100004003100ae0090003e0090001e
:10747000808f5000030039000080eb004007980027
:1074800038003700501a20009e0f10000c00360004
:107490009e00900090272000808f500008003e0042
:1074a000ae009000700a2000808f5000040036006b
:1074b000be00900060142000808f50000300360052
:1074c0000080eb0040079800260037001e0078007f
:1074d0004800de0080407800b00e220001487800ad
:1074e0001e00780080407800d00e2200014878000d
:1074f0001e0090004800de0080407800f00e220060
:10750000014878001e00900080407800100f220093
:10751000014878002e0090004800de00804078008e
:10752000300f2200014878002e0090008040780043
:10753000500f2200014878003e0090004800de0015
:1075400080407800700f2200014878003e009000d3
:1075500080407800900f2200014878000000eb0086
:10756000400798004e0090000080fa0000000600de
:107570000600fa0010079800210798001e009000ee
:107580000000e000060032002e0090000000e00045
:1075900003003200c0c3b300004f78000e00370074
:1075a0001e0090000000e00003003200c0c2b300e3
:1075b000004f7800080037002e0090000000e00027
:1075c00003003200c0c1b300004f78000200370052
:1075d000c0c0b300004f78009e407800b00f22007a
:1075e000014878000080fa00000006000200fa005e
:1075f000000f78001e00e00007003200f0052200b6
:1076000090407800f0c7b30080c06000f005220011
:107610000148780006003700f0052200904078000d
:1076200000c8b30080c07000f00522000148780057
:107630000080fa00000006000400fa00000f780045
:10764000110798001e00e00007003200f00522003c
:1076500090407800f0cbb30080c06000f0052200bd
:107660000148780006003700f005220090407800bd
:1076700000c4b30080c07000f0052200014878000b
:107680001e0090000000e00007003200f00522001c
:1076900090407800f0cdb30080c06000f00522007b
:1076a0000148780006003700f0052200904078007d
:1076b00000c2b30080c07000f005220001487800cd
:1076c0000080fa00000006000a00fa0050052200bf
:1076d000104078000080fb00400798000003200065
:1076e000ce009000808f5000310032000003200057
:1076f000ce009000808f50000b003c004e009000a8
:10770000f00f50002200320000022000ce00900056
:10771000808f5000220032004e0090000000e000f8
:10772000170032003600370000052000ce00900020
:10773000808f50002600320000052000ce0090000f
:10774000808f500005003c0000042000ce00900017
:10775000808f50001a0032002900370000062000f8
:10776000ce009000808f50001d00320000072000e6
:10777000ce009000808f50001d00320020003700a6
:107780000000280001072000008fbe002000370005
:107790000000200061092000008fbe001c0037009f
:1077a0000000240081032000008fbe001800370075
:1077b00000002200c1012000008fbe00140037002d
:1077c00000002100e1002000008fbe001000370003
:1077d0000080200071002000008fbe000c003700e8
:1077e0000040280031002000008fbe000800370054
:1077f00000202c0011002000008fbe000400370084
:107800006000b80020079800310798000b0037008f
:10781000b006220010407800ec4f500004003a00ff
:107820001e00be000000400081804800008fbe00a6
:107830001e00be0020079800310798002e0090001f
:10784000be0090000080fa00000006001000fa0060
:1078500020079800310798004207980053079800c6
:10786000640798005e0090000000e000030035000f
:107870005e009000e30f5000030034000080eb0036
:1078800070079800600037006e0090000000e00074
:10789000030035006e009000e30f50000300340039
:1078a0000080eb00700798005700370086ff070044
:1078b0000002be0084007800606a2000000bb8005f
:1078c0006020b9000701780000014100606a2000d3
:1078d00000a8b90000014100820378002e0090004a
:1078e0006101b9000600be00de04020000000000d5
:1078f0001007980074ff07000002be0084007800a3
:10790000606a2000000bb8006020b9000701780011
:1079100000014100606a200000a8b9000001410098
:10792000820378003e0090006101b9000600be00ad
:10793000de04020000000000000f78001e0090002e
:107940004800de00804078003006220001487800c0
:107950001e00900080407800500622000148780008
:107960001e0078004800de0080407800700622008b
:10797000014878001e0078008040780090062200c0
:10798000014878004e0090000000e000070032003f
:10799000f005220010407800804078000144a000eb
:1079a000f00522000148780006003700f0052200ab
:1079b00090407800f0ceb30080c06000f005220057
:1079c000014878006e009000e34060005e00900087
:1079d000630060004200dd0000c14000f0052200ad
:1079e000104078008040780000cfb30000c06000f5
:1079f0000040410080407800f005220001487800f6
:107a00000000eb00700798007e0090000080fa00f4
:107a1000000006000200fa00000f7800e0ee2100ee
:107a20000080fa00000006000200fa00000f780053
:107a3000e05d29000080fa00000006000800fa005e
:107a4000300798003e0090002c00070020079800a7
:107a50009c8a0200000000000000eb001007980064
:107a60001f0037001e00900000004000804078009a
:107a700000ccb300b08a0200000000000000fb0050
:107a80004800dd00000f78001e009000000040005c
:107a90000040e8008040780000ccb300b08a0200cb
:107aa000000000000000fb001e0f70003e00900070
:107ab000c00090002e009000000040008080400038
:107ac0001e007800800878002e0090000000e8007a
:107ad000200798001e0090000000e80010079800a2
:107ae0001e009000e20f5000deff3600a68a020062
:107af000000000000080fa00000006000200fa000a
:107b0000000f78001e007800600190001e007800d1
:107b10009008900001007800000040000000410043
:107b2000100178008100e9001e007800110898001b
:107b3000020078000080fa00000006000600fa004b
:107b4000200798002e009000ecff07001007980017
:107b50002e009000e9ff0700000f78002e00900033
:107b6000c00090001e00780000004000008040002f
:107b7000100178002e009000c00090001e009000c0
:107b80000000400000804000100078008200780073
:107b90001678020000000000de76020000000000ff
:107ba0000080fa00000006000800fa003007980084
:107bb0003e009000d1ff0700200798003e00900093
:107bc000c00090002e0090000000400000804000a7
:107bd00010007800cf80de00c808dd000080fd00c6
:107be000804078000040eb00008fbe001e00be0009
:107bf000aa78020000000000de760200000000000b
:107c00000080fa00000006000800fa003007980023
:107c10003e009000b9ff0700200798003e0090004a
:107c2000b6ff0700100798003e009000b3ff070062
:107c3000000f78003e009000c00090001e00780009
:107c400000004000008040001000780000417800f3
:107c50003e009000c00090001e0090000000400018
:107c60000080400010007800804178003e009000c5
:107c7000c00090002e0090000000400000804000f6
:107c800010007800834078005a780200000000005d
:107c9000de760200000000000080fa00000006000e
:107ca0000200fa00000f78000080fa0000000600d1
:107cb0000400fa00000f7800110798001e009000e1
:107cc0008000400020ff21000080400090007800ec
:107cd0001e007800010001000080fa00000006008c
:107ce0000200fa00000f7800e0fb21000080fa009b
:107cf000000006000200fa00004f78000e00780035
:107d000011002000968b020000000000ae8b0200e4
:107d1000000000000000e000fcff3a000080fa00d4
:107d2000000006000200fa00000f78000e00780044
:107d300021002000968b020000000000ae8b0200a4
:107d4000000000000000e000fcff3a000080fa00a4
:107d5000000006000800fa001007980021079800ac
:107d6000320798003e0090000080e900edff070018
:107d700060fa8000ebff07000000eb00000f7800c6
:107d8000080037002e009000904078002e009000f0
:107d90000000e8002007980001407800d5ff0700a8
:107da0001e0fe8003e0090009e0f1000f5ff390006
:107db0000080fa00000006000400fa00214d2100b6
:107dc0000040eb008048780070880200000000004e
:107dd0000f0037004288020000000000020020006f
:107de000a33f240000050200000000000000e000a6
:107df00001003c0006003700214d210010c0b300f7
:107e0000804878000000eb00100798000a00370057
:107e1000d08b0200000000000000e000edff320007
:107e20000e007800d88b0200000000001e40780091
:107e30000080fb00100798001e0090000080fa00f0
:107e4000000006000400fa00dbff07000080fb00d2
:107e5000000f7800204d2100104078000004e00061
:107e6000030032000000eb00100798000d003700ff
:107e7000d1ff07000080fb004800dd001e0f7000ee
:107e8000204d2100104078000004e0000300320083
:107e90000000eb0010079800020037001e00780079
:107ea000100798001e0090000080fa0000000600f5
:107eb0001000fa0030079800410798005207980018
:107ec000630798000000eb0020079800d08b0200a9
:107ed000000000000000e00033003200d9ff07007e
:107ee0000080e80010079800204d21001040780025
:107ef0000004e000030032000000eb00700798006f
:107f00002b0037009e0090005e009000808f500094
:107f1000030036000000eb007007980024003700d3
:107f2000c8ff0700800078006e009000010878000c
:107f3000204d2100104078000004e00003003200d2
:107f40000000eb0070079800190037000000eb00fc
:107f5000000f78000f00370097ff0700804078007f
:107f60004e009000014878004e0090000000e800ac
:107f700040079800204d2100104078000004e000e8
:107f8000030032000000eb00700798000800370083
:107f90001e0fe8001e0090009e0f1000eeff39003b
:107fa0001e009000200798002e0090007007980097
:107fb0007e0090000080fa00000006000400fa0035
:107fc000100798001e0090000000e00002003d0035
:107fd0000000eb00100798009e0090003006200083
:107fe000808f5000020034003006200010079800f7
:107ff000b0770200000000000000e0000100320045
:10800000100037001e0090004500dd0052002000e7
:10801000110009000200d800000f78001e0078004f
:10802000160020008500200044002000031e2000d0
:10803000420020008000eb002076020000000000db
:108040000f0037001e0090007800b9005200200099
:10805000110009000200d800000f78009e0078008f
:10806000160020004500200084002000430020006e
:10807000021e200000052000207602000000000003
:108080000080fa00000006000c00fa00889fbe0085
:10809000d1a88000a0608000808f500014003200c2
:1080a000d1a8800080c12f00808f500009003500ca
:1080b000d0a8800020079800803e2000ae009000ed
:1080c000808f500005003400803e2000200798007b
:1080d0000200370081c12f00210798002e00900078
:1080e000a0608800a0608000ae7402000000000064
:1080f000e1a8800090608000808f50001400320062
:10810000e1a8800080c12f00808f50000900350059
:10811000e0a8800010079800803e20009e0090009c
:10812000808f500005003400803e2000100798002a
:108130000200370081c12f00110798001e00900037
:10814000906088009060800032750200000000009e
:1081500030dc8000e10f4000470032000000eb00ff
:10816000000f7800280037001e0078000000400053
:10817000a104200080804000404d2100008040008c
:108180001000780030079800be0090000100e00069
:10819000020032001000200030079800be0090005e
:1081a0001e007800d2440200000000001e04780087
:1081b0001e007800528702000000000000017800d5
:1081c00008004400e106200080804000404d21006e
:1081d00000804000020878001e0478001e0078002d
:1081e0000c87020000000000000178000800440035
:1081f000e105200080804000404d210000804000cb
:10820000020878001e0fe800710020009e8f100009
:10821000d5ff36000080eb0030dc880070a98000bc
:10822000400798004e0090000000e000020032007d
:1082300011002000410798004e0090008a4702007c
:108240000000000080a98000500798005e009000a8
:108250000000e000020032001100200051079800e9
:108260005e009000ca4702000000000080608000ad
:108270000000a000806088000000eb00000f780084
:10828000170037001e0478001e007800884c02009a
:10829000000000000001780008004400e107200011
:1082a00080804000404d210000804000020878009e
:1082b0001e0478001e0078003085020000000000d7
:1082c0000001780008004400211f20008080400049
:1082d000404d210000804000020878001e0fe80099
:1082e000200020009e0f1000e6ff3600a889020043
:1082f000000000000000e000530032000000eb002e
:10830000000f7800390037009e0178001e007800c9
:10831000800040006045210000804000100078008f
:108320004300de007f0060006300b90000017800b8
:10833000038041006108200080804000404d210002
:1083400000804000020878009e0178001e0078003e
:10835000800040006045210000804000100078004f
:10836000670060004301dd001e00780080004000cf
:108370006045210000804000100078004d00de00c4
:10838000000071006300b9000000d1000001780016
:1083900003804100e10f200080804000404d21001b
:1083a00000804000020878009e0178001e007800de
:1083b00080004000604521000080400010007800ef
:1083c0004800de007f0060006300b9000001780013
:1083d000038041006117200080804000404d210053
:1083e00000804000020878001e0fe800b003200063
:1083f0009e0f1000c4ff3600c1aa8000300181002a
:10840000808f50000a003200c0aa8000300189002d
:1084100030018100e9fe070011002000100020005b
:108420009a76020000000000de76020000000000e4
:1084300060452100f8880200000000008060800094
:108440000010a00080608800f875020000000000a5
:1084500010b688000c7602000000000020b68800ec
:10846000406d210064014000406d21008080e800e3
:10847000406d2100c4690200000000007c8a0200f7
:10848000000000000004e00004003200f487020055
:108490000000000090b6880006003700e0c2bf0070
:1084a0000080fb000000d100614060000080fb0004
:1084b00090b68800968702000000000060b6880031
:1084c00040022200104078008000fb0060b680006f
:1084d000808f500003003200806080000020a000e8
:1084e0008060880060b680008040780040022200f2
:1084f0000148780088840200000000000080fb0032
:1085000070b6880080b680000000e00013003400e0
:1085100042880200000000000004be0080b6800017
:10852000cf80de007c050200000000000001be00dc
:108530000800be0000050200000000000000e0008e
:1085400001003d00050037007088020000000000b7
:10855000806080000030a000806088004f04be0072
:108560000080fa00000006000400fa00000f780006
:1085700011079800100020008a4702000000000048
:10858000ffff37000000fa00e4890200000000004d
:10859000fa80020000000000987402000000000051
:1085a0002c8c020000000000168302000000000076
:1085b0000040eb002a54020000000000f2760200a6
:1085c00000000000200320007cfe070011002000b6
:1085d000100020009a76020000000000de76020003
:1085e0000000000040c7bf00614060000004e000e0
:1085f000020032004007a9000000fe000080fa00df
:10860000000006000800fa00300798000000eb00a8
:108610002007980000802f00f1072000008fbe0087
:10862000220020001e00be00140202000000000014
:1086300061c7bf0001c8b300014060000004e00052
:10864000fbff3a0050002000200798002e01900008
:108650001e00be00460202000000000061c7bf000d
:1086600001c8b300014060000004e000fbff3a00d5
:1086700000002f00f1072000008fbe000000eb007b
:108680002007980025003700220020001e00be00b1
:10869000140202000000000061c7bf0001c8b3005f
:1086a000014060000004e000fbff3a003e00900043
:1086b000a00090002e00900022002000811f780072
:1086c000110009000200d80001017800cf007800f5
:1086d0000000400000804000100078000001780099
:1086e0001e00be00460202000000000061c7bf007d
:1086f00001c8b300014060000004e000fbff3a0045
:1087000020002000010020001e0f40005e9748005e
:108710002e0090000080e80020079800ae00900036
:10872000f07f2000808f5000d7ff34000080fa00d7
:10873000000006000200fa00000f78000000fe00b2
:108740000080fa00000006000200fa00e6c2bf0046
:108750000080fb004600de00614060008080fb007e
:10876000e6c2bf000080fb004700de000080fb0087
:108770000000400080807000e7c2bf0061406000e0
:108780000080fb004200dd00008f70001e00e8004a
:1087900060fa8800c0f42100ce260200000000002c
:1087a0001e00e800a0a6880050002000c0a8880095
:1087b00020032000c0aa88001e00780002c3b30076
:1087c00082404000c0ee210001487800744702005a
:1087d000000000000080fa00000006000800fa0017
:1087e00068ff0700d8ff07000886020000000000ad
:1087f0003c5002000000000000802f00f107200024
:108800001007980021079800660147000002eb005e
:10881000230020001e009000ae00900064020200c1
:10882000000000003e009000e50f50002c003a00d0
:1088300000002f00f1072000100798002107980082
:108840000000eb00300798001900370081fa800023
:108850003e00900022002000811f780011000900d6
:108860000200d80001017800cf007800000040002d
:10887000008140000002eb00230020001e00900059
:10888000ae00900064020200000000001e00900094
:10889000ae00900062004000e080480010079800a1
:1088a000210798003e0090000080e8003007980003
:1088b000be009000f07f2000808f5000e3ff340066
:1088c0008080eb00c0f421004e2702000000000071
:1088d000813e2000c0f421001c3002000000000096
:1088e00060452100f8880200000000000000370009
:1088f000e5fd0700c0f42100846e020000000000c6
:10890000813e2000c0f421001c3002000000000065
:10891000d0fa80000000d1000000a20061006000d9
:108920000004e00005003a00d0fa80000000a20038
:10893000610060000004e000edff32008060800014
:108940000000cf00000f78001e00e000e8ff3200ba
:108950001e0fe9009e007800100020000100dd00dd
:108960000080ea0080007800806080000080600065
:108970008060880060fa8000b0a68800e0ff2f00c9
:108980009e005000c0f421004e27020000000000ad
:10899000813e2000c0f421001c30020000000000d5
:1089a000d3ff37000600fa00000f78001107980087
:1089b0001e007800200798002e009000e30f500062
:1089c000670032002e009000e30f500007003e00c9
:1089d0002e009000e10f50002e0032002e0090007b
:1089e000e10f500041003e000d0037002e009000c6
:1089f000e50f5000940032002e009000e50f50006b
:108a0000740039002e009000e60f5000ab003200d9
:108a10002e009000e70f5000c5003200da0037004a
:108a20001e009000e10f50000f003600c4c2bf00ce
:108a30000080fb004600de00614060000004a200f0
:108a400061406000614060004601dd00412c200073
:108a500091407800f0cbb30000c06000024070008d
:108a6000c4e2b7001e0137001e00900061406000a4
:108a7000614060004601dd00412c200091407800fb
:108a8000f0cbb30000c0600002407000c4e2b70049
:108a9000130137001e009000e10f50000b0036005c
:108aa000c4c2bf000080fb004700de000004a2003b
:108ab00061406000c700dd00c4c2bf000074a100b7
:108ac00001407000c4e2b700050137001e009000ad
:108ad00061406000c700dd00c4c2bf000074a10097
:108ae00001407000c4e2b700fd0037001e00900096
:108af000e10f50000f003600c5c2bf000080fb0030
:108b00000000d100614060000004a20061406000ec
:108b10006140600000414000512c200091407800ed
:108b2000d0cfb30000c0600002407000c5e2b700c3
:108b3000eb0037001e009000614060006140600063
:108b400000414000512c200091407800d0cfb3006c
:108b500000c0600002407000c5e2b700e0003700ce
:108b60001e009000e10f50000f003600c5c2bf008c
:108b70000080fb004400de00614060000004a200b1
:108b800061406000614060004401dd00512c200024
:108b900091407800f0ceb30000c060000240700049
:108ba000c5e2b700ce0037001e00900061406000b3
:108bb000614060004401dd00512c200091407800ac
:108bc000f0ceb30000c0600002407000c5e2b70004
:108bd000c30037001e009000e10f50000f00360068
:108be000c5c2bf000080fb004200de0061406000a3
:108bf0000004a20061406000614060004201dd00ad
:108c0000512c200091407800b0cfb30000c060002c
:108c100002407000c5e2b700b10037001e009000ae
:108c200061406000614060004201dd00512c200085
:108c300091407800b0cfb30000c0600002407000e7
:108c4000c5e2b700a60037001e009000e10f5000fb
:108c50000f003600c5c2bf000080fb004500de00eb
:108c6000614060000004a20061406000614060005b
:108c70004501dd00512c200091407800f0cdb3007b
:108c800000c0600002407000c5e2b70094003700e9
:108c90001e00900061406000614060004501dd0001
:108ca000512c200091407800f0cdb30000c060004e
:108cb00002407000c5e2b700890037001e00900036
:108cc000e10f50000f003600c5c2bf000080fb005e
:108cd0004600de00614060000004a20061406000c8
:108ce000614060004601dd00512c20009140780079
:108cf000f0cbb30000c0600002407000c5e2b700d6
:108d0000770037001e009000614060006140600005
:108d10004601dd00512c200091407800f0cbb300db
:108d200000c0600002407000c5e2b7006c00370070
:108d30001e009000e10f50000b003600c5c2bf00be
:108d40000080fb004700de000004a20061406000dc
:108d5000c700dd00c5c2bf000074a1000140700063
:108d6000c5e2b7005e0037001e0090006140600061
:108d7000c700dd00c5c2bf000074a1000140700043
:108d8000c5e2b700560037001e0090006140600049
:108d9000c700dd00c5c2bf000074a1000140700023
:108da000c5e2b700c5c2bf000080fb004700de007f
:108db000614060004601dd00512c200091407800a8
:108dc000f0cbb30000c0600002407000c5e2b70005
:108dd000c5c2bf000080fb004600de0061406000ad
:108de000614060004501dd00512c20009140780079
:108df000f0cdb30000c0600002407000c5e2b700d3
:108e0000c5c2bf000080fb004500de00614060007d
:108e1000614060004201dd00512c2000914078004b
:108e2000b0cfb30000c0600002407000c5e2b700e0
:108e3000c5c2bf000080fb004200de006140600050
:108e4000614060004401dd00512c20009140780019
:108e5000f0ceb30000c0600002407000c5e2b70071
:108e6000c5c2bf000080fb004400de00614060001e
:108e70006140600000414000512c2000914078008a
:108e8000d0cfb30000c0600002407000c5e2b70060
:108e9000c5c2bf000080fb000000d100614060003f
:108ea000c700dd00c4c2bf000074a1000140700013
:108eb000c4e2b700c4c2bf000080fb004700de0070
:108ec000614060004601dd00412c200091407800a7
:108ed000f0cbb30000c0600002407000c4e2b700f5
:108ee0000080fa00000006000000fa00c4c2a900d9
:108ef000c4e2a900c522a900c582a900c542a900f3
:108f0000c5a2a900c5c2a900c5e2a9000080fa0057
:108f1000000006000200fa00000f78001000200098
:108f20009e0f10000f003600d0c2bf000080fb0073
:108f30004200de00614060000004a2006140600069
:108f4000614060004201dd00012d20009140780069
:108f5000b0cfb30000c0600002407000d0e2b700a4
:108f60000a0037001e007800614060006140600028
:108f70004201dd00012d200091407800b0cfb30008
:108f800000c0600002407000d0e2b7000080fa002c
:108f9000000006000200fa00000f78001000200018
:108fa0009e0f10000f003600d0c2bf000080fb00f3
:108fb0000000d100614060000004a2006140600038
:108fc0006140600000414000012d20009140780088
:108fd000d0cfb30000c0600002407000d0e2b70004
:108fe0000a0037001e0078006140600061406000a8
:108ff00000414000012d200091407800d0cfb30007
:1090000000c0600002407000d0e2b7000080fa00ab
:10901000000006000000fa00c4c2bf000080fb0090
:109020004600de006140600000c0ea006140600070
:10903000614060004601dd00412c20009140780035
:10904000f0cbb30000c0600002407000c4e2b70083
:10905000c4c2bf000080fb004700de0000c0ea0081
:1090600061406000c700dd00c4c2bf000074a10001
:1090700001407000c4e2b700c5c2bf000080fb0021
:109080000000d1006140600000c0ea006140600063
:109090006140600000414000512c20009140780068
:1090a000d0cfb30000c0600002407000c5e2b7003e
:1090b000c5c2bf000080fb004400de0061406000cc
:1090c00000c0ea0061406000614060004401dd00d2
:1090d000512c200091407800f0ceb30000c0600019
:1090e00002407000c5e2b700c5c2bf000080fb00af
:1090f0004200de006140600000c0ea0061406000a4
:10910000614060004201dd00512c20009140780058
:10911000b0cfb30000c0600002407000c5e2b700ed
:10912000c5c2bf000080fb004500de00614060005a
:1091300000c0ea0061406000614060004501dd0060
:10914000512c200091407800f0cdb30000c06000a9
:1091500002407000c5e2b700c5c2bf000080fb003e
:109160004600de006140600000c0ea00614060002f
:10917000614060004601dd00512c200091407800e4
:10918000f0cbb30000c0600002407000c5e2b70041
:10919000c5c2bf000080fb004700de0000c0ea003f
:1091a00061406000c700dd00c5c2bf000074a100bf
:1091b00001407000c5e2b7000080fa000000060020
:1091c0000000fa00c4c2bf000080fb004600de00c1
:1091d0006140600000c0ea006140600061406000e2
:1091e0004601dd00412c200091407800f0cbb30017
:1091f00000c0600002407000c4e2b7000080fa00c6
:10920000000006000000fa00c4c2bf000080fb009e
:109210004700de0000c0ea0061406000c700dd00da
:10922000c4c2bf000074a10001407000c4e2b700d6
:109230000080fa00000006000000fa00c5c2bf006e
:109240000080fb000000d1006140600000c0ea0027
:10925000614060006140600000414000512c2000ee
:1092600091407800d0cfb30000c060000240700091
:10927000c5e2b7000080fa00000006000000fa0016
:10928000c5c2bf000080fb004400de0061406000fa
:1092900000c0ea0061406000614060004401dd0000
:1092a000512c200091407800f0ceb30000c0600047
:1092b00002407000c5e2b7000080fa00000006001e
:1092c0000000fa00c5c2bf000080fb004200de00c3
:1092d0006140600000c0ea006140600061406000e1
:1092e0004201dd00512c200091407800b0cfb30046
:1092f00000c0600002407000c5e2b7000080fa00c4
:10930000000006000000fa00c5c2bf000080fb009c
:109310004500de006140600000c0ea00614060007e
:10932000614060004501dd00512c20009140780033
:10933000f0cdb30000c0600002407000c5e2b7008d
:109340000080fa00000006000000fa00c5c2bf005d
:109350000080fb004600de006140600000c0ea00c3
:1093600061406000614060004601dd00512c20003a
:1093700091407800f0cbb30000c060000240700064
:10938000c5e2b7000080fa00000006000000fa0005
:10939000c5c2bf000080fb004700de0000c0ea003d
:1093a00061406000c700dd00c5c2bf000074a100bd
:1093b00001407000c5e2b7000080fa00000006001e
:1093c0000200fa00000f78009e007800a0802400c0
:1093d00024810200000000000080fa000000060066
:1093e0000000fa00a0802400888102000000000034
:1093f0000080fa00000006000200fa00000f78006a
:109400001e00e000040035009e007800a0802400cb
:10941000da810200000000000080fa00000006006f
:109420000000fa0080182200104078000004e000dc
:109430000e003a008000eb007000200059fd07008c
:1094400080182200104078000080fb0011002000ee
:1094500054fd070080182200104078008040e8008a
:10946000801822000148780023003700801822006d
:1094700010407800e74f50000f003a00801822009b
:10948000104078000080fb000000e9008000eb0045
:1094900044fd070080182200104078000080fb0087
:1094a000110020003ffd0700811822000040eb0062
:1094b00080487800100037008018220010407800a3
:1094c0000080fb000000e9008000eb0035fd070094
:1094d00080182200104078000080fb00110020005e
:1094e00030fd070080182200104078008040e8001e
:1094f00080182200014878000080fa000000060071
:109500000200fa0090182200104078000080fb0052
:10951000000f78001e007800e20f50001c0032009f
:109520001e007800e20f500007003c001e0078008b
:109530000000e0000b0032001e007800e10f500038
:109540000c003200230037001e007800e30f5000ab
:10955000160032001e007800e40f50001a0032009e
:109560001c003700210020000000eb000dfd07006b
:1095700018003700210020001000200009fd07001e
:10958000210020007000200006fd070011003700b8
:10959000210020002000200002fd07002100200003
:1095a00060002000fffc07000a00370021002000b7
:1095b00030002000fbfc07002100200050002000ac
:1095c000f8fc0700030037002100200040002000c5
:1095d000f4fc07009018220010407800e34f500080
:1095e00006003e0090182200104078008040e800fd
:1095f00090182200014878000300370091182200db
:109600000040eb00804878000080fa00000006006f
:109610000000fa00a0182200104078000004e000ca
:1096200013003a00001b2200104078000004e00004
:109630000f003200a118220010c0b300804878004b
:109640008000eb000000eb00d6fc0700a018220011
:10965000104078000080fb0011002000d1fc0700c2
:10966000011b22000040eb008048780036003700e4
:10967000a0182200104078000004e00013003a0017
:10968000001b2200104078000004e0000f003a00a8
:10969000a118220070c0b300804878008000eb0061
:1096a0000000eb00bffc0700a0182200104078006b
:1096b0000080fb0011002000bafc0700011b220003
:1096c00010c0b300804878001f003700a0182200a7
:1096d00010407800e74f50000c003a00a11822001b
:1096e0000040eb00804878008000eb007000200014
:1096f000acfc0700a0182200104078000080fb009e
:1097000011002000a7fc07000f003700a01822005e
:1097100010407800e14f50000b003a00a1182200e1
:109720000040eb00804878008000eb001000200033
:109730009cfc0700a0182200104078000080fb006d
:109740001100200097fc07000080fa0000000600ce
:109750000200fa00b0182200104078000080fb00e0
:10976000000f78001e007800e10f50001500320055
:109770001e007800e10f500004003c001e0078003d
:109780000000e000080032001a0037001e007800d8
:10979000e20f5000120032001e007800e30f50006c
:1097a0001300320013003700210020000000eb00fe
:1097b0007cfc0700210020004000200079fc07000d
:1097c0000c003700210020001000200075fc07006d
:1097d000210020003000200072fc07000500370047
:1097e00021002000200020006efc0700010037004f
:1097f000bdfd0700b018220010407800e24f500075
:1098000006003e00b0182200104078008040e800ba
:10981000b01822000148780003003700b118220078
:109820000040eb00804878000080fa00000006004d
:109830000200fa00c0182200104078000080fb00ef
:10984000000f78001e007800e10f50001500320074
:109850001e007800e10f500004003c001e0078005c
:109860000000e000080032001a0037001e007800f7
:10987000e20f5000120032001e007800e30f50008b
:109880001300320013003700210020000000eb001d
:1098900044fc0700210020004000200041fc07009c
:1098a0000c00370021002000700020003dfc070064
:1098b00021002000500020003afc0700050037007e
:1098c000210020006000200036fc07000100370066
:1098d00085fd0700c018220010407800e24f5000bc
:1098e00006003e00c0182200104078008040e800ca
:1098f000c01822000148780003003700c118220078
:109900000040eb00804878000080fa00000006006c
:109910000a00fa00100798000000eb00000f780022
:109920007c8a0200000000000004e0003a003200df
:10993000c01722009040780000c4b30080cf5000d0
:1099400008003a002214220001142200e013220031
:10995000f068020000000000c11722000040eb0088
:10996000804878001e009000300798003e0090006c
:10997000e10f5000110032003e009000e10f500056
:10998000040039003e009000e20f50001500320044
:109990001e003700010a810050098100008f50002d
:1099a0001e007800c480de001e0078004680de00c5
:1099b00080805000210798004c003700f109810099
:1099c00040098100008f50001e007800c480de0036
:1099d0001e0078004680de0080805000210798003d
:1099e00042003700110a8100100d8100008f5000e5
:1099f0001e007800c480de001e0078004680de0075
:109a0000808050002107980038003700a0292000ee
:109a100020079800350037001e009000400798008e
:109a20004e009000e10f5000140032004e009000f4
:109a3000e10f5000040039004e009000e20f50008a
:109a40001b003200270037009e009000d20b8100df
:109a5000200320000088b900020040008000400080
:109a600080a3210000804000900078004009810020
:109a700080805000210798001c0037009e00900055
:109a8000d20b8100200320000088b90002004000b2
:109a90008000400080a321000080400090007800fa
:109aa0005009810080805000210798000f00370086
:109ab0009e009000d20b8100200320000088b90096
:109ac000020040008000400080a321000080400090
:109ad00090007800100d81008080500021079800d0
:109ae00002003700a0292000200798002e009000d7
:109af0000080fa00000006001400fa0050079800e9
:109b0000610798006000b80030079800410798008e
:109b10007c8a0200000000000004e0005c003200cb
:109b2000c01722009040780000c4b30080cf5000de
:109b300008003a002214220001142200e01322003f
:109b4000f068020000000000c11722000040eb0096
:109b500080487800001a2200104078000004e000dd
:109b60001b0032005e009000000f98000e0890006d
:109b7000e10f50000b0032000e089000e10f500082
:109b8000040039000e089000e20f50000900320076
:109b90000c003700626902000000000070079800a6
:109ba000760037003e690200000000007007980050
:109bb00072003700866902000000000070079800fc
:109bc0006e003700a0292000700798006b00370056
:109bd0005e009000100f98001e089000e10f5000ea
:109be000120032001e089000e10f500004003900fe
:109bf0001e089000e20f50001700320021003700cd
:109c0000000a8100000f78001e007800c480de008a
:109c10001e0078004680de0080805000008020001a
:109c2000808040007107980054003700f0098100df
:109c3000000f78001e007800c480de001e0078004f
:109c40004680de0080805000008020008080400040
:109c50007107980049003700100a8100000f780052
:109c60001e007800c480de001e0078004680de0002
:109c700080805000008020008080400071079800a4
:109c80003e003700a0292000700798003b003700f5
:109c90005e009000e20f500031003e006e00900028
:109ca0000000e0002e003200ee00900020032000b3
:109cb000808f50002a003e000000eb002007980033
:109cc000d10b81006e009000008050003003b00086
:109cd00022032000110009000280d8008000fd004e
:109ce000100798001a003700de0090001e01900057
:109cf000200320000088b9000200400080004000de
:109d000080a3210000804000100078006101b900ac
:109d10003e009000ce00900000004100818049008c
:109d200030079800410798002e0090000000e800de
:109d3000200798001e0090000000e8002203200089
:109d4000110009000200d8008000fd0010079800f3
:109d5000ae0090006e009000808f5000e2ff39004e
:109d60006e0090006101b8003e009000ce009000af
:109d7000de04020000000000700798007e009000e2
:109d80000080fa00000006000000fa007c8a020051
:109d9000000000000004e0000a0032000000eb00b8
:109da000dbfe07006009890010002000d8fe0700d4
:109db0007009890020002000d5fe07008009890075
:109dc00015003700510020000000eb004aff07009b
:109dd00080007800400981000080500060098900ff
:109de000510020001000200043ff07008000780091
:109df0005009810000805000700989005100200046
:109e0000200020003cff070080007800100d81003a
:109e100000805000800989000080fa0000000600e0
:109e20000000fa00889fbe008a9fbe00d6ff070090
:109e3000600981006103b900600981006102b90015
:109e40008600780004007800000db80005b0b90065
:109e50000b0178000001410007a0b900000141009a
:109e600082057800700981006104b90070098100e1
:109e70006103b9008800780006007800000ab80085
:109e800007c0b900050178000001410009b0b90020
:109e900000014100820278000a0542008b854a00d9
:109ea000800981006104b900800981006103b90063
:109eb0008800780006007800000ab80007c0b900e2
:109ec000050178000001410009b0b900000141001e
:109ed000820278000a0042008b804a007c05020062
:109ee00000000000e4060200000000009009890064
:109ef000a1098900600981006103b900600981003e
:109f00006102b9008600780004007800000db800f6
:109f100005b0b9000b0178000001410007a0b900ad
:109f20000001410082057800700981006104b900d8
:109f3000700981006103b90088007800060078008c
:109f4000000ab80007c0b90005017800000141000f
:109f500009b0b90000014100820278000a00420005
:109f60008b804a007c05020000000000e40602002d
:109f7000000000000004be0080098100cf80de00e8
:109f80007c050200000000000801be00560302002c
:109f900000000000c209230053262c007c060200aa
:109fa0000000000002002000432b24009c0202005d
:109fb00000000000d0098900e1098900d009810072
:109fc000e109810002002000030a2400fc040200d1
:109fd000000000000000e00009003500d009810009
:109fe000e109810002002000033224000005020084
:109ff000000000000000e00001003c000400370009
:10a000006000b800b0098900c10989001600370056
:10a0100070098100cf80de007c0502000000000096
:10a020000004be0060098100cf80de007c050200d4
:10a03000000000000801be005603020000000000fe
:10a04000c2092300532624007c0602000000000001
:10a0500002002000433324009c02020000000000a4
:10a06000b0098900c10989004f05be004f04be0038
:10a070000080fa00000006000000fa00011a220029
:10a0800010c0b30080487800210320000000eb00de
:10a0900099fe0700400989002103200010002000dc
:10a0a00095fe0700500989007c8a0200000000002c
:10a0b0000004e000070032002103200020002000ff
:10a0c0008dfe070001002c0001004000100d8900ea
:10a0d00006003700210320002000200086fe070034
:10a0e00001d02f0001004000100d8900011a22004c
:10a0f0000040eb00804878000080fa000000060075
:10a100000c00fa00881f78000004780044ff070064
:10a1100090098100a1098100008fbe00b009810073
:10a12000c10981002007980031079800d0098100fb
:10a13000e109810040079800510798008e007800df
:10a14000080078001101be000288be0064004000d3
:10a15000e48040001101be000288be00640040009f
:10a16000e48040001101be000288be0008007800b3
:10a170004f0478000080fa00000006000000fa009a
:10a1800027ff0700d0098100e10981000080fa0063
:10a19000000006000000fa0021ff0700b00981005e
:10a1a000c10981000080fa00000006000000fa00ea
:10a1b0001bff070090098100a10981000080fa00bf
:10a1c000000006000600fa00881f780000047800ee
:10a1d000edfe070060098100000f78007009810022
:10a1e0001007980080098100200798001e00be001b
:10a1f000008cbe00ae00900021049800080078009a
:10a200004f0478000080fa00000006000000fa0009
:10a21000ddfe0700600981000080fa0000000600f2
:10a220000000fa00d8fe0700700981000080fa00e3
:10a23000000006000000fa00d3fe0700800981003c
:10a240000080fa00000006001600fa006000b80066
:10a25000008fbe00cfff0700008fbe0030098100d5
:10a26000cf80de007c050200000000001e01be0061
:10a270009a02020000000000040502000000000035
:10a28000200f98002e0890000000e00003003d0021
:10a29000ae0890008100ea00210f98002e0990007e
:10a2a0006110b9007c0502000000000002002000df
:10a2b000030a240000050200000000000000e00086
:10a2c00001003c0061013700c5e2a900c5c2bf0022
:10a2d0000080fb004700de00614060004601dd00b9
:10a2e000512c200091407800f0cbb30000c06000fa
:10a2f00002407000c5e2b700c5c2bf000080fb008d
:10a300004600de0061406000614060004501dd0004
:10a31000512c200091407800f0cdb30000c06000c7
:10a3200002407000c5e2b700c5c2bf000080fb005c
:10a330004500de0061406000614060004201dd00d8
:10a34000512c200091407800b0cfb30000c06000d5
:10a3500002407000c5e2b700c5c2bf000080fb002c
:10a360004200de0061406000614060004401dd00a9
:10a37000512c200091407800f0ceb30000c0600066
:10a3800002407000c5e2b700c5c2bf000080fb00fc
:10a390004400de0061406000614060000041400018
:10a3a000512c200091407800d0cfb30000c0600055
:10a3b00002407000c5e2b700c5c2bf000080fb00cc
:10a3c0000000d10061406000c700dd00c4c2bf00d2
:10a3d0000074a10001407000c4e2b700c4c2bf0015
:10a3e0000080fb004700de00614060004601dd00a8
:10a3f000412c200091407800f0cbb30000c06000f9
:10a4000002407000c4e2b7000040eb002057980003
:10a4100002002c00833a24001e00be00000502004a
:10a42000000000000000e00001003c0002003700d6
:10a4300011c0b300215798000041eb00125798005b
:10a4400002002000431b24001e00be00fc0402008a
:10a45000000000000000e0000100340002003700ae
:10a4600010c0b30010579800ae5090001e519000dd
:10a4700002c070000004a2000004e00012003a00d4
:10a480000040eb00005798000200280063422400bf
:10a490001e00be00d2050200000000000000e00027
:10a4a00001003a000200370011c0b30001579800c4
:10a4b0000e5090000004a2000004e00002003a00e8
:10a4c000c4c2a800dd0037000041eb00724f9800c5
:10a4d00002002000431b24001e00be0000050200f5
:10a4e000000000000000e00001003c000200370016
:10a4f00010c0b300704f98007e4890000004a20086
:10a500000004e00012003a008040eb00614f980028
:10a5100002002000732824001e00be00fc0402007c
:10a52000000000000000e0000100340002003700dd
:10a5300012c0b300624f98006e4890000004a20061
:10a540000004e00002003a00c5e2a800bb003700aa
:10a550000040eb00504f98000200200073282400b8
:10a560001e00be0000050200000000000000e00028
:10a5700001003c000200370011c0b300514f9800a9
:10a580005e4890000004a2000004e00012003a00bf
:10a590000041eb00424f980002002000132e2400df
:10a5a0001e00be00fc040200000000000000e000ed
:10a5b000010034000200370010c0b300404f980083
:10a5c0004e4890000004a2000004e00002003a009f
:10a5d000c5c2a800990037008040eb00314f9800b9
:10a5e00002002000132e24001e00be000005020001
:10a5f000000000000000e00001003c000200370005
:10a6000012c0b300324f98003e4890000004a200f0
:10a610000004e00012003a000040eb00204f9800d8
:10a6200002002800d33124001e00be00fc040200fa
:10a63000000000000000e0000100340002003700cc
:10a6400011c0b300214f98002e4890000004a200d2
:10a650000004e00002003a00c5a2a800770037001d
:10a660000041eb00124f980002002800d331240073
:10a670001e00be0000050200000000000000e00017
:10a6800001003c000200370010c0b300104f9800da
:10a690001e4890000004a2000004e00012003a00ee
:10a6a0008040eb00014f980002002800a3342400f2
:10a6b0001e00be00fc040200000000000000e000dc
:10a6c000010034000200370012c0b300024f9800ae
:10a6d0000e4890000004a2000004e00002003a00ce
:10a6e000c542a800550037000040eb0070479800b5
:10a6f00002002800a33424001e00be000005020052
:10a70000000000000000e00001003c0002003700f3
:10a7100011c0b300714798007e4090000004a20071
:10a720000004e00012003a000041eb00624798008c
:10a7300002002800733724001e00be00fc04020043
:10a74000000000000000e0000100340002003700bb
:10a7500010c0b300604798006e4090000004a20053
:10a760000004e00002003a00c582a8003300370070
:10a770008040eb0051479800020028007337240006
:10a780001e00be0000050200000000000000e00006
:10a7900001003c000200370012c0b300524798008d
:10a7a0005e4090000004a2000004e00012003a00a5
:10a7b0000040eb00404798000200240023392400a9
:10a7c0001e00be00fc040200000000000000e000cb
:10a7d000010034000200370011c0b3004147980067
:10a7e0004e4090000004a2000004e00002003a0085
:10a7f000c522a800110037000200240023392400dc
:10a800001e00be0000050200000000000000e00085
:10a8100001003c000900370002002c00833a2400ac
:10a820001e00be00fc040200000000000000e0006a
:10a830000100340001003700c4e2a8001e00be0081
:10a840000405020000000000300989000080fa00c1
:10a85000000006000200fa00004f78009687020010
:10a860000000000060dc880010c0b3009e4f1000a4
:10a8700004003a00c17d210010c0b3008048780078
:10a8800003003700c17d21000040eb0080487800c4
:10a890000000eb00001588000000eb001015880098
:10a8a0000000eb00201588000000eb003015880048
:10a8b00060dc8000ea0f500003003a00a802a90003
:10a8c000a822a90002003700a802a800a822a80018
:10a8d000a842a900a862a900a882a900a8a2a9006c
:10a8e000a8c2a900a8e2a900a902a900a922a9005a
:10a8f000a942a900a962a900a982a900a9a2a90048
:10a90000a9c2a900a9e2a900aa02a900aa22a90035
:10a91000aa42a800aa62a800aa82a800aaa2a90026
:10a92000aac2a900aae2a900ab02a900ab22a90011
:10a93000ab42a900ab62a900ab82a900aba2a900ff
:10a94000abc2a900abe2a900112a20009140780017
:10a95000c0cfb30000c06000a1e2b700a042a800d1
:10a96000012a20009140780000ceb30000c07000a2
:10a97000a0e2b700212a20009140780030ccb3003b
:10a9800000c060000034a000a2e2b700a342a8000b
:10a99000512a20009140780000ceb30000c0600032
:10a9a0000004a000a5e2b700c07d2100104078009f
:10a9b0000004e00007003200412a200091407800a6
:10a9c00000ccb30000c060003041b300a4e2b70087
:10a9d00007003700412a20009140780000ccb300e6
:10a9e00000c0600071c2b30001407000a4e2b70073
:10a9f0008560a9008d60a800a1e2a800c07d2100ab
:10aa0000104078000004e00005003a00000000005b
:10aa1000d10b810000032000808f5000fbff360027
:10aa20007c8a0200000000000004e0000200320006
:10aa30000000eb00100d89000080fa000000060005
:10aa4000809fbe00821f78003400f80000002000c4
:10aa5000a00188001000fa00a17d21000040eb0059
:10aa600080487800b17d21000040eb0080487800ec
:10aa70008560a900c017220090407800f0c3b300a1
:10aa800080cf500005003e00c01722001040780023
:10aa90008040e800c017220001487800f00b8100d8
:10aaa000e10f400003003200f00b81000000e800dd
:10aab000f00b8900c07d2100104078000004e00008
:10aac0002e00320000282000000f7800c10b81000a
:10aad0001e0078001000780000017800818040009e
:10aae000007e210000804000020878001e8fe800f0
:10aaf000c10b81001e007800100078000001780072
:10ab000001804000810c200080804000007e2100f8
:10ab100000804000020878001e8fe800c10b810011
:10ab20001e007800100078000001780001804000cd
:10ab30000119200080804000007e2100008040003c
:10ab4000020878001e8fe800c00b81000000e800ba
:10ab5000c00b8900c10b810030062000808f50009f
:10ab6000400236000000eb00c00b8900b17d2100df
:10ab700010c0b300804878003a023700c0012000be
:10ab800050158800212a20009140780030ccb30075
:10ab900000c060000034a000a2e2b700412a2000fb
:10aba0009140780000ccb30000c0600071c2b300d7
:10abb00001407000a4e2b700e07d210090407800e1
:10abc000d0c3b30080cf50000f003a00c00f200068
:10abd00050158800212a20009140780030ccb30025
:10abe00000c060004041b300a2e2b700412a20004b
:10abf0009140780000ccb30000c060003041b30049
:10ac0000a4e2b700f2003700e07d21009040780018
:10ac1000e0c3b30080cf500075003a0060dc8000d4
:10ac2000ea0f500045003a00d07d21001040780026
:10ac3000e34f50000d003e00212a20009140780093
:10ac400030ccb30000c060000044a000a2e2b70016
:10ac5000412a20009140780000ccb30000c0600081
:10ac60007041b300a4e2b7000d003700212a200094
:10ac70009140780030ccb30000c060000034a000e8
:10ac8000a2e2b700412a20009140780000ccb30036
:10ac900000c0600071c2b30001407000a4e2b700c0
:10aca000d07d2100104078000080fb0070079800e4
:10acb0007e009000e20f500017003200fe0090006e
:10acc000e28f500007003c007e0090000000e00092
:10acd0000b003200fe009000e18f50000b003200ac
:10ace000bb0037007e009000e30f50000d003200e3
:10acf000fe009000e48f50000d003200b4003700d9
:10ad0000c011210050158800b1003700c021220079
:10ad100050158800ae003700c0412400501588004f
:10ad2000ab003700c081280050158800a80037000c
:10ad30003000200050158800a5003700212a20008f
:10ad40009140780030ccb30000c060000044a00007
:10ad5000a2e2b700412a20009140780000ccb30065
:10ad600000c060007041b300a4e2b700d07d2100b4
:10ad7000104078000080fb00600798006e00900093
:10ad8000e10f500011003200ee009000e18f500002
:10ad900004003c006e0090000000e000080032005b
:10ada0008b003700ee009000e28f50000a00320066
:10adb0006e009000e30f50000a003200840037005c
:10adc000c01121005015880081003700c0212200e9
:10add000501588007e003700c041240050158800bf
:10ade0007b003700c08128005015880078003700ac
:10adf000e07d210010407800e24f500074003a00de
:10ae000060dc8000ea0f500045003a00d07d210050
:10ae100010407800e34f50000d003e00212a200032
:10ae20009140780030ccb30000c060000044a00026
:10ae3000a2e2b700412a20009140780000ccb30084
:10ae400000c060007041b300a4e2b7000d003700fd
:10ae5000212a20009140780030ccb30000c060006f
:10ae60000034a000a2e2b700412a200091407800ff
:10ae700000ccb30000c0600071c2b300014070009c
:10ae8000a4e2b700d07d2100104078000080fb00d4
:10ae900050079800de009000e28f5000170032004b
:10aea0005e009000e20f500007003c00de009000c2
:10aeb0000100e0000b0032005e009000e10f500046
:10aec0000b00320042003700de009000e38f50009c
:10aed0000d0032005e009000e40f50000d003200c3
:10aee0003b003700c01121005015880038003700a2
:10aef000c02122005015880035003700c0412400d1
:10af00005015880032003700c08128005015880095
:10af10002f00370030002000501588002c0037002b
:10af2000212a20009140780030ccb30000c060009e
:10af30000044a000a2e2b700412a2000914078001e
:10af400000ccb30000c060007041b300a4e2b700c1
:10af5000d07d2100104078000080fb004007980061
:10af6000ce009000e18f5000110032004e009000a2
:10af7000e10f500004003c00ce0090000100e00012
:10af800008003200120037004e009000e20f50001f
:10af90000a003200ce009000e38f50000a00320019
:10afa0000b003700c0112100501588000800370041
:10afb000c02122005015880005003700c041240040
:10afc0005015880002003700c08128005015880005
:10afd00000282000000f7800d07d2100104078006c
:10afe000e34f5000e6003e00c10b81001e007800d8
:10aff000100078000001780081804000007e210070
:10b0000000804000020878001e8fe800c10b81001c
:10b010001e007800100078000001780001804000d8
:10b02000810c200080804000007e210000804000d4
:10b03000020878001e8fe800c10b81001e00780016
:10b040001000780000017800018040000119200004
:10b0500080804000007e21000080400002087800cf
:10b060001e8fe800c00b81000000e800c00b8900c3
:10b07000c10b810030062000808f50000500360093
:10b080000000eb00c00b8900b17d210010c0b300af
:10b0900080487800e07d210090407800e0c3b30054
:10b0a00080cf500028003a00d00b81000000e8005b
:10b0b000d00b8900d10b810010032000808f50003d
:10b0c000020036000000eb00d00b8900d10b81009c
:10b0d0001e00780010007800000178008180400098
:10b0e00080a3210000804000020878001e8fe80045
:10b0f000d10b81001e00780010007800000178005c
:10b1000001804000410620008080400080a3210093
:10b1100000804000020878001e8fe800d10b8100fb
:10b120001e007800100078000001780001804000c7
:10b13000810c20008080400080a32100008040001e
:10b1400002087800b2003700e07d210090407800ce
:10b15000f0c3b30080cf500039003a00d07d210009
:10b16000104078000080fb00300798003e009000ff
:10b17000e10f500017003200be009000e18f500038
:10b1800004003c003e0090000000e0000800320097
:10b190009f003700be009000e28f50001600320082
:10b1a0003e009000e30f50001c0032009800370072
:10b1b0001e0078001000780020db88001e8fe80059
:10b1c0001e0078001000780060db8800e2e2a80032
:10b1d0008f0037001e0078001000780030db8800f8
:10b1e0001e8fe8001e0078001000780070db8800d9
:10b1f000e302a800860037001e00780010007800e7
:10b2000040db88001e8fe8001e00780010007800e8
:10b2100080db8800e802a8007d0037001e0078006f
:10b220001000780050db88001e8fe8001e007800b8
:10b230001000780090db8800e822a8007400370036
:10b24000e07d210010407800e34f500070003a008c
:10b25000d07d2100104078000080fb00200798007e
:10b26000ae009000e18f50001a0032002e009000d6
:10b27000e10f500004003c00ae0090000100e0002f
:10b2800008003200620037002e009000e20f5000ec
:10b290001c003200ae009000e38f50002500320009
:10b2a0005b0037001e00780010007800c0db8800cb
:10b2b0001e8fe8001e0078001000780000dc880077
:10b2c000e2e2a900d17d210010c0b30080487800df
:10b2d0004f0037001e00780010007800d0db880097
:10b2e0001e8fe8001e0078001000780010dc880037
:10b2f000e302a900d17d210020c0b300804878007e
:10b30000430037001e00780010007800e0db880062
:10b310001e8fe8001e0078001000780020dc8800f6
:10b32000e802a900d17d210030c0b3008048780038
:10b33000370037001e00780010007800f0db88002e
:10b340001e8fe8001e0078001000780030dc8800b6
:10b35000e822a90060dc8000ea0f500004003a00f7
:10b36000d17d210040c0b30080487800280037001c
:10b37000d17d21000040eb00804878002400370098
:10b380001e007800100078001e8fe800e07d21008c
:10b3900090407800f0c3b30080cf50000b003a001b
:10b3a0001e00780010007800b0db88001e8fe800d7
:10b3b0001e00780010007800a0db88001e8fe800d7
:10b3c000d042a800d022a80011003700e07d210063
:10b3d00010407800e34f50000d003a001e00780046
:10b3e0001000780050dc88001e8fe8001e007800f6
:10b3f0001000780040dc88001e8fe800d042a900d1
:10b40000d022a900d17d21000040eb0080487800c7
:10b41000e07d210010407800304798000040eb00ac
:10b4200020479800f0c3b300be40900080cf50008a
:10b430000200360010c0b300204798003e40900044
:10b440008040e800e07d210001487800ae40900097
:10b450000104e00003003200e17d21000040eb0028
:10b4600080487800a17d210010c0b300804878009a
:10b470000080fa003400f9004f0178004f00be0050
:10b48000004006000000fa00a07d21001040780076
:10b490000080fb000080fa00000006000000fa00b7
:10b4a000b07d2100104078000080fb000080fa0091
:10b4b000000006000000fa00a1e2a8000080fa00e7
:10b4c000000006000000fa00a1e2a9000080fa00d6
:04b4d0000000060072
:020000040000fa
:10b4d400a821000002000000000000008e1b0000f4
:10b4e4000802000000000000a02100000400000089
:10b4f400020000000000d000070000002621000028
:10b504001e00000000000000782100000800000078
:10b514000200000000000000000000000000000025
:10b52400da170000b403000000000000442100000a
:10b534001400000000000000aa2100000200000026
:10b544000000000028200000d800000002000000d5
:10b554000403050053060300075308000009d10043
:10b564000a000b00070c03000d510e00010fe70049
:10b574001202130002151000164017004018400074
:10b5840019401a00031be6001c001d00701e0a006f
:10b594001f1b2000443b0000468048006049960081
:10b5a4004a004b007d4c00004e084f000a507000ca
:10b5b40059005a00005b00005cac5d00027600009c
:10b5c400771a78002a7937007a427b00567c680023
:10b5d4007d877e00a37fbc0080d48100ea8e380082
:10b5e4008fa590000d919300922d930006948300f3
:10b5f40095aa96004d97250098259b00009c9600df
:10b604009f80a00080a1b600a29da300aba48000ef
:10b61400a500a60007a70100a8e7a90000aa010049
:10b62400ad9fae0022af8c00b007b100ccb20000d9
:10b63400b370b90003bae600bb07bc00ccbd000080
:10b64400be0cc10010c2e000c310c400e0c58000fd
:10b65400c680c70001c8a500c902ca007acb000091
:10b66400cca7cd0001ce4700d43cd50001d8800042
:10b67400961d000050010000000000000a0c0000ac
:10b684000400000000000000802100000800000009
:10b6940000000000ac2100000200000002000000d5
:10b6a40000000000ae2100000200000000000000c5
:10b6b400b0210000020000000200000001000000b0
:10b6c400882100000600000000000000582100004e
:10b6d4001000000000000000040c00000600000040
:10b6e400020000000000000000000000000800004c
:10b6f400040400000200000000000000000000003c
:10b704000000000000000000000000000000000035
:10b714000000000000000000000000000000000025
:10b724000000000000000000000000000000000015
:10b734000000000000000000000000000000000005
:10bc5400000000008e210000060000000200000029
:10bc64000000000000000000a42100000400000007
:10bc7400020000000200ff00ff0000009421000009
:10bc84000600000000000000e61e00004201000063
:10bc940002000000652d700075636b003000e60043
:10bca4001e010000de94010000e194002000e80081
:10bcb40094010000ed94010000f8940001000300d9
:10bcc400950a00000f95080000149500080019005b
:10bcd4009503000021950100002595003c002e00ed
:10bce400953c000036953c00004095000100490059
:10bcf4009501000054950300006095000100640064
:10bd04009501000068950100006c95000100790020
:10bd14009503000081950000000000000100000070
:10bd240004160c008301d400142000001614000033
:10bd340000000000000000000000000000000000ff
:10bd440000000000000000000000000000000000ef
:10bd540000000000000000000000000000000000df
:10bd640000000000f2950400960300002a960000eb
:10bd7400000000002f963e00960100007e96010010
:10bd8400008296000000000000859600969601004f
:10bd940000ae96000000000000b79600c8960100af
:10bda40000e296000100eb0096010000f696000008
:10bdb40000000000ce8d0e008e708e00c68e1a001c
:10bdc4008f6c8f00ba8f180090769000da90400044
:10bdd400918a9100fc91340092889200de922600b0
:10bde400936a9300a493ee0093d29400821f8e0072
:10bdf4001f9e1f00aa1f000000901a00fc1a420098
:10be04001ba61b000c1c72001cd81c007a1d000011
:10be14001e861e00341fe0001fd220005621780029
:10be240021502200c6222000237a23007424940087
:10be3400261e3d009e3dd4003d043e00ff0032001e
:10be440000000000100c0000ca0b000000000000fd
:10be54000e0c00000200000000000000b2210000ef
:10be64000200000000000000002100002600000085
:10be74000200000002219c00210000009c21090016
:10be84000000000002009a00210000009a21060030
:10be94000201000000000000000000000000060095
:10bea40002020000000000009a21000006000000c9
:10beb40000000000682100001000000000000000e5
:10bec400b42100000200000000000000b6210000c0
:10bed4000200000000000000b82100000200000081
:10bee4000200000001000000ba210000020000006e
:08bef400000000000000000046
:020000040000fa
:10befc000200fa00004f78009c8a0200000000004b
:10bf0c001e41780031c0b300c0cdb3000a8b0200d3
:10bf1c0000000000a68a0200000000000080fa0069
:10bf2c00000006000400fa00004f7800114798004a
:10bf3c00224798001e407800edff07009c8a020003
:10bf4c00000000002e4190009e409000c0cdb30038
:10bf5c000a8b020000000000a68a0200000000000c
:10bf6c000080fa00000006000400fa002047980048
:10bf7c00314798002e409000ddff07009c8a02009c
:10bf8c0000000000be409000c0cdb300b08a02009b
:10bf9c0000000000004f7800a68a0200000000009c
:10bfac001e80fb000080fa00000006000400fa006e
:10bfbc00204798002e409000cdff07009c8a02007d
:10bfcc000000000031c0b300c0cdb300b08a020045
:10bfdc0000000000004f7800a68a0200000000005c
:10bfec001e80fb000080fa00000006000200fa0030
:10bffc000040eb00beff07009c8a0200000000001e
:10c00c00b1c5b300c0cdb300b08a0200000000007f
:10c01c00004f78001e40780010479800a68a020056
:10c02c0000000000f1c7b3001e409000014060000a
:10c03c00104798009e409000f0cbb30000c0600009
:10c04c00104798009e40900070cfb30000c0600075
:10c05c00104798009c8a0200000000001e419000ce
:10c06c00b1c5b300c0cdb3000a8b020000000000c4
:10c07c00a68a0200000000001e80fb000080fa006f
:10c08c00000006000200fa000040eb00004f7800b0
:10c09c00d6ff0700004f780080c2b3009b01070059
:10c0ac001e80fb000080fa00000006000200fa006f
:10c0bc00004f78001e417800a1c6b3000040eb0091
:10c0cc0098ff07000080fa00000006000200fa004a
:10c0dc00004f78001e41780071cbb30010c0b30044
:10c0ec0090ff07000080fa00000006000600fa002e
:10c0fc00004f78001e80fb002007980000042000f1
:10c10c00ae009000808f5000160032000008200016
:10c11c00ae009000808f50001f0032000002200003
:10c12c00ae009000808f50000100320027003700d5
:10c13c0010c0b300e5ff07001e41780031c9b30001
:10c14c0010c0b30077ff07001e41780041c9b3004f
:10c15c0010c0b30073ff07000000eb00100798003d
:10c16c001c00370030c0b300d8ff07001e41780018
:10c17c0031c9b30010c0b3006aff07001e4178003c
:10c18c0041c9b30010c0b30066ff07008000eb008c
:10c19c00110798000f00370070c0b300cbff0700e9
:10c1ac001e41780031c9b30010c0b3005dff070019
:10c1bc001e41780041c9b30010c0b30059ff0700fd
:10c1cc000000eb0010079800020037008080eb00a5
:10c1dc00110798001e0090000080fa000000060075
:10c1ec000600fa00004f78001e80fb002007980024
:10c1fc0000042000ae009000808f5000160032002a
:10c20c0000082000ae009000808f50001f0032000c
:10c21c0000022000ae009000808f50000100320020
:10c22c00270037000040eb00a8ff07001e417800f4
:10c23c0031c9b30010c0b3003aff07001e417800ab
:10c24c0041c9b30010c0b30036ff07000000eb007b
:10c25c00100798001c00370010c0b3009bff0700ac
:10c26c001e41780031c9b30010c0b3002dff070088
:10c27c001e41780041c9b30010c0b30029ff07006c
:10c28c008000eb00110798000f00370030c0b3009e
:10c29c008eff07001e41780031c9b30010c0b300f7
:10c2ac0020ff07001e41780041c9b30010c0b30045
:10c2bc001cff07000000eb0010079800020037007d
:10c2cc008080eb00110798001e0090000080fa009f
:10c2dc00000006000600fa00004f78001147980095
:10c2ec001e80fb00200798002e009000e10f5000ec
:10c2fc000f0032002e009000e20f500014003200ac
:10c30c002e0090000000e000010032001800370001
:10c31c0032c4b300e1c4b30010c0b30001ff070086
:10c32c001e40900071ff07001007980012003700a4
:10c33c0002c3b300e1c4b30010c0b300f9fe0700a0
:10c34c001e409000a6ff0700100798000a00370057
:10c35c0022c0b300e1c4b30010c0b300f1fe07006b
:10c36c001e4090009eff0700100798000200370047
:10c37c000080eb00100798001e0090000080fa006f
:10c38c00000006000a00fa00200798003107980008
:10c39c00ae0090003e009000808f500003003900ea
:10c3ac000080eb00400798001e003700be00900094
:10c3bc0070302000808f5000030036000080eb00ae
:10c3cc0040079800170037002e0090000000e9008d
:10c3dc00200798002e009000204798002e00900017
:10c3ec004800de00304798003e009000004f780077
:10c3fc003e0090004800de00104798002e4190004f
:10c40c0091c0b3000040eb00c6fe07003e41900017
:10c41c0081c0b3000040eb00c2fe07000000eb003f
:10c42c00400798004e0090000080fa0000000600c3
:10c43c000800fa0020079800310798000000eb0074
:10c44c000080fa00000006000a00fa00200798009d
:10c45c0031079800ae0090003e009000808f500095
:10c46c00030039000080eb004007980023003700e0
:10c47c00be00900030202000808f5000030036005a
:10c48c000080eb00400798001c0037002e00900045
:10c49c00204798002e0090004800de00304798009e
:10c4ac003e009000004f78003e0090004800de00f7
:10c4bc00104798003e41900001c1b3000040eb00d2
:10c4cc0098fe07002e41900011c1b3000040eb0014
:10c4dc0094fe07001e41900021c1b3000040eb0008
:10c4ec0090fe07001e41780031c1b3000040eb0004
:10c4fc008cfe07000000eb00400798004e009000f7
:10c50c000080fa00000006000200fa00000f78001c
:10c51c001e00e00008003a0002c8b30041c0b3009e
:10c52c0010c0b3007ffe070022c0b30061c0b3008f
:10c53c0010c0b3007bfe07000080fa00000006006c
:10c54c000600fa001007980021079800c1c6b30036
:10c55c000040eb0084fe0700004f78001e009000a6
:10c56c000000e0000300320000c8b3001e4f700052
:10c57c0002003700f0c7b3001e4f60002e00900081
:10c58c000000e0000300320000c4b3001e4f700036
:10c59c0002003700f0cbb3001e4f60001e41780044
:10c5ac00c1c6b3000040eb005efe07000080fa003d
:10c5bc00000006000600fa001007980021079800fa
:10c5cc0080c9b300004f78001e0090000000e0000e
:10c5dc0001003a001e24a0002e0090000000e00094
:10c5ec000a003a001e04a0000041eb0081c4b30015
:10c5fc0020c0b3004bfe07000041eb0091c4b30018
:10c60c0020c0b30047fe07000800370082c0b3000b
:10c61c0081c4b30020c0b30042fe0700c2c0b30007
:10c62c0091c4b30020c0b3003efe07001e41780049
:10c63c0041c0b30020c0b3003afe07000080fa00ee
:10c64c00000006000400fa00004f78001147980023
:10c65c00224798001e41780031c2b3000040eb0025
:10c66c0030fe07001e41900041c2b3000040eb00b9
:10c67c002cfe07002e41900051c2b3000040eb008d
:10c68c0028fe07000080fa00000006000400fa00f3
:10c69c00008fbe001e00be004808de000100200016
:10c6ac000041780021c1b30020c0b3001dfe07007b
:10c6bc001e00be004008de00010020000041780092
:10c6cc0031c1b30020c0b30016fe07001e00be002f
:10c6dc004809dd004800de0000007100c808de00db
:10c6ec000041780041c1b30020c0b3000dfe07002b
:10c6fc001e0078000041780051c1b30020c0b30087
:10c70c0008fe07000080fa00000006000200fa0094
:10c71c00004f78001e417800e1c9b30010c0b3008f
:10c72c0000fe07000080fa00000006000200fa007c
:10c73c00004f78009c8a0200000000001e41780027
:10c74c0031c0b300c0cdb3000a8b02000000000062
:10c75c00a68a0200000000000080fa00000006001b
:10c76c000400fa00004f7800114798002247980007
:10c77c001e407800edff07009c8a020000000000bc
:10c78c002e4190009e409000c0cdb3000a8b020059
:10c79c0000000000a68a0200000000000080fa00e1
:10c7ac00000006000400fa0020479800314798006a
:10c7bc002e409000ddff07009c8a02000000000064
:10c7cc00be409000c0cdb300b08a02000000000053
:10c7dc00004f7800a68a0200000000001e80fb00bb
:10c7ec000080fa00000006000200fa00004f7800fa
:10c7fc001e41780011c9b3000040eb00d8ff0700c0
:10c80c000080fa00000006000200fa00004f7800d9
:10c81c001e41780081c6b30010c0b300d0ff0700e2
:10c82c000080fa00000006000600fa00004f7800b5
:10c83c001e80fb002007980000042000ae00900032
:10c84c00808f50001a00320000082000ae009000cb
:10c85c00808f50002700320000022000ae009000b4
:10c86c00808f5000010032003300370010c0b3003d
:10c87c00e5ff07001e41780001c8b30010c0b300eb
:10c88c00b7ff07001e41780011c8b30010c0b300f9
:10c89c00b3ff070012c0b30021c8b30010c0b3002f
:10c8ac00afff07000000eb001007980024003700d2
:10c8bc0030c0b300d4ff07001e41780001c8b3009c
:10c8cc0010c0b300a6ff07001e41780011c8b300ca
:10c8dc0010c0b300a2ff070012c0b30021c8b30000
:10c8ec0010c0b3009eff07008000eb0011079800fa
:10c8fc001300370070c0b300c3ff07001e4178005f
:10c90c0001c8b30010c0b30095ff07001e417800aa
:10c91c0011c8b30010c0b30091ff070012c0b300e0
:10c92c0021c8b30010c0b3008dff07000000eb005e
:10c93c0010079800020037008080eb001107980068
:10c94c001e0090000080fa00000006000600fa00ad
:10c95c00004f78001e80fb00200798000004200088
:10c96c00ae009000808f50001a00320000082000aa
:10c97c00ae009000808f5000270032000002200093
:10c98c00ae009000808f5000010032003300370061
:10c99c000040eb009cff07001e41780001c8b3006b
:10c9ac0010c0b3006eff07001e41780011c8b30021
:10c9bc0010c0b3006aff070012c0b30021c8b30057
:10c9cc0010c0b30066ff07000000eb0010079800d2
:10c9dc002400370010c0b3008bff07001e41780005
:10c9ec0001c8b30010c0b3005dff07001e41780002
:10c9fc0011c8b30010c0b30059ff070012c0b30038
:10ca0c0021c8b30010c0b30055ff07008000eb0035
:10ca1c00110798001300370030c0b3007aff0700ed
:10ca2c001e41780001c8b30010c0b3004cff0700d2
:10ca3c001e41780011c8b30010c0b30048ff0700b6
:10ca4c0012c0b30021c8b30010c0b30044ff0700ec
:10ca5c000000eb0010079800020037008080eb000c
:10ca6c00110798001e0090000080fa0000000600dc
:10ca7c000600fa00004f7800114798001e80fb005a
:10ca8c00200798002e009000e10f50000f0032009c
:10ca9c002e009000e20f5000140032002e00900087
:10caac000000e0000100320018003700d2c0b300d3
:10cabc0081c3b30010c0b30029ff07001e409000d3
:10cacc0059ff0700100798001200370082c0b3000e
:10cadc0081c3b30010c0b30021ff07001e409000bb
:10caec009aff0700100798000a00370022c0b30015
:10cafc0081c3b30010c0b30019ff07001e409000a3
:10cb0c0092ff070010079800020037000080eb002e
:10cb1c00100798001e0090000080fa00000006002c
:10cb2c000a00fa002007980031079800ae00900028
:10cb3c003e009000808f5000030039000080eb0015
:10cb4c00400798001e003700be009000f031200016
:10cb5c00808f5000030036000080eb0040079800e7
:10cb6c00170037002e0090000000e9002007980005
:10cb7c002e009000204798002e0090004800de0008
:10cb8c00304798003e009000004f78003e00900027
:10cb9c004800de00104798002e41900011c5b300ec
:10cbac0010c0b300eefe07003e41900001c5b3007b
:10cbbc0010c0b300eafe07000000eb00400798002d
:10cbcc004e0090000080fa00000006000800fa00f9
:10cbdc0020079800310798000000eb000080fa0055
:10cbec00000006000a00fa002007980031079800a0
:10cbfc00ae0090003e009000808f50000300390082
:10cc0c000080eb004007980023003700be00900026
:10cc1c00301f2000808f5000030036000080eb0096
:10cc2c00400798001c0037002e0090002047980009
:10cc3c002e0090004800de00304798003e00900027
:10cc4c00004f78003e0090004800de00104798002e
:10cc5c003e41900001c6b30010c0b300c0fe0700f7
:10cc6c002e41900011c6b30010c0b300bcfe0700eb
:10cc7c001e41900021c6b30010c0b300b8fe0700df
:10cc8c001e41780031c6b30010c0b300b4fe0700db
:10cc9c000000eb00400798004e0090000080fa0066
:10ccac00000006000200fa00000f780012c0b3006a
:10ccbc00a1c5b30020c0b300a9fe070012c4b30085
:10cccc0021c3b30010c0b300a5fe07001e00e00096
:10ccdc0011003a0000c1eb0081c8b30010c0b300d2
:10ccec009ffe070000c1eb0091c8b30010c0b30059
:10ccfc009bfe070082c0b300a1c8b30010c0b300f4
:10cd0c0097fe070000c1eb00b1c8b30010c0b30020
:10cd1c0093fe07001000370002c2b30081c8b300b5
:10cd2c0010c0b3008efe070002c8b30091c8b30058
:10cd3c0010c0b3008afe070082c0b300a1c8b300c4
:10cd4c0010c0b30086fe070000c1eb00b1c8b300f1
:10cd5c0010c0b30082fe07000080fa00000006003d
:10cd6c000600fa00100798002107980001c9b300cb
:10cd7c000040eb008bfe0700004f78001e00900077
:10cd8c000000e0000300320000c8b3001e4f70002a
:10cd9c0002003700f0c7b3001e4f60002e00900059
:10cdac000000e0000300320000c4b3001e4f70000e
:10cdbc0002003700f0cbb3001e4f60001e4178001c
:10cdcc0001c9b3000040eb0065fe07000080fa00cb
:10cddc00000006000600fa001007980021079800d2
:10cdec0080c9b300004f78001e0090000000e000e6
:10cdfc0001003a001e24a0002e0090000000e0006c
:10ce0c000a003a001e04a0000041eb0051c5b3001b
:10ce1c0020c0b30052fe07000041eb0061c5b30017
:10ce2c0020c0b3004efe07000800370082c0b300dc
:10ce3c0051c5b30020c0b30049fe0700c2c0b30007
:10ce4c0061c5b30020c0b30045fe07001e41780049
:10ce5c0041c0b30020c0b30041fe07000080fa00bf
:10ce6c00000006000400fa00004f780011479800fb
:10ce7c00224798001e41780041cab30020c0b3007d
:10ce8c0037fe07001e41900051cab30020c0b3000a
:10ce9c0033fe07002e41900061cab30020c0b300de
:10ceac002ffe07000080fa00000006000400fa00c4
:10cebc00008fbe001e00be004808de0001002000ee
:10cecc0000417800c1c2b30020c0b30024fe0700ab
:10cedc001e00be004008de0001002000004178006a
:10ceec00d1c2b30020c0b3001dfe07001e00be005f
:10cefc004809dd004800de0000007100c808de00b3
:10cf0c0000417800e1c2b30020c0b30014fe07005a
:10cf1c001e00780000417800f1c2b30020c0b300bd
:10cf2c000ffe07000080fa00000006000400fa0063
:10cf3c00004f780011479800224798009c8a020005
:10cf4c00000000002e4190009e4090001e40780092
:10cf5c000a8b020000000000a68a020000000000fc
:10cf6c000080fa00000006000400fa002047980038
:10cf7c00314798009c8a020000000000be409000df
:10cf8c002e409000b08a020000000000004f780094
:10cf9c00a68a0200000000001e80fb000080fa0040
:10cfac00000006000a00fa0040479800310798007c
:10cfbc00024f9800134f98000040eb002047980058
:10cfcc000000eb00000f78004e00370010c0b300db
:10cfdc00204798002070020000000000804078007c
:10cfec002e40900001406000204798004e40900079
:10cffc006e72020000000000804078002e4090000d
:10d00c00014060002047980001c8b3000e48900012
:10d01c0000c070006e7202000000000080407800ba
:10d02c002e4090000140600020479800687002007c
:10d03c0000000000804078002e409000014060000d
:10d04c00204798004e4090000040e8006e720200ad
:10d05c0000000000804078002e40900001406000ed
:10d06c00204798000000eb00000f78001a003700f2
:10d07c009e0078003e00900000804000be710200cf
:10d08c0000000000804078002e40900001406000bd
:10d09c00204798001e4890000080fb000000e9002b
:10d0ac009e0f500006003a00547102000000000070
:10d0bc00ae40900000c0600020479800050037008b
:10d0cc00ea70020000000000ae40900000c060005a
:10d0dc00204798001e0fe8001e4890000080fb00bf
:10d0ec009e0f5000e2ff3e00b070020000000000f6
:10d0fc002e4090000004e00005003a00bc6f0200d6
:10d10c00000000002e4090000004e000afff320051
:10d11c002e4090000000fb000080fa00000006008a
:10d12c000000fa009c8a020000000000f2c9b30063
:10d13c0001c2b300c0c3b3000a8b020000000000a0
:10d14c0002c5b30051c2b300c0c3b3000a8b0200c6
:10d15c0000000000f2ccb30001c2b30040cdb3001c
:10d16c000a8b02000000000002c2b30011c2b3001f
:10d17c0040cdb3000a8b0200000000000041eb0020
:10d18c0031c2b30040cdb3000a8b02000000000096
:10d19c00a68a0200000000000080fa0000000600d1
:10d1ac000200fa00000f78009c8a020000000000c8
:10d1bc0063c0b30082c2b3009e007800c0c3b3004a
:10d1cc0078ff0700a68a0200000000000080fa0029
:10d1dc00000006000c00fa00300798004107980088
:10d1ec00520798009c8a02000000000063c0b30044
:10d1fc0082c2b3008e007800c0c3b30069ff070081
:10d20c00a68a0200000000001e4090000080fb0077
:10d21c00c800dd001e4078000080fb0080804000cc
:10d22c003e009000010878003e4090000080fb001a
:10d23c00c800dd002e4090000080fb008080400084
:10d24c004e009000010878005e4090000080fb00ca
:10d25c00c800dd004e4090000080fb008080400044
:10d26c005e009000010878000080fa0000000600c3
:10d27c000200fa009c8a0200000000008e00780078
:10d28c0023c0b30082c2b300c0c3b30045ff070084
:10d29c00a68a0200000000001e4090000000fb0067
:10d2ac00c800dd001e4078000000fb00008040003c
:10d2bc000080fa00000006000200fa009c8a0200be
:10d2cc00000000008e00780023c0b300a2c2b3009f
:10d2dc00c0c3b30033ff0700a68a020000000000a1
:10d2ec001e4090000000fb00c800dd001e407800ce
:10d2fc000000fb00008040000080fa0000000600e7
:10d30c000200fa009c8a0200000000008e007800e7
:10d31c0023c0b300c2c2b300c0c3b30021ff0700d7
:10d32c00a68a0200000000001e4090000000fb00d6
:10d33c00c800dd001e4078000000fb0000804000ab
:10d34c000080fa00000006000200fa00000f7800ce
:10d35c009c8a02000000000063c0b30082c2b300cc
:10d36c009e00780040cdb3000eff0700a68a020095
:10d37c00000000000080fa00000006000c00fa001b
:10d38c003007980041079800520798009c8a0200c9
:10d39c000000000063c0b30082c2b3008e007800ae
:10d3ac0040cdb300fffe0700a68a0200000000007b
:10d3bc001e4090000080fb00c800dd001e4078007d
:10d3cc000080fb0080804000700c81008080500049
:10d3dc003e009000010878003e4090000080fb0069
:10d3ec00c800dd002e4090000080fb0080804000d3
:10d3fc00800c8100808050004e0090000108780065
:10d40c005e4090000080fb00c800dd004e409000a4
:10d41c000080fb0080804000900c810080805000d8
:10d42c005e009000010878000080fa000000060001
:10d43c000200fa009c8a0200000000008e007800b6
:10d44c0023c0b30082c2b30040cdb300d5fe0700a9
:10d45c00a68a0200000000001e4090000000fb00a5
:10d46c00c800dd001e4078000000fb0080804000fa
:10d47c00700c8100008050000080fa000000060053
:10d48c000200fa009c8a0200000000008e00780066
:10d49c0023c0b300a2c2b30040cdb300c1fe07004d
:10d4ac00a68a0200000000001e4090000000fb0055
:10d4bc00c800dd001e4078000000fb0080804000aa
:10d4cc00800c8100008050000080fa0000000600f3
:10d4dc000200fa009c8a0200000000008e00780016
:10d4ec0023c0b300c2c2b30040cdb300adfe0700f1
:10d4fc00a68a0200000000001e4090000000fb0005
:10d50c00c800dd001e4078000000fb008080400059
:10d51c00900c8100008050000080fa000000060092
:10d52c000000fa0061c2b30040cdb3008efe0700cc
:10d53c000000fb000080fa00000006001000fa005a
:10d54c0070079800e80047000000eb0080087800a6
:10d55c00e80047000000eb0090009800e80047004e
:10d56c000000eb00a00098000000eb00000f78001a
:10d57c000000eb00000f78002a0037000e80e80056
:10d58c0071ff070068004700100178000e80e8006a
:10d59c00104090000080fb00c800dd000e80e80009
:10d5ac00104078000080fb000080400080004100ab
:10d5bc0068004700010878006800470010019000df
:10d5cc000e80e800304090000080fb00c800dd00b9
:10d5dc000e80e800204090000080fb00008040009e
:10d5ec008000410068004700110098006800470067
:10d5fc00200190000e80e800504090000080fb005d
:10d60c00c800dd000e80e800404090000080fb0068
:10d61c000080400080004100680047002100980015
:10d62c001e0fe8007e0090009e0f1000d3ff350007
:10d63c0068004700100078007e019000110009007e
:10d64c000200d800700c89006800470010009000a0
:10d65c007e019000110009000200d800800c8900a6
:10d66c0068004700200090007e0190001100090026
:10d67c000200d800900c89000080fa00000006001f
:10d68c000200fa00000f78001e007800cf80de0048
:10d69c007c0502000000000092c22500f3c02300ac
:10d6ac007c060200000000000080fa00000006006a
:10d6bc000200fa00000f78001e007800cf80de0018
:10d6cc007c0502000000000072cf2c0023712300a7
:10d6dc007c060200000000000080fa00000006003a
:10d6ec000600fa0010079800210798000000eb00d4
:10d6fc00000f78000a003700a2ec80009e00780032
:10d70c001e0090000080400090407800e0b821009e
:10d71c00017178000200e800a0ec88001e0fe80000
:10d72c002e0090009e0f1000f3ff39000080fa00cd
:10d73c00000006000200fa00004f780011002000e3
:10d74c000e007800e6ff07000080fa0000000600db
:10d75c000400fa00100798001e009000000f7800db
:10d76c000e00780021002000ddff07000080fa0089
:10d77c00000006000400fa00100798001e0090003c
:10d78c00000f78000e00780021002000d4ff070065
:10d79c000080fa00000006000400fa001007980050
:10d7ac001e009000e407020000000000000f78004b
:10d7bc001e007800dfff0700080037001e009000f5
:10d7cc0010407800804078001e0090000000e800b7
:10d7dc001007980001407800d6ff07001e0090004b
:10d7ec00104078000004e000f4ff3a000080fa00da
:10d7fc00000006000a00fa001007980021079800a4
:10d80c0032079800430798000000eb00a0ec88005a
:10d81c002e009000ceff07000000eb00000f7800f8
:10d82c0006003700be0090001e007800008040000b
:10d83c0010407800bfff07001e0fe8004e0090005c
:10d84c009e0f1000f7ff3900a2ec8000e1b8210018
:10d85c001e009000aa3e0200000000000080fa00aa
:10d86c00000006000800fa00100798002107980035
:10d87c00320798000000eb00a0ec88005000290053
:10d88c00b3ff07002e009000b1ff07002e009000a0
:10d89c00000f7800080037001e009000c0009000b8
:10d8ac001e0078000000400000804000100078004e
:10d8bc00a7ff07001e0fe8002e009000be0090008e
:10d8cc00010040009e0f5000f3ff3e00a2ec8000d0
:10d8dc00e1b821001e009000aa3e020000000000ea
:10d8ec000080fa00000006000e00fa0060079800a5
:10d8fc006e0090000a3d02000000000050079800e6
:10d90c005e0090000080e800400798006e009000d8
:10d91c00703e020000000000300798006e0090007e
:10d92c00143d020000000000200798000000eb00ee
:10d93c00100798000000eb00a0ec88000000290004
:10d94c0083ff07005e0090001000780092ff070034
:10d95c00500020007eff07006e0090001000900029
:10d96c007bff07006e0090005000900078ff0700ce
:10d97c006e0090003000900075ff07000000eb0077
:10d98c0010079800030037001e0090000000e8000c
:10d99c00100798001e0090004200dd008000780007
:10d9ac004e00900000804000100078000000e00065
:10d9bc00f5ff3a001e00900065ff07000000eb0029
:10d9cc0010079800030037001e0090000000e800cc
:10d9dc00100798001e0090004200dd0080007800c7
:10d9ec002e00900000804000100078000000e00045
:10d9fc00f5ff3a001e00900055ff07000000eb00f9
:10da0c0010079800030037001e0090000000e8008b
:10da1c00100798001e009000000040008000780065
:10da2c003e00900000804000100078000000e000f4
:10da3c00f5ff3a001e00900045ff0700a2ec8000a5
:10da4c00e1b821006e009000aa3e02000000000028
:10da5c000000eb00100798001a0037000000eb00e4
:10da6c00a0ec88001000290039ff07001e00900070
:10da7c004200dd00800078004e00900000804000e5
:10da8c001000780032ff07001e0090004200dd00fd
:10da9c00800078004e009000008040001000900044
:10daac003dff0700a2ec8000e1b821006e00900061
:10dabc00aa3e0200000000001e0090000000e800da
:10dacc00100798001e0090004200dd0080007800d6
:10dadc004e00900000804000100090000000e0001c
:10daec00deff3a000000eb00100798001a00370028
:10dafc000000eb00a0ec88002000290014ff0700b8
:10db0c001e0090004200dd00800078002e00900086
:10db1c0000804000100078001fff07001e009000de
:10db2c004200dd00800078002e0090000080400054
:10db3c001000900018ff0700a2ec8000e1b8210053
:10db4c006e009000aa3e0200000000001e00900033
:10db5c000000e800100798001e0090004200dd0055
:10db6c00800078002e0090000080400010007800ab
:10db7c000000e000deff3a000000eb001007980008
:10db8c00540037000000eb00a0ec880030002900a6
:10db9c00effe07001e00900000004000800078009f
:10dbac003e009000008040001000780010007800cb
:10dbbc00f9fe07001e009000000040008000780075
:10dbcc003e00900000804000100078001000900093
:10dbdc00f1fe07000000eb00000f78000100370099
:10dbec001e0fe8001e00900000004000800078002e
:10dbfc003e00900000804000900078001e007800ed
:10dc0c004200dd0064004000608078000000e0000d
:10dc1c00f3ff3a001e007800cdfe07000000eb0079
:10dc2c00000f7800170037001e0090000000400025
:10dc3c00800078003e00900000804000900078004a
:10dc4c001e0078004200dd00640040006080780017
:10dc5c00c8fe07001e009000000040008000780005
:10dc6c003e00900000804000900078001e0078007c
:10dc7c004200dd006600400060807800c6fe0700b0
:10dc8c001e0fe8001e00900000004000800078008d
:10dc9c003e00900000804000900078001e0078004c
:10dcac004200dd0064004000608078000000e0006d
:10dcbc00ddff3a00a2ec8000e1b821006e0090007c
:10dccc00aa3e0200000000001e0090000000e800c8
:10dcdc00100798001e0090000000400080007800a3
:10dcec003e00900000804000100078000000e00032
:10dcfc00a4ff3a000080fa00000006001400fa00ad
:10dd0c00100f98001e0890000a3d02000000000051
:10dd1c007007980070004700800178006220200096
:10dd2c00e1b821001e089000583f020000000000de
:10dd3c00600798006e0090000000e0004b0032007d
:10dd4c00e0b82100900078005107980000b921003c
:10dd5c00400798006e0090000080e9000000d100a0
:10dd6c00300798005e0090000000e000390035009c
:10dd7c001e089000700090000000d1000000a2006e
:10dd8c00610060000004e00006003a001e089000ec
:10dd9c00700090000000a200610060000004e00030
:10ddac00320032007e009000b000900021079800f5
:10ddbc007e009000d0009000110798001e08900083
:10ddcc00c00090002e0090000000400080804000b9
:10dddc000e089000800878002e0090000000e800eb
:10ddec00200798000000eb00000f78000e003700b1
:10ddfc001e089000c00090002e0090001e004000f5
:10de0c0000004000008140001e007800000040002f
:10de1c00800078004e0090000080400010007800d8
:10de2c00000978001e0fe8001e0090009e0f1000e5
:10de3c00030031003e0090009e0f1000ecff3900f3
:10de4c00de0090001e0890004e270200000000002b
:10de5c0006003700be0190004e019000de009000dd
:10de6c001e0890007e310200000000000080fa00c5
:10de7c00000006000000fa000000370006c2bf00d8
:10de8c00614060000004e000fcff3a0006c2bf00e5
:10de9c00644060000004e000f8ff3a0006c2bf00d6
:10deac00684060000004e000f4ff3a0006c2bf00c6
:10debc00704060000004e000f0ff3a0009c2bf00af
:10decc000044b2000004e000ecff3a000080fa00cd
:10dedc00000006000400fa006009200020108800f1
:10deec0007e2a90007e2a80085c0a90085a0a90047
:10defc00b10920009140780080cfb30000c06000d1
:10df0c005040b3009be0b7008da0a9000071220027
:10df1c0001002000008fbe00040037000080eb00e1
:10df2c008080eb001e0f40005e9748001e00be0074
:10df3c00e00f5000e08f5800f8ff3a00100020006e
:10df4c000080fa00000006000000fa0007e2a900b9
:10df5c0085c0a90085a0a9008dc0a9008da0a9002d
:10df6c00100020000080fa00000006000400fa00f7
:10df7c006000b800008fbe0007e2a90085c0a900b0
:10df8c0085a0a9008da0a9000000eb00401088001e
:10df9c000071220001002000008fbe000400370039
:10dfac000080eb008080eb001e0f40005e97480065
:10dfbc001e00be00e00f5000e08f5800f8ff3a0042
:10dfcc00c4ff07000f0007000071220001002000b1
:10dfdc00008fbe00040037000080eb008080eb0057
:10dfec001e0f40005e9748001e00be00e00f500060
:10dffc00e08f5800f8ff3a00100020000080fa0073
:10e00c00000006000000fa0085c0a9008dc0a80021
:10e01c00100020000080fa00000006000000fa004a
:10e02c0085c0a9008dc0a900100020000080fa0056
:10e03c00000006000600fa000118220010c0b30010
:10e04c008048780008c2bf00704060000004e00007
:10e05c00170032000602a800007122000100200007
:10e06c00008fbe000b003700001822001040780013
:10e07c000004e00003003a00100020002007980084
:10e08c000d0037000080eb008080eb001e0f40007d
:10e09c005e9748001e00be00e00f5000e08f580055
:10e0ac00f1ff3a008000eb002107980002003700d6
:10e0bc000000eb00200798002e0090000080fa0072
:10e0cc00000006000600fa000118220060c0b30030
:10e0dc008048780008c2bf00684060000004e0007f
:10e0ec00170032000622a800007122000100200057
:10e0fc00008fbe000b003700001822001040780083
:10e10c000004e00003003a001000200020079800f3
:10e11c000d0037000080eb008080eb001e0f4000ec
:10e12c005e9748001e00be00e00f5000e08f5800c4
:10e13c00f1ff3a008000eb00210798000200370045
:10e14c000000eb00200798002e0090000080fa00e1
:10e15c00000006000600fa000118220050c0b300af
:10e16c00804878000642a8000071220001002000bf
:10e17c00008fbe000b003700001822001040780002
:10e18c000004e00003003a00100020002007980073
:10e19c000a0037000080eb008080eb001e0f40006f
:10e1ac005e9748001e00be00e00f5000e08f580044
:10e1bc00f1ff3a008000eb00210798002e00900040
:10e1cc000080fa00000006000600fa000118220088
:10e1dc0030c0b3008048780006c2bf0061406000c8
:10e1ec000004e00010003a0006c2bf00644060006a
:10e1fc000004e0000c003a0006c2bf00684060005a
:10e20c000004e00008003a0006c2bf007040600045
:10e21c000004e00004003a0006c2bf006240600047
:10e22c000004e000030032000000eb00200798001f
:10e23c001700370006a2a9000682a8000071220070
:10e24c0001002000008fbe000b00370000182200d8
:10e25c00104078000004e00003003a001100200098
:10e26c00210798000a0037000080eb008080eb004b
:10e27c001e0f40005e9748001e00be00e00f5000cd
:10e28c00e08f5800f1ff3a008000eb002107980066
:10e29c002e0090000080fa00000006000600fa0034
:10e2ac000118220030c0b3008048780006c2bf00bd
:10e2bc00614060000004e00010003a0006c2bf009c
:10e2cc00644060000004e0000c003a0006c2bf008d
:10e2dc00684060000004e00008003a0006c2bf007d
:10e2ec00704060000004e00004003a0006c2bf0069
:10e2fc00624060000004e000030032000000eb000c
:10e30c00200798001700370006a2a8000682a80074
:10e31c000071220001002000008fbe000b003700ae
:10e32c0000182200104078000004e00003003a00be
:10e33c0011002000210798000a0037000080eb0034
:10e34c008080eb001e0f40005e9748001e00be0050
:10e35c00e00f5000e08f5800f1ff3a008000eb0016
:10e36c00210798002e0090000080fa0000000600a3
:10e37c000a00fa003007980000712200010020000a
:10e38c0010079800210798000040eb00004f780020
:10e39c000118220040c0b3008048780000712200b0
:10e3ac000100200010079800210798001d0037007d
:10e3bc0006c2bf00614060000004e00013003a0098
:10e3cc0006c2bf00644060000004e0000f003a0089
:10e3dc0006c2bf00684060000004e0000b003a0079
:10e3ec0006c2bf00704060000004e00007003a0065
:10e3fc0009c2bf000044b2000004e00003003a0070
:10e40c0010c0b300004f78000b0037001e009000c6
:10e41c00ae00900061005000e0805800100798009a
:10e42c00210798001e009000ae009000e00f5000f5
:10e43c00e08f5800deff3a001e04e00003003a00b3
:10e44c000000eb00400798001e0037000662a80091
:10e45c00006a28001100200010079800210798007e
:10e46c001100370000182200104078000004e00072
:10e47c0007003a0000108000804078003e009000b9
:10e48c000148780010002000400798000d0037006c
:10e49c001e009000ae00900061005000e08058001b
:10e4ac0010079800210798001e009000ae00900005
:10e4bc00e00f5000e08f5800eaff3a000000eb003c
:10e4cc00400798004e0090000080fa000000060003
:10e4dc000800fa00404798000118220020c0b30041
:10e4ec00804878004e4090000000fb00101088001f
:10e4fc000071220001002000008fbe000b003700cd
:10e50c0000182200104078000004e00003003a00dc
:10e51c0010002000300798000a0037000080eb0044
:10e52c008080eb001e0f40005e9748001e00be006e
:10e53c00e00f5000e08f5800f1ff3a008000eb0034
:10e54c00310798003e0090000080fa0000000600a1
:10e55c00809fbe003400f80000002000a00188005d
:10e56c000000fa0085c0a900011822000040eb0051
:10e57c00804878000080fa003400f9004f00be009b
:10e58c00004006000400fa00200b81000000e000af
:10e59c0020003200c10a810080da2f00808f5000e9
:10e5ac001c003500c10a810080252000808f50009e
:10e5bc0018003c00d602a900d622a900d642a90018
:10e5cc00d662a9000000eb00200b8900c00a810074
:10e5dc0000017800120798001e0190000200e00074
:10e5ec0003003d001e0190000201ea001207980092
:10e5fc00007122001e019000110009000200d800d9
:10e60c00ef005000802c2700da810200000000008f
:10e61c004e003700c00a81000000e0000c003400fe
:10e62c00000b81000000e800000b8900e00a81006b
:10e63c000000e900e00a8900e00a81000000e00027
:10e64c000e003d0030002000e00a89000b0037006e
:10e65c00000b81000000e900000b8900e00a81003a
:10e66c000000e800e00a8900e00a8100e30f500096
:10e67c00020034000000eb00e00a8900e00a81008f
:10e68c00000f78001e017800e10f510013003200da
:10e69c001e007800e10f500004003c001e017800c1
:10e6ac000200e000080032001a0037001e0078005b
:10e6bc00e20f50000e0032001e017800e30f5100f3
:10e6cc001000320013003700d602a900d622a80091
:10e6dc00d642a900d662a8000e003700d602a900c7
:10e6ec00d622a800d642a800d662a900090037009d
:10e6fc00d602a800d622a900d642a800d662a9004c
:10e70c0004003700d602a800d622a900d642a900e0
:10e71c00d662a800c10a810080da2f00808f5000d9
:10e72c000a003500c10a810080252000808f50002e
:10e73c0006003c0010002000200b8900f100200096
:10e74c00802c2700da810200000000000080fa0013
:10e75c00000006000400fa00300b81000000e0000d
:10e76c0020003200d10a810080da2f00808f500007
:10e77c001c003500d10a810080252000808f5000bc
:10e78c0018003c00d682a900d6a2a900d6c2a900c6
:10e79c00d6e2a9000000eb00300b8900d00a810002
:10e7ac0000017800120798001e0190000200e000a2
:10e7bc0003003d001e0190000201ea0012079800c0
:10e7cc00007122001e019000110009000200d80007
:10e7dc00ef005000003b2700da810200000000002f
:10e7ec004e003700d00a81000000e0000c003d0014
:10e7fc00100b81000000e900100b8900f00a810069
:10e80c000000e900f00a8900f00a81000000e00035
:10e81c000e003d0030002000f00a89000b0037008c
:10e82c00100b81000000e800100b8900f00a810039
:10e83c000000e800f00a8900f00a8100e30f5000a4
:10e84c00020034000000eb00f00a8900f00a81009d
:10e85c00000f78001e017800e10f51001300320008
:10e86c001e007800e10f500004003c001e017800ef
:10e87c000200e000080032001a0037001e00780089
:10e88c00e20f50000e0032001e017800e30f510021
:10e89c001000320013003700d682a900d6a2a800bf
:10e8ac00d6c2a900d6e2a8000e003700d682a90075
:10e8bc00d6a2a800d6c2a800d6e2a900090037004b
:10e8cc00d682a800d6a2a900d6c2a800d6e2a9007a
:10e8dc0004003700d682a800d6a2a900d6c2a9008f
:10e8ec00d6e2a800d10a810080da2f00808f500078
:10e8fc000a003500d10a810080252000808f50004d
:10e90c0006003c0010002000300b8900f1002000b4
:10e91c00003b2700da810200000000000080fa00b2
:10e92c00000006000000fa008000eb00802c27009d
:10e93c0024810200000000008000eb00003b270057
:10e94c0024810200000000000080fa000000060094
:10e95c000200fa00000f7800d602a900d622a90006
:10e96c00d642a900d662a9001e00e00007003a00ba
:10e97c000000eb00c00a89008000eb00802c27000f
:10e98c00da810200000000003100370080c12f0046
:10e99c009e0f10000b003d0080c12f00c00a8900a3
:10e9ac00c20a8100008f2d00110009000200d8005e
:10e9bc0080007800802c2700da8102000000000023
:10e9cc0023003700803e20009e0f10000b00340007
:10e9dc00803e2000c00a8900c20a8100007122001a
:10e9ec00110009000200d80080007800802c27005c
:10e9fc00da81020000000000150037001e007800cc
:10ea0c00c00a89001e00e00009003d00008f2d00a7
:10ea1c001e017800110009000200d8008000780067
:10ea2c00802c2700da81020000000000080037006b
:10ea3c00007122001e017800110009000200d800ac
:10ea4c0080007800802c2700da8102000000000092
:10ea5c000080fa00000006000200fa00000f7800a7
:10ea6c00d682a900d6a2a900d6c2a900d6e2a900d6
:10ea7c001e00e00007003a000000eb00d00a8900fd
:10ea8c008000eb00003b2700da8102000000000050
:10ea9c003100370080c12f009e0f10000b003d008d
:10eaac0080c12f00d00a8900d20a8100008f2d006e
:10eabc00110009000200d80080007800003b2700fc
:10eacc00da8102000000000023003700803e2000a5
:10eadc009e0f10000b003400803e2000d00a8900ed
:10eaec00d20a810000712200110009000200d80036
:10eafc0080007800003b2700da8102000000000053
:10eb0c00150037001e007800d00a89001e00e000b6
:10eb1c0009003d00008f2d001e0178001100090036
:10eb2c000200d80080007800003b2700da81020048
:10eb3c000000000008003700007122001e01780060
:10eb4c00110009000200d80080007800003b27006b
:10eb5c00da810200000000000080fa0000000600cc
:10eb6c000800fa00000f7800110798001e007800ca
:10eb7c00300798003e0190000200e00003003d00c9
:10eb8c003e0090000000ea00300798001e01900043
:10eb9c00220798002e0090000000e00003003d00ca
:10ebac002e0190000201ea00220798003e0090001e
:10ebbc002e01900082004000803e2000808f50008b
:10ebcc0006003c001e0090001e00100060ff0700b5
:10ebdc001e0090001e0040009fff07000080fa00fe
:10ebec00000006000000fa00000b81000080fa0013
:10ebfc00000006000200fa00000f78001e007800ea
:10ec0c00000b89000080fa00000006000000fa00ea
:10ec1c00100b81000080fa00000006000200fa00d0
:10ec2c00000f78001e007800100b89000080fa009d
:10ec3c00000006001200fa00000f7800110798007f
:10ec4c00220798003307980044079800550798004e
:10ec5c0066079800500d8100000f980000032600f5
:10ec6c008e089000808f50001400320000032800a2
:10ec7c008e089000808f50001b0032000003230090
:10ec8c008e089000808f5000010032002100370068
:10ec9c006e039000de0290004e029000be019000c8
:10ecac002e0190009e0090001e0078006e7e0200e7
:10ecbc000000000070079800180037006e039000e9
:10eccc00de0290004e029000be0190002e019000da
:10ecdc009e0090001e007800ee78020000000000fc
:10ecec00700798000d0037006e039000de02900054
:10ecfc004e029000be0190002e0190009e009000ec
:10ed0c001e007800ae7b0200000000007007980027
:10ed1c0002003700b0002000700798007e009000c1
:10ed2c000080fa00000006000600fa00000f7800d0
:10ed3c0011079800500d8100200798000003260051
:10ed4c00ae009000808f50000e00320000032800af
:10ed5c00ae009000808f50000f00320000032300a3
:10ed6c00ae009000808f5000010032000e00370082
:10ed7c009e0090001e0078003a3602000000000051
:10ed8c00090037009e0090001e007800b666020055
:10ed9c0000000000040037009e0090001e00780068
:10edac00a6620200000000000080fa0000000600cd
:10edbc000000fa00510d810000032300808f5000e9
:10edcc000100320002003700e433020000000000b2
:10eddc000080fa00000006000400fa00e48902003a
:10edec0000000000888a020000000000d1a2a900e7
:10edfc0040062000100798000400370000000000b7
:10ee0c001e0090000000e900100798001e00900002
:10ee1c000000e000f9ff3a00d1a2a8004006200053
:10ee2c001007980004003700000000001e0090003e
:10ee3c000000e900100798001e0090000000e000a0
:10ee4c00f9ff3a0081e0a900f1048000f0002f00e6
:10ee5c00808060000066200000804000f004880084
:10ee6c008040eb00c0cdb300b08a0200000000006f
:10ee7c001047980011c0b300c0cdb300b08a020097
:10ee8c0000000000004f78001e4090000080fb0046
:10ee9c00c800dd001e80fb0000807000500d890052
:10eeac00510d810000032300808f500004003a00b4
:10eebc008000eb000000eb009bff07001100370007
:10eecc00510d810000032600808f500004003a0091
:10eedc00110020001000200093ff070009003700ec
:10eeec00510d810000032800808f500005003a006e
:10eefc008000eb000000eb008bff07004860020075
:10ef0c0000000000aaff0700500d81000080fa00ed
:10ef1c00000006000800fa0020079800310798004e
:10ef2c0032c0bf000080fb00000f78002e00900064
:10ef3c0032e0b7003e0090001000ba0010079800b5
:10ef4c001e00780032e0b7001e0090000080fa002e
:10ef5c00000006000600fa00500d81002007980002
:10ef6c0000032600ae009000808f5000210032007c
:10ef7c0000032800ae009000808f5000200032006b
:10ef8c0000032300ae009000808f5000010032007f
:10ef9c001e003700e1ff2f00f0072000ddff070007
:10efac0063006000100798001e009000e20f5000f4
:10efbc000a0032009e009000e38f50000a003200dd
:10efcc001e009000e10f50000100320009003700d4
:10efdc0011002000010f78000e00370020002000e7
:10efec00000f78000b0037008000eb00010f780059
:10effc000800370010002000000f780005003700d3
:10f00c0011002000010f7800020037000080eb0097
:10f01c00000f78001e0078000080fa000000060047
:10f02c000600fa00000f780011079800500d8100bf
:10f03c002007980000032600ae009000808f50003f
:10f04c000e00320000032800ae009000808f5000ac
:10f05c000f00320000032300ae009000808f5000a0
:10f06c00010032000e0037009e0090001e00780058
:10f07c00b83a020000000000090037009e00900022
:10f08c001e007800f066020000000000040037004b
:10f09c009e0090001e007800e0620200000000005c
:10f0ac000080fa00000006000600fa00004f78000d
:10f0bc001147980022479800500d810020079800b6
:10f0cc0000032600ae009000808f5000110032002b
:10f0dc0000032800ae009000808f50001300320017
:10f0ec0000032300ae009000808f5000010032001e
:10f0fc00130037002e4290009e4190001e4190005c
:10f10c009e40780080c2b30002370200000000006d
:10f11c000b0037002e4190009e4090001e4078005e
:10f12c003867020000000000050037002e419000f7
:10f13c009e4090001e4078002863020000000000f2
:10f14c000080fa00000006000600fa00008fbe00e6
:10f15c00500d81002007980000032600ae0090009f
:10f16c00808f50000d00320000032800ae0090008c
:10f17c00808f50000d00320000032300ae00900081
:10f18c00808f5000010032000b0037001e00be00c3
:10f19c005839020000000000070037001e00be00b6
:10f1ac005c67020000000000030037001e00be0078
:10f1bc004c630200000000000080fa000000060012
:10f1cc000000fa00500d81000080fa0000000600db
:10f1dc002400fa00000f9800110f9800220f9800dd
:10f1ec00330f9800440f9800550f9800660f980045
:10f1fc000e08900070004000000f98001e08900050
:10f20c0068004000100f98005e0890000000e000bd
:10f21c00030032004e0890000000e00003003a00aa
:10f22c000080eb00700f98002a0137008e089000c8
:10f23c002e08900080804000002d2000808f500010
:10f24c00030036008080eb00710f9800210137001d
:10f25c009e0890003e08900080804000801e200098
:10f26c00808f5000030036000080eb00700f980078
:10f27c00180137002e0890004e099000110009006b
:10f28c000280d8008000fd000000e0000300320086
:10f29c008080eb00710f98000e0137003e08900043
:10f2ac005e099000110009000280d8008000fd006a
:10f2bc000000e000030032000080eb00700f9800ab
:10f2cc00040137005e089000630060000000e0005d
:10f2dc0039003a004e089000630060000000e00026
:10f2ec0011003a0000082000000f780040002000b8
:10f2fc00100798005e0890004200de00300798006e
:10f30c004e0890004200de00200798001e08900076
:10f31c0064005000100f98000e089000640050001c
:10f32c00000f98005a0037004e08900061006000f2
:10f33c000000e00011003a0000042000000f7800eb
:10f34c0020002000100798005e0890000000d100fb
:10f35c00300798004e0890000000d100200798005c
:10f36c001e0890000080e900100f98000e08900015
:10f37c000080e900000f98004500370000022000d3
:10f38c00000f78001000200010079800de08900095
:10f39c00310798004e089000200798001e08900036
:10f3ac000000e900100f98000e0890000000e90022
:10f3bc00000f9800360037005e0890006100600076
:10f3cc000000e00024003a004e089000610060004c
:10f3dc000000e00011003a0000042000000f78004b
:10f3ec0020002000100798005e0890000000d1005b
:10f3fc00300798004e0890000000d10020079800bc
:10f40c001e0890000080e900100f98000e08900074
:10f41c000080e900000f98001d003700000220005a
:10f42c00000f78001000200010079800de089000f4
:10f43c00310798004e089000200798001e08900095
:10f44c000000e900100f98000e0890000000e90081
:10f45c00000f98000e0037001000200010079800d5
:10f46c0000022000000f7800ce08900021079800c1
:10f47c005e089000300798001e0890000000e9001c
:10f48c00100f98000e0890000000e900000f980083
:10f49c002e0090000000e900600798003e009000ec
:10f4ac000000e900700798002e0890004e099000ab
:10f4bc00110009000280d800500798003e08900007
:10f4cc005e099000110009000280d80040079800e6
:10f4dc00102d20001e019000110009000200d80020
:10f4ec00800078001e0190000e089000811f7800ab
:10f4fc00110009000280d80001017800cf007800cb
:10f50c0096650200000000000000e00003003200dd
:10f51c008080eb00710f98006e003700901e200069
:10f52c001e019000110009000200d8008000780034
:10f53c001e0190001e089000811f78001100090028
:10f54c000280d80001017800cf007800ec65020041
:10f55c00000000000000e000030032000080eb001f
:10f56c00700f98005b003700811e20001e08900071
:10f57c00f8650200000000000000e000030032000b
:10f58c008080eb00710f9800520037006e089000dd
:10f59c000000e0001b003a001e00780000179800e5
:10f5ac00000420008e109000808f50000d0032005f
:10f5bc00000820008e109000808f50000d0032004b
:10f5cc00000220008e109000808f5000010032004d
:10f5dc002600370000c9b300fa63020000000000e7
:10f5ec002200370000c5b300fa63020000000000df
:10f5fc001e00370000c1b300fa63020000000000d7
:10f60c001a0037001e007800101798000004200024
:10f61c009e109000808f50000d00320000082000da
:10f62c009e109000808f50000d00320000022000d0
:10f63c009e109000808f5000010032000b003700ac
:10f64c0000cbb300fa630200000000000700370093
:10f65c0000c9b300fa630200000000000300370089
:10f66c0000c5b300fa630200000000001e00780021
:10f67c00804078006e0890003e650200000000009b
:10f68c000000e000030032000080eb00700f9800d7
:10f69c00100037006e089000110007000001780080
:10f6ac007e029000ee019000de0090004e00900073
:10f6bc0010890200000000000000e000030032008e
:10f6cc008080eb00710f9800020037000000eb0007
:10f6dc00700f98007e0890000080fa000000060071
:10f6ec000600fa00000f78001e0078002007980032
:10f6fc002e009000e10f50000a0032002e00900006
:10f70c00e20f50000a0032002e0090000000e000d2
:10f71c00010032000900370010002000100798008b
:10f72c000800370020002000100798000500370063
:10f73c002000200010079800020037001000200065
:10f74c00100798001e0090000080fa0000000600d0
:10f75c002400fa00000f9800110f9800220f980057
:10f76c00330f9800440f9800550f9800660f9800bf
:10f77c000e08900064004000000f98001e089000d6
:10f78c0064004000100f98005e0890000000e0003c
:10f79c00030032004e0890000000e00003003a0025
:10f7ac0010002000700f98002a0137008e0890007e
:10f7bc002e08900080804000402c2000808f50004c
:10f7cc000300360021002000710f98002101370042
:10f7dc009e0890003e08900080804000401e200053
:10f7ec00808f50000300360030002000700f98000e
:10f7fc00180137002e0890004e09900011000900e6
:10f80c000280d8008000fd000000e0000300320000
:10f81c0041002000710f98000e0137003e08900047
:10f82c005e099000110009000280d8008000fd00e4
:10f83c000000e0000300320050002000700f980020
:10f84c00040137005e089000630060000000e000d7
:10f85c0039003a004e089000630060000000e000a0
:10f86c0011003a0000082000000f78004000200032
:10f87c00100798005e0890004200de0030079800e8
:10f88c004e0890004200de00200798001e089000f1
:10f89c0064005000100f98000e0890006400500097
:10f8ac00000f98005a0037004e089000610060006d
:10f8bc000000e00011003a0000042000000f780066
:10f8cc0020002000100798005e0890000000d10076
:10f8dc00300798004e0890000000d10020079800d7
:10f8ec001e0890000080e900100f98000e08900090
:10f8fc000080e900000f980045003700000220004e
:10f90c00000f78001000200010079800de0890000f
:10f91c00310798004e089000200798001e089000b0
:10f92c000000e900100f98000e0890000000e9009c
:10f93c00000f9800360037005e08900061006000f0
:10f94c000000e00024003a004e08900061006000c6
:10f95c000000e00011003a0000042000000f7800c5
:10f96c0020002000100798005e0890000000d100d5
:10f97c00300798004e0890000000d1002007980036
:10f98c001e0890000080e900100f98000e089000ef
:10f99c000080e900000f98001d00370000022000d5
:10f9ac00000f78001000200010079800de0890006f
:10f9bc00310798004e089000200798001e08900010
:10f9cc000000e900100f98000e0890000000e900fc
:10f9dc00000f98000e003700100020001007980050
:10f9ec0000022000000f7800ce089000210798003c
:10f9fc005e089000300798001e0890000000e90097
:10fa0c00100f98000e0890000000e900000f9800fd
:10fa1c002e0090000000e900600798003e00900066
:10fa2c000000e900700798002e0890004e09900025
:10fa3c00110009000280d800500798003e08900081
:10fa4c005e099000110009000280d8004007980060
:10fa5c00502c20001e019000110009000200d8005b
:10fa6c00800078001e0190000e089000811f780025
:10fa7c00110009000280d80001017800cf00780045
:10fa8c00c8610200000000000000e000030032002a
:10fa9c0061002000710f98006e003700501e20008e
:10faac001e019000110009000200d80080007800af
:10fabc001e0190001e089000811f780011000900a3
:10facc000280d80001017800cf0078001e6202008d
:10fadc00000000000000e000030032007000200075
:10faec00700f98005b003700411e20001e0890002c
:10fafc002a620200000000000000e0000300320057
:10fb0c0081002000710f9800520037006e089000a1
:10fb1c000000e0001b003a001e007800001798005f
:10fb2c00000420008e109000808f50000d003200d9
:10fb3c00000820008e109000808f50000d003200c5
:10fb4c00000220008e109000808f500001003200c7
:10fb5c002600370040c0b3005c60020000000000cb
:10fb6c002200370020c0b3005c60020000000000df
:10fb7c001e0037000040eb005c600200000000003b
:10fb8c001a0037001e00780010179800000420009f
:10fb9c009e109000808f50000d0032000008200055
:10fbac009e109000808f50000d003200000220004b
:10fbbc009e109000808f5000010032000b00370027
:10fbcc0050c0b3005c60020000000000070037006a
:10fbdc0040c0b3005c60020000000000030037006e
:10fbec0020c0b3005c600200000000001e00780022
:10fbfc00804078006e0890007061020000000000e8
:10fc0c000000e0000300320090002000700f98000c
:10fc1c00100037006e0890001100070000017800fa
:10fc2c007e029000ee019000de0090004e009000ed
:10fc3c0010890200000000000000e0000300320008
:10fc4c00a1002000710f9800020037000000eb00ab
:10fc5c00700f98007e0890000080fa0000000600eb
:10fc6c000600fa00000f78001e00780020079800ac
:10fc7c002e009000e10f50000a0032002e00900080
:10fc8c00e20f50000a0032002e0090000000e0004d
:10fc9c000100320009003700100020001007980006
:10fcac0008003700200020001007980005003700de
:10fcbc0020002000100798000200370010002000e0
:10fccc00100798001e0090000080fa00000006004b
:10fcdc002200fa0070079800010f9800120f98008c
:10fcec00230f9800340f9800450f9800560f98007a
:10fcfc007e009000200db000700798000e08900058
:10fd0c0067004000000f98004e0890000000e000d3
:10fd1c00030032003e0890000000e00003003a00af
:10fd2c000080eb00600f980010013700fe0090007f
:10fd3c001e0890008080400020352000808f5000ed
:10fd4c00030036008080eb00610f9800070137003c
:10fd5c008e0890002e08900080804000701e2000bd
:10fd6c00808f5000030036000080eb00600f98007d
:10fd7c00fe0037001e0890003e099000110009009b
:10fd8c000280d8008000fd000000e000030032007b
:10fd9c008080eb00610f9800f40037002e08900073
:10fdac004e099000110009000280d8008000fd006f
:10fdbc000000e000030032000080eb00600f9800b0
:10fdcc00ea0037004e089000630060000000e0007d
:10fddc0033003a003e089000630060000000e00031
:10fdec000f003a0030032000000f78004e089000fe
:10fdfc004200de00200798003e0890004200de0022
:10fe0c00100798000e08900064005000000f980036
:10fe1c007e0090006400500070079800500037007e
:10fe2c003e089000610060000000e0000f003a0006
:10fe3c0010012000000f78004e0890000000d10047
:10fe4c00200798003e0890000000d1001007980091
:10fe5c000e0890000080e900000f98007e009000d2
:10fe6c000080e900700798003d0037004004200036
:10fe7c00000f7800ce089000210798003e089000f3
:10fe8c00100798000e0890000000e900000f980081
:10fe9c007e0090000000e9007007980030003700e9
:10feac004e089000610060000000e00020003a0065
:10febc003e089000610060000000e0000f003a0076
:10fecc0010012000000f78004e0890000000d100b7
:10fedc00200798003e0890000000d1001007980001
:10feec000e0890000080e900000f98007e00900042
:10fefc000080e900700798001900370040042000ca
:10ff0c00000f7800ce089000210798003e08900062
:10ff1c00100798000e0890000000e900000f9800f0
:10ff2c007e0090000000e900700798000c0037007c
:10ff3c0040042000000f7800be08900011079800c4
:10ff4c004e089000200798000e0890000000e90071
:10ff5c00000f98007e0090000000e90070079800e8
:10ff6c001e0090000000e900500798002e00900041
:10ff7c000000e900600798001e0890003e09900000
:10ff8c00110009000280d800400798002e0890004c
:10ff9c004e099000110009000280d800300798002b
:10ffac005e08900050340200000000000000e000e9
:10ffbc00030032008080eb00610f98006b0037006b
:10ffcc001e00780094340200000000000000e000e5
:10ffdc00030032000080eb00600f980063003700d4
:10ffec005e0890000000e0001a003a009e007800c5
:10fffc00710f980030032000fe089000808f500095
:020000040001f9
:10000c001000320040042000fe089000808f500049
:10001c00040032007e089000f10f50000500320001
:10002c002500370000032000c2340200000000004d
:10003c002100370000022000c23402000000000042
:10004c001d0037000000eb00c2340200000000006d
:10005c00190037009e00780001179800300320002b
:10006c008e109000808f5000100032004004200051
:10007c008e109000808f5000040032000e10900003
:10008c00f10f5000050032000b0037000004200077
:10009c00c2340200000000000700370000032000fb
:1000ac00c2340200000000000300370000022000f0
:1000bc00c234020000000000313520007e009000a8
:1000cc000c350200000000000000e00003003200cc
:1000dc008080eb00610f980024003700811e200007
:1000ec000e08900068350200000000000000e000df
:1000fc00030032000080eb00600f98001b003700fb
:10010c007e0090000001e800711e20000e08900097
:10011c00be350200000000000000e00003003200c9
:10012c008080eb00610f9800100037005e08900093
:10013c0011000700000178006e029000de019000b3
:10014c00ce0090003e0090001089020000000000dc
:10015c000000e000030032000080eb00600f98000c
:10016c00020037008000eb00610f98006e089000d1
:10017c000080fa00000006000600fa00000f78006c
:10018c001e007800200798002e009000e10f500010
:10019c000a0032002e009000e20f50000a003200dc
:1001ac002e0090000000e000010032000900370032
:1001bc0010002000100798000800370020002000d5
:1001cc001007980005003700200020001007980049
:1001dc000200370010002000100798001e0090004d
:1001ec000080fa00000006000000fa000000eb009e
:1001fc00800888000111200091407800f0ccb300f9
:10020c0000c0600010e1b7000000eb00300888006f
:10021c00205c20006008880084c0a9008cc0a80065
:10022c0011e1a8000080fa00000006000000fa00ae
:10023c0011e1a9000080fa00000006000800fa0095
:10024c001007980021079800700d8100000f7800ae
:10025c000b0037001e007800b00090001e009000cc
:10026c00808f500003003a001100200031079800e5
:10027c00210037001e007800c0009000010f7800ac
:10028c001e00e000f3ff3a00a0002000f00702007f
:10029c0000000000000f78001e00e00003003a0090
:1002ac0010002000a407020000000000ae00900027
:1002bc001e007800010878009e0078000000eb001a
:1002cc00900098009e00780010c0b300c0409800c9
:1002dc001e0078009e00900031009800710d810086
:1002ec001e007800410098001e007800700d8900f7
:1002fc0011002000310798003e0090000080fa00a9
:10030c00000006000800fa00200798000000eb002f
:10031c0010079800700d8100000f78001b0037004b
:10032c001e007800b00090002e009000808f5000ce
:10033c0011003a001e0090000000e00005003200a1
:10034c001e007800c00090001e0090004100980034
:10035c00030037001e00780040009000700d8900eb
:10036c001e0078001409020000000000110020009b
:10037c0031079800090037001e007800100798001c
:10038c001e007800c0009000010f78001e00e000f5
:10039c00e3ff3a0020002000300798003e00900058
:1003ac000080fa00000006000800fa001007980010
:1003bc0021079800700d8100000f78000e003700a7
:1003cc001e007800b00090001e009000808f50003e
:1003dc0006003a00ae0090001e007800010878007c
:1003ec001100200031079800070037001e0078002c
:1003fc00c0009000010f78001e00e000f0ff3a00f2
:10040c0020002000300798003e0090000080fa0089
:10041c00000006000600fa0010079800700d81001d
:10042c00000f78000e0037001e007800b00090001e
:10043c001e009000808f500006003a009e0078004d
:10044c000000eb009000980011002000210798009c
:10045c00070037001e007800c0009000010f7800e4
:10046c001e00e000f0ff3a0020002000200798005a
:10047c002e0090000080fa00000006000600fa0032
:10048c0010079800700d8100000f78000e003700e7
:10049c001e007800b00090001e009000808f50006d
:1004ac0006003a009e0078000040eb00c040980027
:1004bc001100200021079800070037001e0078006b
:1004cc00c0009000010f78001e00e000f0ff3a0021
:1004dc0020002000200798002e0090000080fa00d9
:1004ec00000006000600fa0010079800700d81004d
:1004fc00000f78000e0037001e007800b00090004e
:10050c001e009000808f500006003a009e0078007c
:10051c0010c0b300c04098001100200021079800c3
:10052c00070037001e007800c0009000010f780013
:10053c001e00e000f0ff3a00200020002007980089
:10054c002e0090000080fa00000006003600f80033
:10055c00809fbe00829fbe00849fbe00869fbe000f
:10056c003400f80000002000a00188000200fa000e
:10057c00700d8100000f780084c0a9001e003700a8
:10058c001e00780040409000e14f500017003a00e8
:10059c001e007800100078000000e000130032000c
:1005ac001e007800100090008000e8001e0078000b
:1005bc00110098001e007800100090008000780058
:1005cc001e007800100078000000e900808f5000b9
:1005dc00060036001e00780030009000000001007c
:1005ec009e0078000000eb00900098001e00780040
:1005fc00c0009000010f78001e00e000e0ff3a0000
:10060c000080fa003400f9004f03be004f02be0018
:10061c004f01be004f00be003600f900004006003e
:10062c000000fa00dec2a8008200a8008400a90025
:10063c008c00a8000080fa00000006003600f800cc
:10064c00809fbe00829fbe00849fbe00869fbe001e
:10065c003400f80000002000a00188000000fa001f
:10066c008c00a90051012000603628002481020072
:10067c0000000000511922000040eb008048780077
:10068c00501922009040780040192200014878004f
:10069c00401922009040780060192200014878002f
:1006ac000080fa003400f9004f03be004f02be0078
:1006bc004f01be004f00be003600f900004006009e
:1006cc000200fa00300d8100e10f40001e003a00dc
:1006dc00e0c2bf000044b2000004e0000800320099
:1006ec008c00a8008400a9006036280088810200d4
:1006fc00000000000080eb00300d89006d00370019
:10070c009100200060362800da8102000000000011
:10071c00511922000040eb0080487800501922004b
:10072c0090407800401922000148780040192200be
:10073c009040780060192200014878000000eb001e
:10074c00300d89005b003700300d8100e10f500047
:10075c0010003a00e0c2bf000080fb004600de0043
:10076c0061406000804078006019220001487800e8
:10077c002101200060362800da8102000000000010
:10078c001100200010002000d244020000000000e4
:10079c0048003700300d8100e10f50001500340087
:1007ac00300d8100e60f500012003c00e0c2bf008b
:1007bc000080fb004600de0061406000104798009e
:1007cc001e4090008080fb00300d81006600100000
:1007dc000008dd0010479800401922009040780076
:1007ec001e40900080c04000401922000148780053
:1007fc0030003700300d8100e60f5000130034003c
:10080c00300d8100ec0f500010003c00e0c2bf0026
:10081c000080fb004600de0061406000004f780065
:10082c009e80fb00300d81006c0010000008dd0084
:10083c00004f780050192200104078009e40400074
:10084c0050192200014878001a003700300d810041
:10085c00ed0f500017003a008000eb001000200054
:10086c00d2440200000000008c00a8008400a90003
:10087c006036280088810200000000000080eb0038
:10088c00300d89006019220090407800401a220037
:10089c00014878004019220090407800701922001d
:1008ac0001487800501922009040780080192200ed
:1008bc0001487800300d8100e10f40000300320048
:1008cc00300d81000000e800300d89000080fa0036
:1008dc00000006000000fa00401a220010407800c8
:1008ec000080fb000080fa00000006000000fa0007
:1008fc0070192200104078000080fb000080fa0084
:10090c00000006000000fa00801922001040780058
:10091c000080fb000080fa00000006000200fa00d4
:10092c00000f78009e007800c20b8100400620006a
:10093c000088b9000200400080004000007e2100c9
:10094c0000804000100078000080fa0000000600d3
:10095c000c00fa0040079800510798006000b8009e
:10096c0020079800310798004e009000e20f5000cd
:10097c0030003e005e0090000000e0002d003200d0
:10098c00de00900040062000808f500029003e00c1
:10099c000000eb0010079800c10b81005e00900076
:1009ac00008050005006b0004206200011000900e3
:1009bc000280d8008000fd00000f7800190037007d
:1009cc00ce0090001e017800400620000088b9007f
:1009dc000200400080004000007e210000804000aa
:1009ec00100078006101b9002e009000be0090004c
:1009fc0000004100818049002007980031079800d1
:100a0c001e0090000000e800100798001e00e8008f
:100a1c0042062000110009000200d8008000fd00f1
:100a2c00000f78009e0090005e009000808f5000b8
:100a3c00e3ff39005e0090006101b8002e009000c9
:100a4c00be009000de040200000000000080fa00ee
:100a5c00000006000800fa00300798000000eb00c8
:100a6c001007980070382100000f78000000eb0090
:100a7c00200798002e003700be0090002e01900039
:100a8c00400620000088b9000200400080004000b1
:100a9c00007e210000804000900078001e00900035
:100aac00808f50000b003400be0090002e0190008f
:100abc00400620000088b900020040008000400081
:100acc00007e210000804000900078001107980003
:100adc0014003700be0090002e019000400620004c
:100aec000088b9000200400080004000007e210018
:100afc0000804000100078009e0f500009003d005f
:100b0c00be0090002e019000400620000088b90025
:100b1c000200400080004000007e21000080400068
:100b2c00100f78002e0090000000e80020079800bd
:100b3c00ae00900030062000808f5000ceff3400b5
:100b4c001e0090001e0050000080fa0000000600fd
:100b5c000800fa0010079800210798003207980047
:100b6c003e0090000000e00024003200be00900027
:100b7c0040062000808f500020003e000000eb005b
:100b8c00000f7800190037003e0090001e00500046
:100b9c0000004000800078002e0090000080400093
:100bac000082e9009e019000c10b81001e007800bc
:100bbc000080400042062000110009000280d8008d
:100bcc008000fd0000017800400620000098b9006c
:100bdc000200400080004000007e210000804000a8
:100bec0010007800000a78001e0fe8009e007800c4
:100bfc003e009000808f5000e3ff39000080fa0027
:100c0c00000006003000fa00889fbe008a1f7800a2
:100c1c000000eb00300798000000eb002007980064
:100c2c000f0037003e00900080004000401422006e
:100c3c00808040000000eb00800878003e009000af
:100c4c00e80047004200dd00010140006000b800f0
:100c5c000089be003e0090000000e80030079800bc
:100c6c003e009000e90f5000eeff340027003700e3
:100c7c000000eb00300798001e0037003e05900086
:100c8c003e009000e80047004200dd0001004000fb
:100c9c001004be003e00900045000700cf80de002f
:100cac000801400089814800e80047004250dd00ff
:100cbc00010040000288be006000b800008fbe003a
:100ccc000400370010002000010020001e0f40001f
:100cdc005e974800703e200001002000be0f1000ff
:100cec00ae8f1800f7ff34003e0090000000e800c3
:100cfc00300798003e009000e90f5000dfff3400f1
:100d0c002e0090000000e80020079800ae00900034
:100d1c0030062000808f5000d5ff34000000eb001f
:100d2c00300798001b0037003e0590003e009000f5
:100d3c00e80047004200dd00010040001000be004a
:100d4c007c050200000000000004be002e00900094
:100d5c00cf80de007c050200000000000001be0018
:100d6c000800be005a040200000000000405020046
:100d7c0000000000000178008a00450040142200a9
:100d8c0000804000020878003e0090000000e8005f
:100d9c00300798003e009000e90f5000e2ff34004d
:100dac004f0578004f04be000080fa0000000600da
:100dbc000400fa00000f7800900020009e0f100035
:100dcc00030036000000eb00100798000c00370001
:100ddc001e0078008000400040b6210000804000da
:100dec00100178001e0078008000400080b72100c0
:100dfc00008040001000780000015100120798009c
:100e0c001e0090000080fa00000006000600fa00a8
:100e1c00100798001e009000e90f500003003600e8
:100e2c000000eb0020079800180037001e0090000f
:100e3c008000400040b62100008040001001780086
:100e4c001e0090008000400080b721000080400010
:100e5c0010007800000151001e009000800040003e
:100e6c00401422000080400010007800000f510058
:100e7c001e00e000030034001e00780020079800dc
:100e8c00020037000000eb00200798002e009000b5
:100e9c000080fa00000006000400fa00000f780041
:100eac00900020009e0f1000030036000000eb00a5
:100ebc0010079800060037001e00780080004000e4
:100ecc0040b6210000804000100078001007980008
:100edc001e0090000080fa00000006000800fa00d6
:100eec0020079800310798006000b800008fbe0002
:100efc000400370010002000010020001e0f4000ed
:100f0c005e9748002e009000be009000be0f1000af
:100f1c00ae8f1800f7ff35000080fa0000000600c5
:100f2c000000fa00e6c2bf000080fb004600de00b5
:100f3c00614060000081fb00e7c2bf000080fb0045
:100f4c000000d100614060000080fb000000400008
:100f5c0080007800e7c2bf00614060000080fb00a9
:100f6c00008040000000400080007800e6c2bf0016
:100f7c000080fb004700de000080fb00008040008a
:100f8c0000004000000041000080fa000000060054
:100f9c000200fa007c8a0200000000000004e0005d
:100fac0009003200d00b810000004000810c2000b1
:100fbc008080400080a32100008040001000780059
:100fcc00000f7800020037000000eb00000f7800e3
:100fdc001e0078000080fa00000006000200fa00f3
:100fec007c8a0200000000000004e00018003200bf
:100ffc00d00b810000004000810c2000808040005c
:10100c0080a321000080400090007800a07e2f007b
:10101c0000804000cf80de007c0502000000000054
:10102c0002002000832c24007c060200000000003b
:10103c0002002000533f24005a040200000000006c
:10104c004605020000000000000f78000200370087
:10105c000000eb00000f78001e0078000080fa0002
:10106c00000006000000fa000000eb00f00b890005
:10107c000080fa00000006000400fa00881f7800c7
:10108c00f80b81006140b9007c05020000000000f3
:10109c00008fbe000800e00006003d0002002000aa
:1010ac00037824001e00be009c0202000000000019
:1010bc00008fbe001e00be0032b22d0093d723005d
:1010cc007c060200000000004f0478000080fa004b
:1010dc00000006000800fa00881f7800f80b810059
:1010ec006140b9007c050200000000002007980058
:1010fc00310798000800e00008003d0002002000c5
:10110c00037824002e009000be0090009c02020088
:10111c000000000020079800310798002e00900076
:10112c00be00900032b22d0093d723007c06020043
:10113c0000000000008fbe000000eb00f00b8900e7
:10114c001e00be004f0478000080fa00000006006c
:10115c003400f800881f780008002000a8018800df
:10116c004f0478000000fa0086c0a9001fe1a80017
:10117c0021e1a9000080fa003400f90000400600cb
:10118c000000fa0020002000000988000000eb009d
:10119c00c008880010002000e008880086c0a90064
:1011ac008ec0a80021e1a8000080fa000000060013
:1011bc000000fa0020002000f0088800b0ec80004d
:1011cc00a0088800b0ec80000000e800d00888007f
:1011dc0086a0a9001fe1a9008ea0a8000080fa003b
:1011ec00000006000200fa00000f78000000eb007f
:1011fc00506088001e007800c0ec88000000eb00f6
:10120c00d0ec8800eaff0700ddff07000080fa0041
:10121c00000006001200fa00300798004107980001
:10122c005207980063079800740798000000eb00c1
:10123c0010079800ce0090005e0090000088b90066
:10124c00800078006e0090000000e8000088b90073
:10125c000000e80080007800a0142000808f50006f
:10126c00030036000080eb00000f980032003700be
:10127c000000eb0020079800210037000000eb0075
:10128c00000f7800080037001e019000c1d9210022
:10129c0010c0b30000f178001e0090000000e800c0
:1012ac00100798001e0fe8005e0090009e0f1000c3
:1012bc00f5ff35000000eb00000f78000800370048
:1012cc001e019000c1d921000040eb0000f1780014
:1012dc001e0090000000e800100798001e0fe800a8
:1012ec00ee0090005e0090000088b9009e0f500048
:1012fc00f3ff3c002e0090000000e800200798004f
:10130c00ae0090004e009000808f5000dbff350047
:10131c001e019000c1d9210020c0b30000f178005b
:10132c007e009000b0ec88003e0090006060880069
:10133c000000eb00000f98000e0890000080fa00ef
:10134c00000006000000fa00d0ec80000080fa00db
:10135c00000006000200fa00888a0200000000006b
:10136c00bc6f0200000000009c8a0200000000001c
:10137c00f1c0b300c0c3b300b08a0200000000008b
:10138c00004f7800a68a02000000000000c4b300e1
:10139c009e4f100004003a00c11a220010c0b30086
:1013ac008048780003003700c11a22000040eb008f
:1013bc00804878000080fa00000006000000fa0067
:1013cc00c4c2a900c4e2a900c522a900c582a90013
:1013dc00c542a900c5a2a900c5c2a900c5e2a900c1
:1013ec00c0c2a900c0e2a900c122a900c182a90003
:1013fc00c142a900c1a2a900c1c2a900c1e2a900b1
:10140c00d022a900cc22a900d042a900cc42a9002c
:10141c00e2e2a900e302a900e802a900e822a9007f
:10142c00dee2a900df02a900e402a900e422a9007f
:10143c00e202a900de02a900d602a900d622a90068
:10144c00d642a900d662a900d682a900d6a2a900cc
:10145c00d6c2a900d6e2a900d202a900d222a900c4
:10146c00d242a900d262a900d282a900d2a2a900bc
:10147c00d2c2a900d2e2a900d1a2a900cda2a90092
:10148c00e842a900e862a900e442a900e462a900cc
:10149c00de22a800dec2a800e4c2a800e4e2a80094
:1014ac00e502a800e522a800d302a800d322a800d8
:1014bc00d342a800d362a800d382a800d3a2a8006c
:1014cc00d3c2a800d3e2a800a2ff0700c01a2200d2
:1014dc00104078000004e000020032009668020020
:1014ec00000000000080fa00000006000000fa0076
:1014fc00c01a2200104078000080fb000080fa0027
:10150c00000006000000fa00706f020000000000ee
:10151c000080fa00000006000000fa00aa6f02002a
:10152c00000000000080fa00000006000000fa0035
:10153c0008700200000000000080fa0000000600a5
:10154c000000fa0014700200000000000080fa0095
:10155c00000006000400fa0020479800314798006c
:10156c000040eb00004f78002100370010c0b300a2
:10157c00004f780020700200000000001e4f600039
:10158c002e4090006e720200000000001e4f6000a2
:10159c003e4090006e720200000000001e4f600082
:1015ac0068700200000000001e4f60002e4090008a
:1015bc000040e8006e720200000000001e4f600048
:1015cc000e00e800be710200000000001e4f60001b
:1015dc005471020000000000b07002000000000016
:1015ec001e04e00004003a00bc6f02000000000082
:1015fc001e04e000ddff32001e4090000000fb00e6
:10160c000080fa00000006000600fa00204798004f
:10161c0031479800424798000040eb00004f78009b
:10162c001800370010c0b300004f78002070020083
:10163c00000000001e4f60002e4090006e720200f1
:10164c00000000001e4f60003e4090006e720200d1
:10165c00000000001e4f60004e4090006e720200b1
:10166c00000000001e4f6000b0700200000000007f
:10167c001e4f60001e04e00004003a00bc6f020024
:10168c00000000001e04e000e6ff32001e00fb001c
:10169c000080fa00000006008540a900809fbe0073
:1016ac00821f7800080ce20015003200040ce200e6
:1016bc0016003200060ce20014003200216080009b
:1016cc00420020000f22af00feff37003060800088
:1016dc000000e000070032000000e90006acb70093
:1016ec003140780010e2b7000201e900f5ff3a0042
:1016fc0002003700042cef00010037002160880045
:10170c004f0178004f00be00004006000000200092
:10171c00406088004f0178004f00be00004006007a
:10172c00080ce200feff3a008d40a9008100e900a0
:10173c0031608800b04078008110880020608800fb
:10174c0011002000416088008d40a80000000600b8
:10175c004060800000000600809fbe008520a9002c
:10176c000e22a9000e02ab000800320000608000bf
:10177c00f03fb200018020008100400012c2bf0087
:10178c0080487800002cec00f6ff37004f00be00bc
:10179c0000400600006080001160800001005000d5
:1017ac000000060001608000126080000208e10069
:1017bc0008003200f23fb20001802000028140009c
:1017cc009240780001487800022cec0010002000b8
:1017dc00000006000000eb000000060000a0fe0068
:1017ec0086a0a9001421ef0000000000c1ec8000cd
:1017fc00c2d9210013002000321ce1000500320088
:10180c00080035000000000000000000000000008f
:10181c00f9ff3700a01680004800de0080587800e1
:10182c00f5ff3700c1ec88000a2cec0050608000fa
:10183c000c0ce30003003a0010002000d0ec8800f0
:10184c001fe1a9000080fe00004006000c22ef0002
:10185c000e22ef000ee2a9000ec2a9008520a900fd
:10186c008d20a8000de2a80070002000a0108800b8
:10187c008540a9008d40a80081e0a900c00480002b
:10188c00f1002f0000806000015520000080400016
:10189c00c00488000fe2a8000f42a800002cef0043
:0818ac00022cef000000060011
:020000040000fa
:0200000400fffb
:10e000000000000000000000000000000000000010
:10e010000000000000000000000000000000000000
:10e0200000000000000000000000000000000000f0
:10e0300000000000000000000000000000000000e0
:020000040000fa
:0200000400fffb
:04f00000000000000c
:00000001FF
